S018000066726F6E745F646F6F725F626F6172642E7372656369
S3150802000000000A20C5AA0208419502084995020875
S3150802001051950208599502086195020815AB02081E
S3150802002000000000000000000000000015AB0208F6
S31508020030699502080000000041030208E10202086D
S3150802004015AB020815AB020815AB020815AB020878
S3150802005015AB020815AB020815AB020815AB020868
S3150802006015AB020815AB020815AB020815AB020858
S3150802007015AB020815AB020815AB020815AB020848
S3150802008015AB020815AB020815AB020815AB020838
S3150802009015AB020815AB020815AB020815AB020828
S315080200A015AB020815AB020815AB020879950208CA
S315080200B015AB020815AB020815AB020815AB020808
S315080200C015AB020815AB020815AB020815AB0208F8
S315080200D00000000015AB020815AB02088D95020850
S315080200E015AB020815AB020815AB020815AB0208D8
S315080200F015AB020815AB020815AB020815AB0208C8
S3150802010015AB0208A195020815AB020815AB020841
S3150802011015AB020815AB020815AB020815AB0208A7
S3150802012015AB020815AB0208B595020815AB02080D
S3150802013015AB0208C9950208DD95020815AB020837
S3150802014015AB020815AB020815AB020815AB020877
S3150802015015AB020815AB020815AB020815AB020867
S3150802016015AB020815AB020815AB020815AB020857
S3150802017015AB020815AB020815AB020815AB020847
S3150802018015AB020815AB0208F195020815AB020871
S3150802019015AB020815AB020815AB020815AB020827
S315080201A015AB020815AB020815AB020815AB020817
S315080201B015AB020815AB020815AB020815AB020807
S315080201C015AB020815AB020815AB020815AB0208F7
S315080201D015AB020815AB020815AB020815AB0208E7
S315080201E015AB020815AB020815AB020815AB0208D7
S315080201F015AB020815AB020815AB020815AB0208C7
S3150802020015AB020815AB020815AB02080000000080
S315080202100000000015AB02080000000015AB02083A
S3150802022015AB020815AB020815AB020815AB020896
S3150802023015AB020815AB020815AB020815AB020886
S3150802024015AB020815AB020815AB02080000000040
S3150802025010B5054C237833B9044B13B10448AFF3F0
S3150802026000800123237010BD6809002000000000E9
S31508020270A840040808B5034B1BB103490348AFF36A
S31508020280008008BD000000006C090020A840040890
S3150802029072B64FF0E0201749C0F8081D16480168E3
S315080202A041F00101016015481249096801604FF0E1
S315080202B0E020134941614FF0070101614FF0000147
S315080202C0C0F8181D4FF07F41C0F81C1D0D49C0F833
S315080202D0201D7047FFF7FEBF01B5BDE80140704714
S315080202E001B500F09DF8BDE801407047FFF7FEBF73
S315080202F0FFF7FEBF00000208001000E008CF00204A
S315080203008FD003000000FF40EFF3108180F31088BE
S31508020310081C70474FF000002D4A1060EFF3148056
S3150802032020F0040080F3148862B64FF080504FF034
S31508020330E021C1F8040DBFF34F8FBFF36F8FFEE7BD
S315080203402448254A4FF00003016891B10360EFF390
S31508020350098C2CE9F00F1EF0100F01D12CED108A32
S315080203601E4C4CF804EDC1F808C025680DB18D6124
S31508020370236072B61168D1B1016062B64F68174C34
S315080203808D6907F101074F602560D1F80CC08CF31F
S315080203900B88D1F808C05CF804EB1EF0100F01D1E7
S315080203A0BCEC108ABCE8F00F8CF30988704772B669
S315080203B01168016009B962B6F9E74FF000674FF0B4
S315080203C0E028C8F8047D62B6D8E700BF7047000087
S315080203D0A4CF00200CCF002010CF002010D500207B
S315080203E0026922F00702A2F144026FF04303136086
S315080203F04FF0000353609360D360136153619361B6
S31508020400D361136253629362D362136353634FF0E9
S31508020410FF339363D1634FF080731364826070472E
S315080204202249086800F101000860214B1A683AB1AE
S31508020430A2F101021A601AB91E4B4FF001001860A8
S315080204401D490868026822B11C4B4FF001021A6066
S3150802045008E000F104001A4B1A68904201D1194BC0
S3150802046018680860134B1A6812B914490868C8B1A3
S3150802047001B51249086808B119F020FC0D4B1A6833
S3150802048072B119F08DFB1048016849B90F48016825
S315080204900F4A13680F484FF08052994200D0026003
S315080204A0BDE80140BFF34F8F70470000B0CF002070
S315080204B010D50020B4CF002040D0002044D0002020
S315080204C03CD0002038D00020A4CF00200CCF00203A
S315080204D010CF002004ED00E0034613F8012B002A92
S315080204E0FBD1181A0138704781F0004102E000BFBB
S315080204F083F0004330B54FEA41044FEA430594EAD4
S31508020500050F08BF90EA020F1FBF54EA000C55EA0E
S31508020510020C7FEA645C7FEA655C00F0E2804FEADF
S315080205205454D4EB5555B8BF6D420CDD2C4480EAC1
S31508020530020281EA030382EA000083EA010180EAF1
S31508020540020281EA0303362D88BF30BD11F0004F3F
S315080205504FEA01314FF4801C4CEA113102D0404275
S3150802056061EB410113F0004F4FEA03334CEA1333B0
S3150802057002D0524263EB430394EA050F00F0A780C8
S31508020580A4F10104D5F1200E0DDB02FA0EFC22FAC3
S3150802059005F2801841F1000103FA0EF2801843FAB7
S315080205A005F359410EE0A5F120050EF1200E012AA8
S315080205B003FA0EFC28BF4CF0020C43FA05F3C018E6
S315080205C051EBE37101F0004507D54FF0000EDCF15F
S315080205D0000C7EEB00006EEB0101B1F5801F1BD308
S315080205E0B1F5001F0CD349085FEA30004FEA3C0C0C
S315080205F004F101044FEA445212F5800F80F09A8002
S31508020600BCF1004F08BF5FEA500C50F1000041EB05
S31508020610045141EA050130BD5FEA4C0C404141EB09
S315080206200101013C28BFB1F5801FE9D291F0000F04
S3150802063004BF01460020B1FA81F308BF2033A3F1B3
S315080206400B03B3F120020CDA0C3208DD02F1140CAA
S31508020650C2F10C0201FA0CF021FA02F10CE002F1E5
S315080206601402D8BFC2F1200C01FA02F120FA0CFCDE
S31508020670DCBF41EA0C019040E41AA2BF01EB045127
S31508020680294330BD6FEA04041F3C1CDA0C340EDC25
S3150802069004F11404C4F1200220FA04F001FA02F368
S315080206A040EA030021FA04F345EA030130BDC4F126
S315080206B00C04C4F1200220FA02F001FA04F340EA1B
S315080206C00300294630BD21FA04F0294630BD94F0CC
S315080206D0000F83F4801306BF81F480110134013DB3
S315080206E04EE77FEA645C18BF7FEA655C29D094EA24
S315080206F0050F08BF90EA020F05D054EA000C04BFA2
S315080207001946104630BD91EA030F1EBF002100208C
S3150802071030BD5FEA545C05D14000494128BF41F02B
S31508020720004130BD14F580043CBF01F5801130BD8F
S3150802073001F0004545F0FE4141F470014FF000001A
S3150802074030BD7FEA645C1ABF194610467FEA655CCB
S315080207501CBF0B46024650EA013406BF52EA03356D
S3150802076091EA030F41F4002130BD00BF90F0000F5B
S3150802077004BF0021704730B54FF4806404F1320497
S315080207804FF000054FF0000150E700BF90F0000F50
S3150802079004BF0021704730B54FF4806404F1320477
S315080207A010F0004548BF40424FF000013EE700BF47
S315080207B042004FEAE2014FEA31014FEA02701FBFD7
S315080207C012F07F4393F07F4F81F06051704732F009
S315080207D07F4208BF704793F07F4F04BF41F4002160
S315080207E0704730B54FF4607401F0004521F00041BE
S315080207F01CE700BF50EA010208BF704730B54FF048
S3150802080000050AE050EA010208BF704730B511F048
S31508020810004502D5404261EB41014FF4806404F180
S3150802082032045FEA915C3FF4D8AE4FF003025FEA06
S31508020830DC0C18BF03325FEADC0C18BF033202EB8A
S31508020840DC02C2F1200300FA03FC20FA02F001FAE4
S3150802085003FE40EA0E0021FA02F11444BDE600BF87
S3150802086070B54FF0FF0C4CF4E06C1CEA11541DBF36
S315080208701CEA135594EA0C0F95EA0C0F00F0DEF801
S315080208802C4481EA030621EA4C5123EA4C5350EAE6
S31508020890013518BF52EA033541F4801143F4801337
S315080208A038D0A0FB02CE4FF00005E1FB02E506F0C8
S315080208B00042E0FB03E54FF00006E1FB03569CF01D
S315080208C0000F18BF4EF0010EA4F1FF04B6F5007F23
S315080208D064F5407404D25FEA4E0E6D4146EB060695
S315080208E042EAC62141EA55514FEAC52040EA5E501E
S315080208F04FEACE2EB4F1FD0C88BFBCF5E06F1ED8C8
S31508020900BEF1004F08BF5FEA500E50F1000041EBFE
S31508020910045170BD06F0004646EA010140EA0200AB
S3150802092081EA0301B4EB5C04C2BFD4EB0C0541EACD
S31508020930045170BD41F480114FF0000E013C00F3E2
S31508020940AB8014F1360FDEBF002001F0004170BD06
S31508020950C4F10004203C35DA0C341BDC04F114041F
S31508020960C4F1200500FA05F320FA04F001FA05F2AB
S3150802097040EA020001F0004221F0004110EBD37078
S3150802098021FA04F642EB06015EEA430E08BF20EAA4
S31508020990D37070BDC4F10C04C4F1200500FA04F347
S315080209A020FA05F001FA04F240EA020001F00041D9
S315080209B010EBD37041F100015EEA430E08BF20EA4C
S315080209C0D37070BDC4F1200500FA05F24EEA020E94
S315080209D020FA04F301FA05F243EA020321FA04F0C3
S315080209E001F0004121FA04F220EA020000EBD3707A
S315080209F05EEA430E08BF20EAD37070BD94F0000F7A
S31508020A000FD101F00046400041EB010111F4801FAD
S31508020A1008BF013CF7D041EA060195F0000F18BF5E
S31508020A20704703F00046520043EB030313F4801F9A
S31508020A3008BF013DF7D043EA0603704794EA0C0F54
S31508020A400CEA135518BF95EA0C0F0CD050EA41066A
S31508020A5018BF52EA4306D1D181EA030101F00041E7
S31508020A604FF0000070BD50EA410606BF104619460F
S31508020A7052EA430619D094EA0C0F02D150EA01361B
S31508020A8013D195EA0C0F05D152EA03361CBF10465C
S31508020A9019460AD181EA030101F0004141F0FE41FB
S31508020AA041F470014FF0000070BD41F0FE4141F47F
S31508020AB0780170BD70B54FF0FF0C4CF4E06C1CEA7F
S31508020AC011541DBF1CEA135594EA0C0F95EA0C0F34
S31508020AD000F0A7F8A4EB050481EA030E52EA0335EF
S31508020AE04FEA013100F088804FEA03334FF0805510
S31508020AF045EA131343EA12634FEA022245EA11153D
S31508020B0045EA10654FEA00260EF000419D4208BFED
S31508020B10964244F1FD0404F5407402D25B084FEA9A
S31508020B203202B61A65EB03055B084FEA32024FF446
S31508020B3080104FF4002CB6EB020E75EB030E22BFA3
S31508020B40B61A754640EA0C005B084FEA3202B6EB63
S31508020B50020E75EB030E22BFB61A754640EA5C0012
S31508020B605B084FEA3202B6EB020E75EB030E22BFA2
S31508020B70B61A754640EA9C005B084FEA3202B6EBA3
S31508020B80020E75EB030E22BFB61A754640EADC0062
S31508020B9055EA060E18D04FEA051545EA16754FEAC4
S31508020BA006164FEAC30343EA52734FEAC2025FEAE2
S31508020BB01C1CC0D111F4801F0BD141EA00014FF071
S31508020BC000004FF0004CB6E711F4801F04BF014342
S31508020BD00020B4F1FD0C88BFBCF5E06F3FF6AFAE5E
S31508020BE0B5EB030C04BFB6EB020C5FEA500C50F1EE
S31508020BF0000041EB045170BD0EF0004E4EEA113171
S31508020C0014EB5C04C2BFD4EB0C0541EA045170BD77
S31508020C1041F480114FF0000E013C90E645EA060EBB
S31508020C208DE60CEA135594EA0C0F08BF95EA0C0FE9
S31508020C303FF43BAF94EA0C0F0AD150EA01347FF431
S31508020C4034AF95EA0C0F7FF425AF104619462CE708
S31508020C5095EA0C0F06D152EA03353FF4FDAE10466B
S31508020C60194622E750EA410618BF52EA43067FF4BC
S31508020C70C5AE50EA41047FF40DAF52EA43057FF44C
S31508020C80EBAE12E74FF0FF3C06E000BF4FF0010C57
S31508020C9002E000BF4FF0010C4DF804CD4FEA410CBB
S31508020CA07FEA6C5C4FEA430C18BF7FEA6C5C1BD088
S31508020CB001B050EA410C0CBF52EA430C91EA030F09
S31508020CC002BF90EA020F0020704710F1000F91EA66
S31508020CD0030F58BF994208BF90422CBFD8176FEA34
S31508020CE0E37040F0010070474FEA410C7FEA6C5C02
S31508020CF002D150EA013C07D14FEA430C7FEA6C5C09
S31508020D00D6D152EA033CD3D05DF8040B704700BF34
S31508020D108446104662468C461946634600E000BF82
S31508020D2001B5FFF7B7FF002848BF10F1000F01BD54
S31508020D304DF808EDFFF7F4FF0CBF012000205DF81F
S31508020D4008FB00BF4DF808EDFFF7EAFF34BF0120A4
S31508020D5000205DF808FB00BF4DF808EDFFF7E0FF3D
S31508020D6094BF012000205DF808FB00BF4DF808ED8E
S31508020D70FFF7CEFF94BF012000205DF808FB00BFF5
S31508020D804DF808EDFFF7C4FF34BF012000205DF8D7
S31508020D9008FB00BF4FEA410C7FEA6C5C02D150EABD
S31508020DA0013C0AD14FEA430C7FEA6C5C02D152EA53
S31508020DB0033C02D14FF0000070474FF00100704724
S31508020DC04FEA410212F5001215D211D56FF4787363
S31508020DD0B3EB625212D94FEAC12343F0004343EA06
S31508020DE0505311F0004F23FA02F018BF40427047E1
S31508020DF04FF00000704750EA013005D111F000406B
S31508020E0008BF6FF0004070474FF00000704700BF00
S31508020E104A0011D212F5001211D20DD56FF4787369
S31508020E20B3EB62520ED44FEAC12343F0004343EABE
S31508020E30505323FA02F070474FF00000704750EA09
S31508020E40013002D14FF0FF3070474FF00000704773
S31508020E504FEA4102B2F1E04324BFB3F5001CDCF1CC
S31508020E60FE5C0DD901F0004C4FEAC0024CEA507004
S31508020E70B2F1004F40EB830008BF20F00100704733
S31508020E8011F0804F21D113F13872BCBF01F0004036
S31508020E90704741F480114FEA5252C2F11802C2F168
S31508020EA0200C10FA0CF320FA02F018BF40F00100E9
S31508020EB04FEAC1234FEAD32303FA0CFC40EA0C009B
S31508020EC023FA02F34FEA4303CCE77FEA625307D1D8
S31508020ED050EA01331EBF4FF0FE4040F4400070470F
S31508020EE001F0004040F0FE4040F40000704700BFA9
S31508020EF053B94AB9002908BF00281CBF4FF0FF3171
S31508020F004FF0FF3000F0B4B9ADF1080C6DE904CE2C
S31508020F1000F03CF8DDF804E0DDE9022304B070478E
S31508020F2038B50022002304460D46FFF70BFF28B901
S31508020F3020462946BDE8384000F00AB8204605F1A1
S31508020F40004100F005F8404261EB410138BD00BF9F
S31508020F50D0B500220B4B06460F46FFF781FCFFF77A
S31508020F6057FF0446FFF702FC0022074BFFF778FCFF
S31508020F7002460B4630463946FFF7BAFAFFF748FFEC
S31508020F802146D0BD0000F03D0000F0412DE9F04FAA
S31508020F90099D0C46002B4DD18A420F468446964639
S31508020FA0B2FA82F360D94BB102FA03FEC3F1200208
S31508020FB09F4000FA03FC20FA02F217434FEA1E4644
S31508020FC01FFA8EF44FEA1C42B7FBF6F106FB1177BD
S31508020FD001FB04F042EA0742904208D91EEB0202DC
S31508020FE001F1FF3702D2904200F22D813946121AD8
S31508020FF01FFA8CFCB2FBF6F006FB102200FB04F487
S315080210004CEA024C644508D91EEB0C0C00F1FF327F
S3150802101002D2644500F21A81104640EA0140ACEB5E
S31508021020040C002125B12CFA03F30022C5E900328B
S31508021030BDE8F08F8B4205D90DB1C5E90001002143
S315080210400846F5E7B3FA83F100294DD1A342C0F069
S31508021050F280904280F0EF80064623460846002D2D
S31508021060E6D0C5E90063E3E7002B40F0A2808A1ABE
S315080210704FEA1E471FFA8EF60121B2FBF7F407FB69
S3150802108014204FEA1C4242EA004206FB04F0904250
S315080210900FD91EEB020204F1FF382CBF4FF00109EB
S315080210A04FF00009904203D9B9F1000F00F0C88049
S315080210B04446121A1FFA8CFCB2FBF7F007FB102201
S315080210C000FB06F64CEA024C664508D91EEB0C0CE8
S315080210D000F1FF3202D2664500F2BB801046ACEB45
S315080210E0060C40EA04409DE7C1F120068B4004FA4B
S315080210F001FE22FA06F720FA06FCF4408A401F434C
S315080211004EEA0C0300FA01FE4FEA17484FEA134962
S315080211101FFA87FCB4FBF8F008FB104449EA0444BA
S3150802112000FB0CF9A1450ED93C1900F1FF3A2CBF78
S315080211304FF0010B4FF0000BA14503D9BBF1000F8D
S3150802114000F093805046A4EB09041FFA83F9B4FB16
S31508021150F8F308FB134403FB0CFC49EA0444A445D0
S3150802116006D93C1903F1FF3801D2A4457AD8434679
S3150802117043EA0040A4EB0C04A0FB02984445CC4683
S31508021180434602D306D1CE4504D20138B9EB020C46
S3150802119068EB07035DB1BEEB0C0264EB030404FAC9
S315080211A006F622FA01F3CC401E43C5E90064002183
S315080211B03EE702FA03FEC3F1200104FA03F200FA3B
S315080211C003FCCC404FEA1E4720FA01F11FFA8EF6BD
S315080211D0B4FBF7F00A4307FB1044110C41EA044139
S315080211E000FB06F48C420ED91EEB010100F1FF3812
S315080211F02CBF4FF001094FF000098C4202D9B9F110
S31508021200000F2CD04046091B92B2B1FBF7F407FB3C
S31508021210141142EA014204FB06F1914207D91EEB78
S31508021220020204F1FF3801D2914215D84446521AF5
S3150802123044EA004121E7861A64EB030301200EE71C
S31508021240023C724435E702397244D0E6F444023865
S31508021250E3E6F444023842E7023C7244E7E702381E
S315080212607144D0E7023B3C4482E702383C446AE7D1
S31508021270704700BF80B586B002AF78600023FB6076
S31508021280342300934FF4C8430B4A0C490C4818F010
S31508021290BFFF0346002B0AD1094BBB60B86803F0AF
S315080212A047FEF860FB68002B01D000BFFDE700BFD0
S315080212B01037BD4680BD00BF84090020C04004081F
S315080212C0846D002080B400AF034B1B781846BD46D8
S315080212D05DF8047B704700BFB86D002080B483B008
S315080212E000AF0346FB71054AFB79137001231846C2
S315080212F00C37BD465DF8047B704700BFB86D002009
S3150802130080B400AF034B1B781846BD465DF8047BD4
S31508021310704700BFB96D002080B483B000AF0346A2
S31508021320FB71054AFB791370012318460C37BD4633
S315080213305DF8047B704700BFB96D002080B500AF29
S315080213404FF400710A480CF04BF80346002B06D1FD
S315080213500020FFF7C3FF074808F064FF05E00120F5
S31508021360FFF7BCFF044808F05DFF00BF80BD00BF61
S3150802137000080242D4400408F040040880B500AFD1
S315080213804FF480410A480CF02BF80346002B06D18D
S315080213900020FFF7C1FF074808F044FF05E00120D7
S315080213A0FFF7BAFF044808F03DFF00BF80BD00BF43
S315080213B0000C0242084104082041040880B582B0A4
S315080213C000AF0023FB7101210B480CF009F8034614
S315080213D0002B01D10123FB71022107480CF000F80A
S315080213E00346002B02D1FB790233FB71FB791846BF
S315080213F00837BD4680BD00BF000C024280B500AF6B
S31508021400084B1B6863225A630021064813F0A0F8AA
S31508021410044B1B6863229A630421024813F098F866
S3150802142000BF80BDFCC0002080B582B000AF034675
S31508021430FB710A4B1B68FA795A630021074813F0B5
S3150802144087F8064B1B6800229A630421034813F0A7
S31508021450DFF900BF0837BD4680BD00BFFCC00020CB
S3150802146080B500AF084B1B6800225A630021064864
S3150802147013F0CEF9044B1B684B229A6304210248E7
S3150802148013F066F800BF80BDFCC0002080B500AF2F
S31508021490084B1B6863229A630421064813F058F81E
S315080214A0044B1B686322DA630821024813F050F8DA
S315080214B000BF80BDB0C0002080B582B000AF034631
S315080214C0FB710A4B1B6800229A630421074813F032
S315080214D09FF9064B1B68FA79DA630821034813F069
S315080214E037F800BF0837BD4680BD00BFB0C0002030
S315080214F080B500AF084B1B6863229A63042106482D
S3150802150013F026F8044B1B680022DA630821024806
S3150802151013F07EF900BF80BDB0C0002080B400AFD2
S3150802152000BFBD465DF8047B704780B400AF002358
S315080215301846BD465DF8047B704780B400AF0023A9
S315080215401846BD465DF8047B704780B400AF002399
S315080215501846BD465DF8047B704780B400AF002389
S315080215601846BD465DF8047B704780B400AF002379
S315080215701846BD465DF8047B704780B400AF00BFCD
S31508021580BD465DF8047B704780B584B000AF7860CD
S315080215900023FB7300F00EF80346002B01D001234B
S315080215A0FB737B68043B7B60FB7B18461037BD46A2
S315080215B080BD000080B500AF4FF4006105480BF00E
S315080215C00FFF0346002B01D0012300E00023184633
S315080215D080BD00BF00040242B0B594B000AF034616
S315080215E0FB7108F09FF80346184608F097FA034677
S315080215F0002B00F09180FB79002B48D008F092F876
S3150802160003460121184608F0B4FA08F08BF8034697
S315080216100221184608F01CFA08F084F8034602214B
S31508021620184608F001FA034683F00103DBB2002BE1
S3150802163027D007F108030B2118461AF0ACFC07F16C
S315080216400803152118461AF0C1FC07F10C0207F126
S315080216500803114618461BF008F919F097FF0446C5
S3150802166007F10C0318461AF010FE054607F10C039B
S3150802167018461AF016FE03461A46294620461DF053
S3150802168081FF0022042126480BF0C2FE44E0012213
S31508021690042123480BF0BCFE08F044F80346002157
S315080216A0184608F066FA08F03DF80346022118467D
S315080216B008F0F2F908F036F803460221184608F04F
S315080216C0B3F90346002B27D007F108030B21184666
S315080216D01AF061FC07F10803162118461AF076FC7F
S315080216E007F10C0207F10803114618461BF0BDF86C
S315080216F019F04CFF044607F10C0318461AF0C5FD0B
S31508021700054607F10C0318461AF0CBFD03461A469E
S31508021710294620461DF036FF00BF5037BD46B0BDEC
S315080217200004024280B582B000AF07F0FBFF034611
S31508021730184608F061F878601022002178681FF0D0
S31508021740EDF94FF47A7314220549064814F017FC8A
S315080217507B68054A1A6000BF0837BD4680BD00BFD0
S315080217603441040870C200200345434980B588B055
S3150802177000AFF860B9601346FB710023FB610023D2
S315080217803B61BB687B617B69BB610023FB6110E03F
S31508021790FA69FB68134418461BF0D5FE03463B61FB
S315080217A03A69BB691A60BB690433BB61FB690433D6
S315080217B0FB61FB79FA699A42EADB0123184620376C
S315080217C0BD4680BD80B586B000AF07F0ABFF0346C5
S315080217D0184608F011F878611022002178691FF07E
S315080217E09DF93B1D1022002118461FF097F93B1D53
S315080217F0102219460D48FFF7B9FF7B680C4A934237
S3150802180002D0FFF78FFF0CE03B1D102219467869BC
S315080218101FF03BFA4FF47A730F220649064814F072
S31508021820AEFB002318461837BD4680BD00C01F0808
S31508021830034543494C41040870C2002090B589B05B
S3150802184000AF0023FB6107F06DFF0346184607F059
S31508021850D3FF78617B69BB61FE201BF0A3FE0023E0
S31508021860FB6116E0BB693C1D186859689A68DB6813
S315080218700FC4FB6903F1016303F57C233A1D114684
S3150802188018461BF074FEBB691033BB61FB69103343
S31508021890FB61FB690F2BE5D9012318462437BD46A0
S315080218A090BD80B483B000AF78607B681B79184618
S315080218B00C37BD465DF8047B704780B483B000AF31
S315080218C078600B46FB707B68FA781A7100BF0C3792
S315080218D0BD465DF8047B704780B483B000AF78607C
S315080218E07B685B7918460C37BD465DF8047B704702
S315080218F080B483B000AF78600B46FB707B68FA78D9
S315080219005A7100BF0C37BD465DF8047B704780B438
S3150802191083B000AF78607B689B6818460C37BD4673
S315080219205DF8047B704780B483B000AF7860396095
S315080219307B683A689A6000BF0C37BD465DF8047B3F
S315080219407047000080B400AF034B1B681846BD46BB
S315080219505DF8047B704700BFBC6D002080B483B07D
S3150802196000AF7860044A7B68136000BF0C37BD4637
S315080219705DF8047B704700BFBC6D002080B483B05D
S3150802198000AF0346FB71044AFB79137000BF0C379C
S31508021990BD465DF8047B70478982002080B586B013
S315080219A000AFF8600B467A60FB720023FB752B4882
S315080219B008F038FC0023FB7547E0FB7D284A9C218A
S315080219C001FB03F313441B78012B3BD1FB7D9C22BD
S315080219D002FB03F3224A134402331946214808F04C
S315080219E021FC214808F01EFCFB7D9C2202FB03F326
S315080219F018331B4A1344043319461A4808F012FCD2
S31508021A001A4808F00FFCFB7D154A9C2101FB03F3DB
S31508021A1013445C331B782D2B11D0154808F002FCB1
S31508021A20FB7D9C2202FB03F358330D4A134404330D
S31508021A3019460C4808F0F6FB0C4808F0F3FB0B486D
S31508021A4008F0F0FBFB7D0133FB75FB7D0B2BB4D94C
S31508021A5000BF00BF1837BD4680BD00BF5C41040801
S31508021A600000002084410408884104088C410408C7
S31508021A709041040880B586B000AFF8600B467A60DC
S31508021A80FB720023FB75FB7A012B40F288807B6888
S31508021A9003F500730622454918461FF047F8034620
S31508021AA0002B2CD17B6803F500731846FEF714FD4C
S31508021AB00346062B23D1FFF781FC0346FB75FB7D04
S31508021AC0032B70D801A252F823F000BFDD1A0208D0
S31508021AD0E51A0208ED1A0208F51A0208344808F04F
S31508021AE0A1FB0BE0334808F09DFB07E0324808F0FB
S31508021AF099FB03E0314808F095FB00BF53E07B6889
S31508021B0003F5007302222E4918461FF00FF8034602
S31508021B10002B1BD17B6803F500731846FEF7DCFC25
S31508021B200346022B12D1FFF7EBFB0346FB75FB7D3F
S31508021B30002B02D0012B04D035E0224808F072FBB4
S31508021B4003E0214808F06EFB00BF2CE07B6803F532
S31508021B50007305221D4918461EF0E8FF0346002BAE
S31508021B6019D17B6803F500731846FEF7B5FC0346E0
S31508021B70052B10D107F0D6FD0346184607F03CFEA2
S31508021B80034600211846FFF7B3FEFFF757FE104833
S31508021B9008F048FB07E00F4808F044FB03E00D484D
S31508021BA008F040FB00BF1837BD4680BD9C410408BB
S31508021BB0A4410408CC410408DC410408EC410408A9
S31508021BC00C42040810420408284204084042040849
S31508021BD0484204086042040880B588B000AFF8603D
S31508021BE00B467A60FB720023FB610023BB6100236C
S31508021BF0FB75FB7A012B23D97B6803F5007318461C
S31508021C001DF04CFEF861FB69BB61FB69002B13DD15
S31508021C10FB69022B10DC7B6803F5806318461DF00E
S31508021C203DFEF861FB69FB75BB69DBB2FA7D1946B5
S31508021C30012002F096F807E0054808F0F3FA03E0F7
S31508021C40034808F0EFFA00BF2037BD4680BD00BF43
S31508021C506042040880B58AB004AFF8600B467A6021
S31508021C60FB7200237B610023FB740023BB740023F1
S31508021C707B7400233B74FB7A032B6ED97B6803F5CE
S31508021C80007318461DF00AFE78617B69002B60DB3B
S31508021C907B69022B5DDC7B69FB747B6803F58063D9
S31508021CA018461DF0FBFD78617B69BB747B6803F5FA
S31508021CB0C06318461DF0F2FD78617B697B747B6808
S31508021CC003F5006318461DF0E9FD78617B693B74EC
S31508021CD0FB7C012B0ED105F051FB797CBA7C0023E3
S31508021CE00293002301933B7C00930B46072106F0DF
S31508021CF08DF836E0FB7C022B0ED105F03FFB797C92
S31508021D00BA7C00230293002301933B7C00930B4683
S31508021D10072106F0DDF824E005F030FB797CBA7C71
S31508021D2000230293002301933B7C00930B46072171
S31508021D3006F06CF805F022FB797CBA7C0023029344
S31508021D40002301933B7C00930B46072106F0C0F85B
S31508021D5007E0054808F066FA03E0034808F062FA65
S31508021D6000BF1837BD4680BD6042040880B586B0FC
S31508021D7000AFF8600B467A60FB7200237B61FB7A40
S31508021D80002B15D07B6803F5007318461DF086FDF7
S31508021D9078617B69002B0BDB7B69012B08DC07F07A
S31508021DA0C1FC02467B69DBB21946104607F098FE6B
S31508021DB000BF1837BD4680BD80B586B000AFF86053
S31508021DC00B467A60FB7200237B61FB7A012B76D97C
S31508021DD07B6803F5007303223C4918461EF0A6FEEB
S31508021DE00346002B17D17B6803F500731846FEF7E6
S31508021DF073FB0346032B0ED103F09CFA03461946DE
S31508021E00334808F00FFA03F0B1FA03461946314887
S31508021E1008F008FA57E07B6803F5007304222E4996
S31508021E2018461EF083FE0346002B16D17B6803F57F
S31508021E3000731846FEF750FB0346042B0DD103F038
S31508021E40D9FAF0EE407AFDEEE77A17EE903A7B6120
S31508021E507969224808F0E6F935E07B6803F50073EC
S31508021E6004221F4918461EF061FE0346002B0BD1B9
S31508021E707B6803F500731846FEF72EFB0346042B10
S31508021E8002D103F08BFA1EE07B6803F50073032286
S31508021E90144918461EF04AFE0346002B0BD17B68EE
S31508021EA003F500731846FEF717FB0346032B02D108
S31508021EB003F0F2FA07E00C4808F0B4F903E00A481E
S31508021EC008F0B0F900BF1837BD4680BDD0420408F5
S31508021ED0D4420408E0420408F4420408FC42040816
S31508021EE008430408104304086042040880B584B015
S31508021EF000AFF8600B467A60FB72FB7A012B04D1BD
S31508021F00FFF79CFC034808F08DF900BF1037BD4661
S31508021F1080BD00BF1443040890B585B000AF786051
S31508021F200023BB730023FB734FF4A05200211F4802
S31508021F301EF0F4FD07F10E030A221C49786818F010
S31508021F4063FE0346012B2CD10023FB7326E0FB7BA1
S31508021F509C2202FB03F3164A13449C1C1348FEF701
S31508021F60BBFA03461A46114920461EF0DFFD034610
S31508021F70002B10D1FB7B0E4A9C2101FB03F3134471
S31508021F8018331B68B97B094A00209847094808F0A4
S31508021F9049F9012306E0FB7B0133FB73FB7B0B2B21
S31508021FA0D5D9002318461437BD4690BDC06D00200A
S31508021FB0000000208C41040880B582B000AF0346B9
S31508021FC0FB71FB790D2B24D14F4B00221A704F4817
S31508021FD008F028F94E4B1B78002B16D04D48FFF710
S31508021FE09BFF0346012B08D1642200214A481EF0B2
S31508021FF095FD484948481EF032FE454B00221A70A4
S315080220006422002143481EF089FD444808F00AF973
S3150802201075E0FB790A2B03D13B4B00221A706EE05E
S31508022020FB791B2B03D1384B01221A7067E0FB7927
S315080220305B2B07D1344B1B78012B03D1324B02227F
S315080220401A705CE0FB79412B1FD12F4B1B78022BB0
S315080220501BD12D4B00221A702D4B1B78002B4ED10B
S315080220602D492F4808F0DEF82B48FEF735FA0346C5
S31508022070DAB2274B1A706422002126481EF04EFD5A
S31508022080254924481EF0EBFD39E0FB79082B02D0DE
S31508022090FB797F2B16D11C4B00221A701C4B1B781E
S315080220A0002B2CD01A4B1B78013BDAB2184B1A704C
S315080220B0174B1B781A46174B00219954194808F0F2
S315080220C0B1F81CE0124B1B785A1CD1B2104A117097
S315080220D01946104AFB7953540D4B1B78124AA2FB38
S315080220E003125209642101FB02F29B1ADAB2084B67
S315080220F01A70FB7919460D4808F094F8FFE700BFF5
S315080221000837BD4680BD00BF8A8200208C4104087C
S315080221108882002024820020C081002024430408EB
S3150802212084410408284304081F85EB512C430408FC
S3150802213080B58EB008AF78607B687B6100233B610F
S315080221400A220C21184808F02DF903463B6107F1CB
S315080221500C0100234FF48052786917F0E5FF034615
S31508022160002B01D002231AE0FB68B0220692012254
S315080221700592002204920A2203920A2202924FF43C
S315080221808052019200933B69084A0749084818F0A9
S3150802219011FA0346002B01D00E2300E0002318464D
S315080221A01837BD4680BD00BF38430408C53A020841
S315080221B08C82002080B588B004AF07F0B3FAB86005
S315080221C00023FB7300237B60994B1B78002B00F0DE
S315080221D0F584974B1B78032B40F0E481954B1B78CB
S315080221E0042B13DC002BC0F2D684042B00F2D38412
S315080221F001A252F823F000BF17220208532202084E
S31508022200C72202083F230208E7230208FE2B00F032
S31508022210B78100F0C0BC884B41F288321A60854B00
S315080222201B781946844B1B681A46844807F0FAFF3E
S31508022230834807F0F7FF0221B86807F035FBFFF776
S315080222400FF97C4B1B780133DAB27A4B1A7000F01D
S31508022250B5BC794B1B685A1E77490A60012B1DD9F2
S31508022260784B1B78002B00F09884774807F0DAFF42
S315080222700321B86807F018FBFFF7C0F86D4B1B7807
S315080222800133DAB26B4B1A70694B5B684FF47A7298
S3150802229002FB03F3684A136000F090BC0421B86895
S315080222A007F03FFB1BF052F801230422FC211BF026
S315080222B097F8FFF7A3F8654807F0B4FF5D4BFE22CF
S315080222C01A7000F06ABC5C4B1B685A1E5A490A60AF
S315080222D0012B28D9FFF714F80346002B09D0564BD1
S315080222E01B6841F28732934203D8534B41F2883234
S315080222F01A60544B1B78002B03D0FFF77FF800F0C7
S315080223004EBC4D4B1A68524BA3FB02139B0940F66F
S31508022310B83101FB03F3D31A002B40F04084FFF7D0
S315080223209FF800F03CBC434B1B780133DAB2414BB1
S315080223301A70414B41F288321A6000F030BC04210F
S31508022340B86807F0B1FA434807F06CFFB86807F0B7
S3150802235053FA03461846FFF7BFFA0346FF2B09D07E
S31508022360B86807F049FA03461846FFF7B5FA03466E
S31508022370002B08D1384B1B789B00DBB23233DAB21A
S31508022380364B1A7023E0B86807F036FA0346184641
S31508022390FFF7A2FA03461A462F4B1B7819468900FD
S315080223A00B44DBB21344DAB22C4B1A702A4B1B7855
S315080223B0002B0CD0294B1B78002202920022019294
S315080223C00022009201220321B86807F0F0FB234B92
S315080223D01B781846FFF728F8164B1B780133DAB232
S315080223E0144B1A70EAE3144B1B685A1E12490A6008
S315080223F0012B40F2B180104B1B68B3F57A7F45D2A8
S31508022400B86807F0F9F903461846FFF765FA03466E
S31508022410FF2B09D0B86807F0EFF903461846FFF70D
S315080224205BFA0346002B1BD10F23FB731AE000BF8E
S315080224303C830020E983002054070020484304080F
S315080224405043040854830020684304088043040860
S31508022450F119760598430408EA83002051070020FB
S315080224600223FB739C4B1B78FA7B9A420ED99A4B32
S315080224701B780133DAB2984B1A70984B00221A70FD
S31508022480974B41F288321A60FEF7B8FFFEF738FF1B
S315080224900346002B0CD08021B86807F0D9FA8F4B77
S315080224A000221A708E4B41F288321A60FEF7A6FF96
S315080224B08C4B1B78002B00F074838021B86807F0D8
S315080224C0EBFA0521B86807F0EFF90021B86807F0BA
S315080224D028FA854807F0A6FEFEF790FF7F4BFE22F4
S315080224E01A70B86807F088F903461846FFF7F4F930
S315080224F00346FF2B09D0B86807F07EF9034618464B
S31508022500FFF7EAF90346002B1DD1754B1B6840F607
S31508022510AB52934217D8B86807F06EF90246734B66
S315080225201B7819461046FFF7E3F9FFF787F9B868EB
S3150802253007F062F903461846FFF7CEF9034619462D
S315080225406B4807F06FFE6B4B5B684FF47A7202FBBF
S3150802255003F3634A136031E30521B86807F0E1F92A
S315080225601AF0F4FE01230722FC211AF039FFFEF7BE
S3150802257045FF614807F056FE584BFE221A7010E3D3
S31508022580564B00221A705B4B00221A70594B41F2C5
S3150802259088325A60524B41F288321A604E4B0022F8
S315080225A01A700BE3534B1B78022B40F0C7814B4B37
S315080225B01B78042B12DC002BC0F2F582042B00F2E6
S315080225C0F28201A252F823F0E52502088F260208B4
S315080225D01728020841280208AD280208FE2B00F037
S315080225E09B81E0E20421B86807F05EF943490220BC
S315080225F007F05EFBB86807F0FFF803461846FFF7D0
S315080226006BF90346FF2B09D0B86807F0F5F80346BD
S315080226101846FFF761F90346002B08D12E4B1B78A3
S315080226209B00DBB23233DAB2304B1A7023E0B86859
S3150802263007F0E2F803461846FFF74EF903461A462C
S31508022640254B1B78194689000B44DBB21344DAB2D0
S31508022650264B1A70204B1B78002B0CD0234B1B7869
S3150802266000220292002201920022009201220321F4
S31508022670B86807F09CFA1D4B1B781846FEF7D4FE7D
S31508022680164B1B780133DAB2144B1A7096E2144BC6
S315080226901B685A1E12490A60012B40F2A780104B8A
S315080226A01B68B3F57A7F3DD2B86807F0A5F80346EA
S315080226B01846FFF711F90346FF2B09D0B86807F049
S315080226C09BF803461846FFF707F90346002B17D16E
S315080226D00F23FB7316E000BFEA830020E98300207C
S315080226E05407002055830020B043040851070020F0
S315080226F0C84304083C83002080430408984304081E
S315080227000223FB73964B1B78FA7B9A420AD9944B9F
S315080227101B780133DAB2924B1A70924B02221A7064
S31508022720FEF76CFEFEF7ECFD0346002B08D080216F
S31508022730B86807F08DF9FEF761FE8A4B02221A7015
S31508022740894B1B78002B00F030828021B86807F08D
S31508022750A3F90521B86807F0A7F80021B86807F0B9
S31508022760E0F88249022007F0A3FAFEF747FE7D4BFE
S31508022770FE221A70B86807F03FF803461846FFF7B4
S31508022780ABF80346FF2B09D0B86807F035F80346BD
S315080227901846FFF7A1F80346002B1ED1744B1B6897
S315080227A040F6AB52934218D8B86807F025F80246A5
S315080227B0704B1B7819461046FFF79AF8FFF73EF852
S315080227C0B86807F019F803461846FFF785F803466E
S315080227D01A466949022007F06BFA684B5B684FF4A0
S315080227E07A7202FB03F3624A1360E7E10521B868CD
S315080227F007F097F81AF0AAFD01230722FC211AF01E
S31508022800EFFDFEF7FBFD5E49022007F051FA554B34
S31508022810FE221A70C9E1564B4EF660221A605949D1
S31508022820022007F045FA0221B86807F03DF8FEF7DC
S3150802283017FE4C4B1B780133DAB24A4B1A70BDE1CC
S315080228404B4B1B685A1E4A490A60012B19D94E4B33
S315080228501B78002B00F0AB814C49022007F028FABE
S315080228600321B86807F020F8FEF7C8FD3D4B1B7830
S315080228700133DAB23B4B1A703D4B41F288321A6089
S315080228809CE10421B86807F04CF81AF05FFD0123B1
S315080228900422FC211AF0A4FDFEF7B0FD38490220F5
S315080228A007F006FA2F4BFE221A7080E1304B1B689E
S315080228B05A1E2F490A60012B26D9FEF721FD034627
S315080228C0002B09D02A4B1B6841F28732934203D860
S315080228D0274B41F288321A602B4B1B78002B02D009
S315080228E0FEF78CFD65E1224B1A68294BA3FB0213FE
S315080228F09B0940F6B83101FB03F3D31A002B40F0CB
S315080229005881FEF7ADFD54E1164B00221A70184B9A
S3150802291041F288321A604CE1114B00221A70114BAF
S3150802292000221A70154B00221A70144B41F2883293
S315080229305A600F4B41F288321A603FE10F4B1B78FF
S31508022940012B40F03B81074B1B78FE2B00F01481CC
S31508022950FE2B00F33081002B1CD0012B59D02AE123
S31508022960EA830020E983002055830020E043040817
S315080229705407002051070020C84304083C8300205E
S3150802298000440408504304085483002020440408E1
S31508022990F11976058B4B41F288321A608A4B5B7ABB
S315080229A0012B25D106F0BEFE03460421184607F080
S315080229B03BF80346002B1BD006F0B4FE0346102153
S315080229C0184607F031F8034683F00103DBB2002B01
S315080229D00ED006F0A7FE03461021184607F038F86F
S315080229E0784B4EF660221A60784B41F288321A60AA
S315080229F07749022007F05CF90221B86806F054FF0D
S31508022A00FEF72EFD734B1B780133DAB2714B1A703F
S31508022A10D4E06D4B5B7A012B25D106F083FE034683
S31508022A200421184607F000F80346002B1BD006F0CF
S31508022A3079FE03461021184606F0F6FF034683F090
S31508022A400103DBB2002B0ED006F06CFE0346102102
S31508022A50184606F0FDFF5B4B4EF660221A605B4B8A
S31508022A6041F288321A60574B1B685A1E55490A604A
S31508022A70012B68D906F056FE03461021184606F0C1
S31508022A80D3FF0346002B44D0504B1B68002B04D0BF
S31508022A904E4B1B68013B4D4A13604C4B1B68002B7F
S31508022AA037D14D4B1B78002B26D04B4B00221A7080
S31508022AB0FEF7A4FC4949022007F0FAF81CF0A8FF21
S31508022AC00146474B83FB01239A10CB17D21A1346AA
S31508022AD09B0013445B00CA1A531C7B607A684149FF
S31508022AE0022007F0E5F87B684FF47A7202FB03F3DB
S31508022AF01A46364B1A600CE0374B01221A703A49CD
S31508022B00022007F0D5F8FEF7ABFC304B41F28832CB
S31508022B101A60364B1B78002B4FD03549022007F036
S31508022B20C7F80321B86806F0BFFE1021B86806F098
S31508022B30B3FFFEF763FC274BFE221A70214B41F2C4
S31508022B4088321A603AE00421B86806F0EAFE1AF0FA
S31508022B50FDFB01230422FC211AF042FC1021B8686D
S31508022B6006F09AFFFEF74AFC2249022007F0A0F86F
S31508022B70184BFE221A7020E0164B00221A70124BCE
S31508022B8000221A70104B41F288325A600D4B41F2FC
S31508022B9088321A6012E000BF10E000BF0EE000BFE4
S31508022BA00CE000BF0AE000BF08E000BF06E000BF75
S31508022BB004E000BF02E000BF00E000BF00BF10371C
S31508022BC0BD4680BD540700203C83002058070020DC
S31508022BD050430408E98300205C07002040440408A7
S31508022BE0676666665C4404088044040854830020C9
S31508022BF0204404080044040880B586B004AF06F0F1
S31508022C0091FD38600023FB719C4B1B78002B00F06A
S31508022C1054849A4B1B78032B40F0FD81984B1B7802
S31508022C20042B13DC002BC0F23584042B00F2328409
S31508022C3001A252F823F000BF572C0208932C02086F
S31508022C40072D0208792D0208332E0208FE2B00F002
S31508022C50D08100F01FBC8B4B41F288321A60884B38
S31508022C601B781946874B1B681A46874807F0DAFA13
S31508022C70864807F0D7FA0621386806F015FEFEF7E9
S31508022C8037FC7F4B1B780133DAB27D4B1A7000F0A2
S31508022C9014BC7C4B1B685A1E7A490A60012B25D93B
S31508022CA07B4B1B78002B00F0F7830721386806F068
S31508022CB0FBFD784807F0B6FA714B1B781946714B3B
S31508022CC01B681A46704807F0ADFAFEF7DFFB6C4B35
S31508022CD01B780133DAB26A4B1A70684B5B684FF499
S31508022CE07A7202FB03F3674A1360E6E30621386841
S31508022CF006F017FEFEF7CAFB674807F093FA604B21
S31508022D00FE221A70C8E35F4B1B685A1E5D490A60A9
S31508022D10012B26D9FEF7D6FA0346002B09D0594BC2
S31508022D201B6841F28732934203D8564B41F28832E6
S31508022D301A60574B1B78002B02D0FEF7A7FBADE3B0
S31508022D40504B1A68554BA3FB02139B0940F6B83140
S31508022D5001FB03F3D31A002B40F0A083FEF7C8FB4E
S31508022D609CE3474B1B780133DAB2454B1A70454B45
S31508022D7042F6E0621A6091E3414B1B781946414BD1
S31508022D801B681A46404807F04DFA454807F04AFAC2
S31508022D900821386806F088FD386806F02DFD0346D6
S31508022DA01846FEF77EFD0346FF2B09D0386806F063
S31508022DB023FD03461846FEF774FD0346002B08D189
S31508022DC0384B1B780A33DBB29B00DAB2364B1A70E1
S31508022DD023E0386806F010FD03461846FEF761FD43
S31508022DE003461A462F4B1B78194689000B44DBB259
S31508022DF01344DAB22C4B1A702A4B1B78002B0CD0D0
S31508022E00294B1B780022029200220192002200928C
S31508022E1001220421386806F0CAFE234B1B7818469D
S31508022E20FEF74AFB164B1B780133DAB2144B1A70BB
S31508022E3043E3144B1B685A1E12490A60012B40F2DF
S31508022E40CB80104B1B68B3F57A7F45D2386806F0FB
S31508022E50D3FC03461846FEF724FD0346FF2B09D08A
S31508022E60386806F0C9FC03461846FEF71AFD0346FB
S31508022E70002B1BD10F23FB711AE000BF48830020E9
S31508022E80EB83002060070020484304089C4404089A
S31508022E9056830020B4440408D0440408F119760580
S31508022EA0EC440408EC830020500700200223FB713F
S31508022EB0A54B1B78FA799A420ED9A34B1B78013394
S31508022EC0DAB2A14B1A70A14B00221A70A04B41F23A
S31508022ED088321A60FEF7DAFAFEF7F4F90346002B8F
S31508022EE008D09A4B00221A70994B41F288321A601E
S31508022EF0FEF7CCFA974B1B78002B00F0D1820921FA
S31508022F00386806F0D1FC0021386806F00AFD9248B6
S31508022F1007F088F9FEF7BAFA8C4BFE221A7038685F
S31508022F2006F06AFC03461846FEF7BBFC0346FF2B6F
S31508022F3009D0386806F060FC03461846FEF7B1FC6D
S31508022F400346002B3FD106F0EDFB0346184606F072
S31508022F50E5FD0346012B1ED87D4B1B6841F6573209
S31508022F60934230D8386806F047FC02467B4B1B78FA
S31508022F7019461046FEF7A1FCFEF760FC386806F013
S31508022F803BFC03461846FEF78CFC03461946744872
S31508022F9007F048F917E0386806F02EFC02466F4B30
S31508022FA01B7819461046FEF788FCFEF747FC386878
S31508022FB006F022FC03461846FEF773FC034619463A
S31508022FC0674807F02FF9674B5B684FF47A7202FB82
S31508022FD003F35F4A136070E20721386806F0A1FC22
S31508022FE0FEF754FA604807F01DF9584BFE221A708C
S31508022FF056E2564B00221A705A4B00221A70594B47
S3150802300042F6E0625A60524B42F6E0621A604E4B52
S3150802301000221A7051E2534B1B78022B40F0BF81F3
S315080230204A4B1B78042B13DC002BC0F23B82042B81
S3150802303000F2388201A252F823F000BF5930020882
S31508023040013102088D320208B53202080F3302082E
S31508023050FE2B00F0928125E2444807F0E3F80821A6
S31508023060386806F021FC386806F0C6FB034618469F
S31508023070FEF717FC0346FF2B09D0386806F0BCFB9F
S3150802308003461846FEF70DFC0346002B08D12E4BC5
S315080230901B780A33DBB29B00DAB2304B1A7023E094
S315080230A0386806F0A9FB03461846FEF7FAFB0346FC
S315080230B01A46254B1B78194689000B44DBB2134482
S315080230C0DAB2264B1A70204B1B78002B0CD0234BF6
S315080230D01B7800220292002201920022009201220B
S315080230E00421386806F063FD1C4B1B781846FEF768
S315080230F0E3F9164B1B780133DAB2144B1A70DCE18A
S31508023100134B1B685A1E12490A60012B40F2B18002
S315080231100F4B1B68B3F57A7F3CD2386806F06CFB16
S3150802312003461846FEF7BDFB0346FF2B09D038684F
S3150802313006F062FB03461846FEF7B3FB0346002B6E
S3150802314016D10F23FB7115E0EC830020EB830020D8
S315080231506007002057830020044504085007002012
S315080231602045040848830020D0440408EC44040897
S315080231700223FB71AA4B1B78FA799A420AD9A84B01
S315080231801B780133DAB2A64B1A70A64B02221A70C2
S31508023190FEF77CF9FEF796F80346002B04D0FEF7F5
S315080231A075F9A04B02221A709F4B1B78002B00F070
S315080231B07B810921386806F077FB0021386806F01A
S315080231C0B0FB9A4807F02EF8FEF760F9954BFE22F7
S315080231D01A70974B1B7A002B10D004F0CFF840F6E2
S315080231E0B83302930023019399230093002399226B
S315080231F0072104F06DFE0120FEF7EEF9386806F0A5
S31508023200FBFA03461846FEF74CFB0346FF2B09D08A
S31508023210386806F0F1FA03461846FEF742FB0346FB
S31508023220002B1DD1834B1B6841F65732934217D8A0
S31508023230386806F0E1FA02467F4B1B7819461046B3
S31508023240FEF73BFBFEF7FAFA386806F0D5FA0346AC
S315080232501846FEF726FB03461946784806F0E2FFAB
S31508023260734B5B684FF47A7202FB03F3714A13607D
S3150802327023E10721386806F054FBFEF707F9704880
S3150802328006F0D0FF674BFE221A700DE1694B41F238
S3150802329088321A606B4806F0C5FF0621386806F0C0
S315080232A003FBFEF725F95F4B1B780133DAB25D4B58
S315080232B01A7002E15F4B1B685A1E5E490A60012BAF
S315080232C018D9614B1B78002B00F0F080072138686B
S315080232D006F0EAFA5D4806F0A5FFFEF7D7F8514B65
S315080232E01B780133DAB24F4B1A70524B41F28832CD
S315080232F01A60E2E00621386806F013FBFEF7C6F804
S31508023300534806F08FFF474BFE221A70CEE0494B10
S315080233101B685A1E47490A60012B26D9FDF7D2FFB8
S315080233200346002B09D0434B1B6841F2873293426E
S3150802333003D8404B41F288321A60434B1B78002B64
S3150802334002D0FEF7A3F8B3E03A4B1A68414BA3FB47
S3150802335002139B0940F6B83101FB03F3D31A002B7B
S3150802336040F0A680FEF7C4F8A2E02E4B00221A709F
S31508023370304B42F6E0621A609AE0294B00221A7034
S31508023380284B00221A702A4B00221A70284B42F642
S31508023390E0625A60274B42F6E0621A608DE0244BDF
S315080233A01B78012B40F089801E4B1B78FE2B62D0BE
S315080233B0FE2B7FDC002B02D0012B14D07AE01D4BAA
S315080233C041F288321A601F4806F02CFF0621386837
S315080233D006F06AFAFEF78CF8124B1B780133DAB25A
S315080233E0104B1A7069E0134B1B685A1E11490A6082
S315080233F0012B33D9144B1B78002B5DD00721386873
S3150802340006F052FA144806F00DFFFEF73FF8054B90
S31508023410FE221A70074B42F6E0621A604DE000BFC0
S31508023420EC830020EB8300205783002038450408EC
S315080234304883002060070020500700202045040822
S31508023440584504089C44040856830020B4440408DA
S31508023450D0440408F1197605784504080621386827
S3150802346006F05FFAFEF712F8164806F0DBFE164B70
S31508023470FE221A7020E0144B00221A70134B002207
S315080234801A70124B42F6E0625A60114B42F6E0623B
S315080234901A6012E000BF10E000BF0EE000BF0CE0A9
S315080234A000BF0AE000BF08E000BF06E000BF04E074
S315080234B000BF02E000BF00E000BF00BF0837BD46FC
S315080234C080BD00BF58450408EB83002048830020CE
S315080234D060070020B0B584B004AF0121904809F016
S315080234E07FFF0346002B07D18E4B1B7803F001039F
S315080234F0DAB28C4B1A7002E08A4B00221A70022149
S31508023500874809F06DFF0346002B07D1864B1B78C7
S3150802351003F00103DAB2844B1A7002E0824B0022EE
S315080235201A70FEF712F80346002B07D07F4B1B785A
S3150802353003F00103DAB27D4B1A7002E07B4B0022DC
S315080235401A70FEF70AF80346002B07D0784B1B7849
S3150802355003F00103DAB2764B1A7002E0744B0022CA
S315080235601A70FEF702F80346002B07D0714B1B7838
S3150802357003F00103DAB26F4B1A7002E06D4B0022B8
S315080235801A704FF400716C4809F02AFF0346002BA3
S315080235900BD1FDF797FE0346002B02D0674806F0CB
S315080235A041FE0020FDF79AFE0AE0FDF78BFE034670
S315080235B0002B02D1624806F035FE0120FDF78EFE89
S315080235C04FF48041564809F00BFF0346002B0BD1F6
S315080235D0FDF796FE0346002B02D05A4806F022FE55
S315080235E00020FDF799FE0AE0FDF78AFE0346002B46
S315080235F002D1554806F016FE0120FDF78DFE534B03
S315080236001B785A1CD1B2514A1170042B40F2BA8067
S315080236104F4B1B78002B07D006F084F8034601218E
S31508023620184606F0B0F906E006F07CF803460121D2
S31508023630184606F0CDF9474B1B78002B07D006F043
S3150802364071F803460221184606F09DF906E006F0CF
S3150802365069F803460221184606F0BAF93E4B1B786A
S31508023660002B07D006F05EF803460421184606F03A
S315080236708AF906E006F056F803460421184606F0CB
S31508023680A7F9364B1B78002B07D006F04BF80346F2
S315080236900821184606F077F923E006F043F80346B0
S315080236A00821184606F094F906F03CF8034618462F
S315080236B006F070FA0346002B0DD003F05FFE40F6C3
S315080236C0B833029300230193992300930023992286
S315080236D0082104F0FDFB224B00221A600020FDF7A8
S315080236E07BFF124B1B78002B07D006F01BF803460C
S315080236F01021184606F06CF906E006F013F80346A0
S315080237001021184606F03FF9094B1B78002B29D0E1
S3150802371006F008F803464021184606F059F928E04B
S31508023720000C024264070020650700206607002095
S315080237306707002068070020000802429845040827
S31508023740B4450408CC450408E4450408ED83002082
S315080237505483002055830020568300205783002077
S315080237605883002005F0DEFF03464021184606F07E
S315080237700AF9844B00221A70834B01221A70834B72
S3150802378001221A70824B1B685A1C81490A60C72B90
S3150802379025D9804B1A78804B1A70804B1A78804B41
S315080237A01A70804B1A78804B1A70804B1A78804BA5
S315080237B01A7005F0B7FF03460121184606F0BBF951
S315080237C0734B00221A60734B01221A70734B012243
S315080237D01A70744B01221A70744B01221A70FDF783
S315080237E08FFD03461A46734B1B789A4240D0FDF763
S315080237F087FD03461A466F4B1A7001216E4818F068
S31508023800CAFB6C4B1B78002B0FD001216A4818F0B3
S31508023810DDFB05F087FF03460421184606F018F972
S315080238206649022006F044FA0EE00221624818F0C0
S31508023830CDFB05F077FF03460421184606F02CF95E
S315080238405F49022006F034FA5E495B4819F00DF822
S3150802385017F09CFE04465B4818F017FD05465948C2
S3150802386018F01FFD03461A46294620461BF08AFE13
S31508023870FDF728FD03461A46534B1B789A4238D061
S31508023880FDF720FD03461A464F4B1A7002214A4895
S3150802389018F081FB4C4B1B78002B0BD001214648B4
S315080238A018F094FB05F03EFF03460821184606F079
S315080238B0CFF80AE00221404818F088FB05F032FFEB
S315080238C003460821184606F0E7F83E493A4818F032
S315080238D0CCFF17F05BFE04463A4818F0D6FC0546BC
S315080238E0384818F0DEFC03461A46294620461BF0DD
S315080238F049FE05F017FF0346184606F02DF903465A
S31508023900002B3CD005F00EFF03460221184606F0AE
S3150802391026F803461A462D4B1B789A422FD005F0F5
S3150802392001FF03460221184606F019F803461A460D
S31508023930264B1A70CA21264818F07EFB234B1B78A1
S31508023940002B04D00B21224818F091FB03E00C212E
S315080239501F4818F08CFB1F491D4818F0E2FF17F0A4
S3150802396015FE04461B4818F090FC0546194818F03F
S3150802397098FC03461A46294620461BF003FE00BF5A
S31508023980BD46B0BDED83002066070020670700200C
S31508023990F083002064070020548300206907002072
S315080239A0568300206A0700205783002065070020F7
S315080239B055830020F4830020A0830020F8450408DC
S315080239C0044604085C830020F58300206B07002068
S315080239D0A4830020A883002080B584B004AF05F034
S315080239E0A1FE0346184606F0D5F80346002B1CD05E
S315080239F00F4B1B685A1C0E490A604EF65F22934209
S31508023A0013D90020FDF7E8FD03F0B8FC40F6B833F9
S31508023A1002930023019399230093002399220821F4
S31508023A2004F056FA024B00221A6000BFBD4680BD5A
S31508023A3058830020B0B500AF05F074FE0346802116
S31508023A40184605F0F1FF03461A461B4B1B789A42A5
S31508023A502FD005F067FE03468021184605F0E4FFDD
S31508023A6003461A46144B1A70134B1B78002B04D0C4
S31508023A700B21124818F0AAFA03E00C210F4818F095
S31508023A80A5FA01210D4818F086FA0D490B4818F0D7
S31508023A90ECFE17F07BFD0446094818F0F6FB0546CE
S31508023AA0074818F0FEFB03461A46294620461BF02D
S31508023AB069FD00BFB0BD00BFF6830020A0830020C9
S31508023AC05C83002080B584B000AF78607B68FB60B9
S31508023AD041F2883015F092FD05F024FE0346184699
S31508023AE005F08AFE03461846FDF7DBFE034619462D
S31508023AF03A4806F097FBFDF721FCFDF73FFC384BE9
S31508023B001B78002B42D10221364809F069FC03468C
S31508023B101A46354B1A70354B1B78002B0CBF0123FE
S31508023B200023DBB21A46314B1A702F4B1B78002B37
S31508023B300CBF01230023DBB21A462B4B1A702A4B01
S31508023B401B78002B03D0294B1B78002B14D1264B4C
S31508023B501B78002B05D1264B02221A70244B05220C
S31508023B605A60224B1B78002B10D1224B02221A7064
S31508023B70204B0C225A6009E0194B01221A7005F0F3
S31508023B80D1FD03460121184605F08EFEFEF712FB0B
S31508023B90FFF732F8FFF79EFCFFF71EFF104B1B7864
S31508023BA0002B11D1104B1B78002B0DD00F4B1B7815
S31508023BB0002B09D00A4B01221A7005F0B3FD034601
S31508023BC00121184605F070FEFB68DBB2184606F0BE
S31508023BD093FC012015F012FDD8E700BF144604082D
S31508023BE0F7830020000C02425583002057830020E9
S31508023BF03C8300204883002080B58EB008AF7860E9
S31508023C007B687B6100233B613C220F211A4806F040
S31508023C10C9FB03463B6140221849194817F05EF86A
S31508023C2007F10C0100234FF48052786916F07CFAEA
S31508023C300346002B01D002231AE0FB68B022069243
S31508023C4001220592002204920A2203920A22029271
S31508023C504FF48052019200933B690A4A06490A4880
S31508023C6016F0A8FC0346002B01D00E2300E0002321
S31508023C7018461837BD4680BD2C460408088400201D
S31508023C80F8830020654502084884002080B582B082
S31508023C9000AF78600B467B807B881A4679680448B1
S31508023CA017F031FA034618460837BD4680BD00BFED
S31508023CB0F883002080B582B000AF7860796804483E
S31508023CC017F032FA03469BB218460837BD4680BD3E
S31508023CD0F883002080B586B000AF03460A46FB711A
S31508023CE01346BB7101233B72FB797B72BB79BB72AC
S31508023CF0FF233B6107F1080310211846FFF7C6FFA9
S31508023D0000BF1837BD4680BD80B586B000AF0346F2
S31508023D100A46FB711346BB7102233B72FB797B721F
S31508023D20BB79BB72FF233B6107F1080310211846D2
S31508023D30FFF7ACFF00BF1837BD4680BD80B586B019
S31508023D4000AF0346FB7105233B72FB797B7207F1D1
S31508023D50080310211846FFF799FF00BF1837BD461A
S31508023D6080BD80B586B000AF0346FB710B46BB71BA
S31508023D7013467B7104233B72FB797B72BB79BB7258
S31508023D807B793B6107F1080310211846FFF77EFF8E
S31508023D9000BF1837BD4680BD80B586B000AF034662
S31508023DA0FB710B46BB801346BB7106233B72FB793C
S31508023DB07B72BB79BB72BB88BB8207F108031021F1
S31508023DC01846FFF763FF00BF1837BD4680BD80B4AB
S31508023DD083B000AF0346FB71012318460C37BD4674
S31508023DE05DF8047B704780B586B000AF0346FB7169
S31508023DF00023FB7542F228333B610023FB7305F06F
S31508023E0091FCB8605EE0FB79012B2AD10B21B868D8
S31508023E1005F04AFDFB7D002B0AD1FDF786FB03461A
S31508023E20012B02D10123FB7549E00223FB7546E00B
S31508023E30FB7D012B07D1FDF778FB0346002B3ED10C
S31508023E400223FB753BE0FB7D022B38D1FDF76DFBA8
S31508023E500346012B33D10A2015F0D0FBFDF75EFB92
S31508023E6035E0FB79022B2AD10C21B86805F01CFD36
S31508023E70FB7D002B0AD1FDF760FB0346012B02D11D
S31508023E800123FB751BE00223FB7518E0FB7D012B62
S31508023E9007D1FDF752FB0346002B10D10223FB750F
S31508023EA00DE0FB7D022B0AD1FDF747FB0346012BEA
S31508023EB005D10A2015F0A2FBFDF730FB07E0012029
S31508023EC015F09CFB3B695A1E3A61012B9BD83B694C
S31508023ED0002B0CD1FDF722FBFB79012B02D1022321
S31508023EE0FB7304E0FB79022B01D10323FB73FB7BF3
S31508023EF018461837BD4680BD80B584B000AF00238A
S31508023F00FB7342F210737B600023BB7305F00AFC55
S31508023F10B8600E21B86805F0C7FC30E0FB7B002BC1
S31508023F200CD13B1D1846FDF72FFB0346002B02D189
S31508023F300123FB7320E00223FB731DE0FB7B012BAD
S31508023F4009D13B1D1846FDF71FFB0346012B13D16A
S31508023F500223FB7310E0FB7B022B0DD13B1D184697
S31508023F60FDF712FB0346002B06D1FDF706FB0F21D0
S31508023F70B86805F099FC07E0012015F03FFB7B685D
S31508023F805A1E7A60012BC9DC7B68002B03D1FDF728
S31508023F90F4FA0B23BB73BB7B18461037BD4680BDAC
S31508023FA0B0B59AB002AF07F1080383E803001346D7
S31508023FB0FB7143F69823FB6543F69823BB650023FA
S31508023FC0A7F856304EF66023FB6592E0554B1B78F0
S31508023FD0022B03D0534B1B78002B75D105F0A2FB9D
S31508023FE00346184605F054FC0346184618F02AFFFD
S31508023FF00346A7F85630B7F85630002B64D1494B1A
S3150802400000221A7005F08EFB0346184605F030FEAC
S315080240100346DBB2BB72FB7A19463B7B18463B89E1
S31508024020BA7A0192009303460A463F49022005F0EE
S315080240303FFE07F1140207F108031146184619F064
S31508024040ACF817F0CDFA044607F11403184617F030
S3150802405085F9054607F11403184617F08BF9034646
S315080240601A46294620461BF08DFA40F6B833BB6538
S315080240700DE02C4B1B78002B0DD1FB79184606F068
S315080240803BFA642015F0BAFABB6D643BBB65BB6D9F
S31508024090002BEED100E000BFBB6D002B0CD12349EB
S315080240A0022005F005FE19F051F901236522662161
S315080240B019F096F9002331E01A4B1B78022B03D12B
S315080240C01B49022005F0F4FD164B1B78012B04D17F
S315080240D01849022005F0ECFD0FE0FB79184606F0B8
S315080240E00BFA4FF47A7015F089FAFB6DA3F57A7319
S315080240F0FB65FB6D002B7FF469AFFB6D002B0CD1C2
S315080241000D49022005F0D4FD19F020F90123672292
S31508024110662119F065F9002300E001231846603785
S31508024120BD46B0BD04850020A8460408C04604085A
S31508024130E0460408004704081C470408B0B59CB0CA
S3150802414002AF03463A60FB800B467B7141F2883325
S315080241507B664EF660233B66002387F85F300023B2
S3150802416087F85E30FB883B830023BB7607F118028B
S3150802417007F11C031146184617F05BF917F0FCF90C
S31508024180044607F11C03184618F07FF8054607F19E
S315080241901C03184618F085F803461A46294620468F
S315080241A01BF0F0F941F288337B66B94B00221A708C
S315080241B024E0B74B1B78002B15D0B54B1B78012B87
S315080241C004D1B449022005F073FD1AE0B24902206F
S315080241D005F06EFD19F0BAF801230D22FC2119F03B
S315080241E0FFF80023B8E13B68DBB2184606F084F90B
S315080241F0642015F003FA7B6E643B7B667B6E002BAC
S31508024200D7D17B6E002B0CD1A449022005F050FDB4
S3150802421019F09CF801230E22FC2119F0E1F800237B
S315080242209AE19F49022005F043FD9E4B00221A702F
S315080242300623FB7201233B73FB883B819A4B07F1EA
S31508024240080292E803001860043319803B68DBB25F
S315080242501A4607F1080393E80300FFF7A1FE03468F
S31508024260012B01D0002377E147F230537B668F4B4F
S3150802427000221A7024E08D4B1B78002B15D08B4B2D
S315080242801B78022B04D18A49022005F011FD1AE097
S315080242908849022005F00CFD19F058F80123682216
S315080242A0662119F09DF8002356E13B68DBB21846F1
S315080242B006F022F9642015F0A1F97B6E643B7B6651
S315080242C07B6E002BD7D17B6E002B0CD17A4902204C
S315080242D005F0EEFC19F03AF801236622662119F078
S315080242E07FF8002338E1754B00221A704EF66023D8
S315080242F03B66B6E097F85F30002B40F0B7806F4B0D
S315080243001B78022B04D06D4B1B78002B40F09C8047
S315080243106B49022005F0CCFC684B00221A70012377
S315080243203B7505237B750023BB7507F11C0207F154
S3150802433014031146184618F074FE17F051F904468C
S3150802434007F11C03184617F009F8054607F11C037E
S31508024350184617F00FF803461A46294620461BF058
S3150802436011F940F6B8337B660EE0544B1B78002BE6
S315080243700ED13B68DBB2184606F0BEF8642015F08B
S315080243803DF97B6E643B7B667B6E002BEDD100E0CC
S3150802439000BF4A4B1B78012B3AD14A49022005F045
S315080243A087FC44F620637B661FE005F0BBF90346EB
S315080243B0184605F06DFA0346184618F0ECFC034653
S315080243C0052B07D1012387F85F303F49022005F004
S315080243D06FFC0DE03B68DBB2184606F08DF86420E8
S315080243E015F00CF97B6E643B7B667B6E002BDCD189
S315080243F07B6E002B28D13549022005F059FC18F0AE
S31508024400A5FF01236622662118F0EAFF0023A3E02E
S315080244102A4B1B78022B17D12D49022005F048FC9E
S3150802442005F080F90346184605F032FA034618469F
S3150802443018F0B1FC0346012B06D02649022005F0E6
S3150802444037FC012387F85F303B68DBB2184606F073
S3150802445053F84FF47A7015F0D1F83B6EA3F57A73D8
S315080244603B663B6E002B7FF445AF00E000BF3B6E18
S31508024470002B33D11849022005F01AFC18F066FF02
S3150802448001236722662118F0ABFF002364E000BF10
S31508024490F984002038470408504704086847040886
S315080244A08847040804850020FC840020F88400203C
S315080244B0A4470408BC470408D44704080885002012
S315080244C0F4470408184804083448040850480408FD
S315080244D06848040888480408A44804080223FB74A8
S315080244E0FB883B827B79BB7407F11C0207F1100338
S315080244F01146184618F09FFB17F048F8044607F1CC
S315080245001C03184617F0C1FE054607F11C03184698
S3150802451017F0C7FE03461A46294620461BF032F80C
S315080245203B8A1A46BB7C1946FB7C00930B460C4910
S31508024530022005F0BDFB012387F85E3097F85E304E
S31508024540002B01D0012307E018F000FF01230F22F8
S31508024550FC2118F045FF002318466837BD46B0BD52
S31508024560CC480408B0B5A2B004AF78607B683B6754
S315080245700023FB66002387F8773005F0D3F8B86680
S31508024580CD4816F035FC034683F00103DBB2002B57
S3150802459000F0318307F158031846FFF78BFB0346F1
S315080245A0FB66FB6E002B00F03F8397F85830002B12
S315080245B006D097F85830062B02D8C04B01221A703B
S315080245C097F85830013B052B00F20B8301A252F8EB
S315080245D023F000BFED450208AB460208DD47020894
S315080245E015490208B34A0208654B020897F85A3079
S315080245F01846FFF7F8FB034687F8773097F87730BF
S31508024600002B35D197F85A301946AD4805F00AFEFF
S3150802461097F85A30012B04D10B21AA4817F00CFD42
S3150802462007E097F85A30022B03D10C21A54817F058
S3150802463003FD0121A34817F01AFD07F110031946D5
S31508024640A04818F06EF916F0A1FF044607F1100308
S31508024650184617F01AFE054607F11003184617F012
S3150802466020FE03461A46294620461AF08BFF08E022
S3150802467097F85A30194697F877301A46924805F04D
S31508024680D1FD97F877301946B86E05F04AF905F064
S3150802469049F80346184605F0EFF8024697F87730C8
S315080246A01946104617F0A0F8A2E297F85A30012BDD
S315080246B047D1FCF74AFF0346002B03D0082387F8A5
S315080246C0773090E297F85A301846FFF780FB034690
S315080246D087F8773097F87730002B25D17B4805F095
S315080246E0A1FD0121774817F0A7FC0121754817F0AB
S315080246F0BEFC07F110031946724818F012F916F0B3
S3150802470045FF044607F11003184617F0BEFD054695
S3150802471007F11003184617F0C4FD03461A46294640
S3150802472020461AF02FFF05E097F8773019466848B1
S3150802473005F078FD97F877301946B86E05F0F1F866
S3150802474051E297F85A30022B40F04D82FCF705FFEA
S315080247500346002B03D0092387F8773043E297F8FC
S315080247605A301846FFF733FB034687F8773097F82F
S315080247707730002B25D1554805F054FD02215148C2
S3150802478017F05AFC01214F4817F071FC07F1100384
S3150802479019464C4818F0C5F816F0F8FE044607F113
S315080247A01003184617F071FD054607F1100318465F
S315080247B017F077FD03461A46294620461AF0E2FE06
S315080247C005E097F877301946414805F02BFD97F82A
S315080247D077301946B86E05F0A4F804E297F85B300C
S315080247E0002B15D00120FFF7FEFA034687F877302B
S315080247F097F87730002B04D10121364805F012FDCF
S3150802480006E097F877301A460121334805F00AFD83
S3150802481097F85C30002B15D00220FFF7E4FA03461E
S3150802482087F8773097F87730002B04D10221294888
S3150802483005F0F8FC06E097F877301A460221264872
S3150802484005F0F0FC04F06EFF0346184605F014F86E
S31508024850024697F877301946104616F0C5FF97F8BC
S315080248605D30002B16D01D4805F0DCFC0120FFF751
S31508024870AEFA034687F8773097F87730002B03D1DC
S31508024880174805F0CFFC05E097F877301946154822
S3150802489005F0C8FC97F85E30002B2DD00220FFF7F2
S315080248A096FA034687F8773097F87730002B1DD1AA
S315080248B00D4805F0B7FC1FE0F8830020FA840020B3
S315080248C0F04804080C85002008490408244904080D
S315080248D0384904084C49040864490408804904080C
S315080248E090490408A0490408B449040897F877309F
S315080248F01946C54805F096FC04F014FF0346184607
S3150802490004F0BAFF024697F877301946104616F0B1
S315080249106BFF6DE197F85A30012B41D1BB4B1B78DF
S31508024920002B40F062813B6E002B0CD1B74B022262
S315080249301A70B64B0F225A60B44B00221A72B34B46
S3150802494000225A7251E13B6EFD2B0CD1AF4B01226C
S315080249501A70AE4B03225A60AC4B00221A72AB4B4A
S3150802496001225A7241E13B6EFF2B0CD1A74B012261
S315080249701A70A64B03225A60A44B00221A72A34B42
S3150802498001225A7231E1A14B03221A703B6E9F4AE9
S3150802499053609E4B00221A729C4B00225A7224E1E3
S315080249A097F85A30022B40F02081994B1B78002B3E
S315080249B040F01B813B6E002B0CD1954B02221A70DC
S315080249C0934B0C225A60924B00221A72904B002289
S315080249D05A720AE13B6EFE2B0CD18D4B02221A70DB
S315080249E08B4B0C225A608A4B01221A72884B002280
S315080249F05A72FAE03B6EFF2B2DD104F093FE034662
S31508024A00184605F0C7F80346002B17D002F0B6FC85
S31508024A1040F6B833029300230193992300930023A7
S31508024A209922082103F054FA7A4B00221A600020D0
S31508024A30FCF7D2FD40F6B83014F0E0FD744B0122C3
S31508024A401A70734B03225A60714B00221A72704B0A
S31508024A5000225A72C9E004F065FE0346184605F0BC
S31508024A6099F80346002B17D002F088FC40F6B833B3
S31508024A700293002301939923009300239922082184
S31508024A8003F026FA634B00221A600020FCF7A4FD05
S31508024A9040F6B83014F0B2FD5D4B03221A703B6E35
S31508024AA05B4A53605A4B00221A72594B00225A72B9
S31508024AB09BE004F037FE0346184605F02FF8034636
S31508024AC0002B00F09480FFF717FA034687F8773031
S31508024AD097F87730002B09D14F4805F0A3FB07F169
S31508024AE054030121184617F08CFA0BE097F8773031
S31508024AF019464A4805F096FB07F15403022118465F
S31508024B0017F07FFA97F877301946B86E04F009FF5E
S31508024B1004F008FE0346184604F0AEFE024697F86D
S31508024B2077301946104616F05FFE07F1100207F1B4
S31508024B3054031146184617F0D5FE16F027FD04460B
S31508024B4007F11003184617F0A0FB054607F11003F4
S31508024B50184617F0A6FB03461A46294620461AF0B7
S31508024B6011FD44E0B7F8643097F85A103A6F1846C0
S31508024B70FFF7E4FA034687F87730B7F864301A463F
S31508024B8097F85A30194697F8773000930B46244916
S31508024B90022005F08DF897F87730FB73B7F8643082
S31508024BA0BB8197F85A30BB7307F1100207F10C0361
S31508024BB01146184618F03FF816F0E8FC044607F1C5
S31508024BC01003184617F061FB054607F1100318464D
S31508024BD017F067FB03461A46294620461AF0D2FC06
S31508024BE006E000BF04E000BF02E000BF00E000BF2D
S31508024BF00C4B00221A703B6FDBB2184605F07CFCA0
S31508024C00642014F0FBFCBBE4C84904083C8300207A
S31508024C104883002058830020E0490408F449040820
S31508024C20CC480408FA84002000BF7837BD46B0BDD8
S31508024C30B0B594B000AF5C4BD3F8F430002B09DA68
S31508024C405A4805F0EFFA07F148030621184617F005
S31508024C5049F85DE0544BD3F8F43003F08043002B57
S31508024C6009D0534805F0DEFA07F14803052118462C
S31508024C7017F038F84CE04C4BD3F8F43003F00053F5
S31508024C80002B09D04B4805F0CDFA07F14803042159
S31508024C90184617F027F83BE0434BD3F8F43003F0F5
S31508024CA08053002B09D0444805F0BCFA07F14803A3
S31508024CB00321184617F016F82AE03B4BD3F8F430CE
S31508024CC003F00063002B09D03C4805F0ABFA07F164
S31508024CD048030221184617F005F819E0324BD3F8B3
S31508024CE0F43003F08063002B09D0354805F09AFAB0
S31508024CF007F148030121184616F0F4FF08E0314887
S31508024D0005F090FA07F148030021184616F0EAFF63
S31508024D10254BD3F8F430244A43F40003C2F8F4309E
S31508024D20294818F0FBFB03461B0ADAB207F14803C7
S31508024D301146184616F0F1FF234818F0EFFB034612
S31508024D40DAB207F148031146184617F001F81F4B65
S31508024D509A7807F148031146184617F014F81B4BC0
S31508024D60DA7807F148031146184617F027F83A1D6C
S31508024D7007F148031146184617F0CBFC16F006FC55
S31508024D8004463B1D184617F080FA05463B1D184691
S31508024D9017F087FA03461A46294620461AF0F2FB06
S31508024DA000BF5037BD46B0BD000C0244084A04088D
S31508024DB0244A0408404A04085C4A04087C4A04084F
S31508024DC0944A0408AC4A040800E00108E0BF1F0838
S31508024DD0B0B592B000AF114B1A883B461146184639
S31508024DE017F007F83A1D3B461146184617F0D0FC4D
S31508024DF016F0CCFB04463B1D184617F046FA054644
S31508024E003B1D184617F04DFA03461A462946204610
S31508024E101AF0B8FB00BF4837BD46B0BD628700200E
S31508024E20B0B592B000AF04F07DFC0346184604F014
S31508024E3093FE0346002B1DD004F074FC0346184665
S31508024E4004F01AFD02463B1D1946104617F088FA69
S31508024E5016F0AAFB04463B1D184617F016FA054635
S31508024E603B1D184617F01DFA03461A4629462046E0
S31508024E701AF088FB00BF4837BD46B0BDB0B5A2B030
S31508024E8000AF18F063FA0346184618F075FA034697
S31508024E90002B36D03B1D0121184616F0C0FB3B1DE0
S31508024EA00121184616F0D6FB18F050FA03461846A2
S31508024EB018F08AFA02463B1D1146184616F0EAFB16
S31508024EC007F144023B1D1146184616F026FC16F059
S31508024ED091FB044607F14403184616F0EBFB054618
S31508024EE007F14403184616F0F1FB03461A4629460B
S31508024EF020461AF047FB18F029FA0346184618F016
S31508024F0055FA0A4B1B685A1C08490A60632B08D9CA
S31508024F1018F01CFA0346184618F03AFA034B002210
S31508024F201A6000BF8837BD46B0BD00BF648700203F
S31508024F3080B58EB008AF786000237B617B683B61E1
S31508024F4006221021494805F02DFA07F10C01002323
S31508024F504FF48052386915F0E7F80346002B01D062
S31508024F6002237EE0FB68B022069201220592002205
S31508024F7004920A2203920A2202924FF48052019262
S31508024F80009300233A4A3B493B4815F013FB034674
S31508024F90002B01D00E2364E0342300223749384817
S31508024FA015F0D6F90346002B01D01C2359E0786880
S31508024FB005F0B4F97868FEF71FFE7868FDF7B8F8C9
S31508024FC0786804F0A3FF342300222E492E4815F0F0
S31508024FD0BFF90346002B01D01C2342E034230022EA
S31508024FE02A492B4815F0B4F90346002B01D01C2395
S31508024FF037E0342300222749274815F0A9F9034642
S31508025000002B01D01C232CE03423002223492448F8
S3150802501015F09EF90346002B01D01C2321E0342308
S3150802502000222049204815F093F90346002B01D0A7
S315080250301C2316E0342300221C491D4815F088F962
S315080250400346002B01D01C230BE034230022194906
S31508025050194815F07DF90346002B01D01C2300E000
S315080250607B6918461837BD4680BD00BFC84A040882
S31508025070BD500208DC4A040810850020EC4A0408E0
S31508025080C0850020FC4A0408F4850020104B040859
S31508025090288600202C4B04085C860020444B040812
S315080250A0908600205C4B0408C4860020744B0408D2
S315080250B0F8860020884B04082C870020B0B596B0E5
S315080250C000AF78607B683B650023A7F856303B6DD6
S315080250D0DBB21846FCF752FC002387F8553000234A
S315080250E087F8543004F01EFB0346184604F016FDF2
S315080250F0034619466D4805F095F8B7F85630013358
S31508025100A7F8563000F018FF00F086FE00F000FD02
S3150802511000F0B8FE01F026FB19F042FA19F0C2FCBB
S3150802512019F03AFF3B6DDBB2184601F055FFB7F8A6
S3150802513056305F4AA2FB03125209642101FB02F2AE
S315080251409B1A9BB2002B32D13B6DDBB2184604F098
S31508025150DBFF3B6DDBB2184604F050FF19F01AFC70
S3150802516019F092FE1AF006F901F0BEFF19F03CFB9F
S3150802517019F0B4FD1AF028F8FEF75CFC04F0D2FA2E
S315080251800346184604F05DFB0346002B08D004F0DC
S31508025190C9FA03460021184604F05FFBFFF740FEF2
S315080251A0FFF76CFE3B6DDBB2184605F0A5F9B7F8BA
S315080251B05630404AA2FB031252094FF4FA7101FB18
S315080251C002F29B1A9BB2002B01D1FFF729FEB7F810
S315080251D05630384AA2FB031292094FF47A7101FB40
S315080251E002F29B1A9BB2002B40D1334B1B78013338
S315080251F0DAB2314B1A70314B1B8801339AB22F4BF4
S315080252001A8097F85530032B27D197F85430002B7C
S315080252102CD1012387F85430FFF70AFD01233B728C
S3150802522007F10C0207F108031146184617F0D3F9DD
S3150802523016F0ACF9044607F10C03184617F025F8E0
S31508025240054607F10C03184617F02BF803461A46CB
S31508025250294620461AF096F908E097F85530032BA6
S3150802526004D897F85530013387F85530B7F85630D1
S31508025270134AA2FB0312120B43F6982101FB02F210
S315080252809B1A9BB2002B04D10023A7F8563001F0D3
S31508025290EDF9094B1B783B2B04D9074B00221A70F0
S315080252A0FFF796FD012014F0A9F926E7AC4B04088E
S315080252B01F85EB51D34D621060870020628700205C
S315080252C073B2E74580B500AF13F038FA00BF80BD68
S315080252D080B586B004AF00237B60342300221149CF
S315080252E0114815F035F804F01DFA0346184604F07D
S315080252F083FA03461846FCF70AFB7860FCF722FB9A
S3150802530002467B68029301924FF480630093074B2F
S315080253104FF400620549064801F062FD00BF0837EE
S31508025320BD4680BDBC4B040868870020000C0242BB
S315080253309C87002080B500AF024801F099FD03461C
S31508025340184680BD9C87002080B582B000AF034610
S31508025350FB71FB791946044801F0E2FD034618463B
S315080253600837BD4680BD00BF9C87002080B500AFC8
S31508025370024801F06DFD0346184680BD9C87002051
S3150802538080B500AFFCF7DEFA03461946024801F07B
S31508025390EAFD00BF80BD00BF9C87002080B58AB0A9
S315080253A000AF00237B624FF47A71104815F06EF84D
S315080253B00346002B06D10520FFF7C6FF78620B4885
S315080253C015F0BEF8786AFCF7C9FAFFF7D9FF381D57
S315080253D07B6A052206491BF00DFB3B1D184604F0A5
S315080253E021FF00BF2837BD4680BD00BF6887002061
S315080253F0D44B040880B584B000AF4FF00003BB60FD
S315080254004FF00003FB6040F6B831214815F03EF82C
S315080254100346002B0BD10120FFF796FF07EE900AF1
S31508025420F8EEE77AC7ED037A194815F089F8FCF71A
S3150802543089FA07EE900AF8EEE77AC7ED017A04F0E0
S3150802544071F90346184604F0D7F903461846FCF7DD
S315080254505EFA07EE900AF8EEE77AC7ED007A97ED5C
S31508025460037AD7ED017A77EE676A97ED007AC6EE88
S31508025470877A9FED087A67EE877AC7ED027ABB6864
S3150802548007EE903AB0EE670A1037BD4680BD00BFF8
S31508025490688700200000484390B583B000AF002318
S315080254A07B6040F6B831124814F0F0FF0346002B31
S315080254B00BD11E20FFF748FF0446FCF743FA0346C2
S315080254C0E31A7B600A4815F03BF804F02BF9034609
S315080254D0184604F091F9034679681846FCF723FA48
S315080254E07968044804F09EFE00BF0C37BD4690BD9D
S315080254F068870020EC4B040880B400AF034B1B6896
S315080255001846BD465DF8047B704700BFB887002081
S3150802551080B500AF4FF400620E490F4815F0DEFB66
S315080255204FF400620D490E4815F0D8FB4FF400728D
S315080255300C490D4815F0D2FB4FF400620B490C4892
S3150802554015F0CCFB4FF400620A490B4815F0C6FB6E
S3150802555000BF80BDCC870020BC870020DC8F0020DE
S31508025560CC8F00201098002000980020509A002026
S31508025570109A002090A2002050A2002080B483B086
S3150802558000AF78607B68002B01D1002346E07B6878
S31508025590012B01D1012341E07B68022B01D10223B1
S315080255A03CE07B68032B01D1032337E07B68042B9D
S315080255B001D1042332E07B68052B01D105232DE0B6
S315080255C07B68062B01D1062328E07B68072B01D1CD
S315080255D0072323E07B68082B01D108231EE07B689A
S315080255E0092B01D80C2319E07B680A2B01D8102352
S315080255F014E07B680B2B01D814230FE07B680C2B75
S3150802560001D818230AE07B680D2B01D8202305E070
S315080256107B680E2B01D8302300E0402318460C374E
S31508025620BD465DF8047B704780B483B000AF03467D
S31508025630FB80FB88002B01D1002346E0FB88012B67
S3150802564001D1012341E0FB88022B01D102233CE070
S31508025650FB88032B01D1032337E0FB88042B01D1F6
S31508025660042332E0FB88052B01D105232DE0FB88B4
S31508025670062B01D1062328E0FB88072B01D1072335
S3150802568023E0FB88082B01D108231EE0FB880C2B9C
S3150802569001D8092319E0FB88102B01D80A2314E044
S315080256A0FB88142B01D80B230FE0FB88182B01D893
S315080256B00C230AE0FB88202B01D80D2305E0FB8882
S315080256C0302B01D80E2300E00F2318460C37BD46AF
S315080256D05DF8047B7047000084B0B0B400AF07F1F0
S315080256E00C0484E80F00074B1D4607F10C040FCC87
S315080256F00FC50FCC0FC523682B6000BFBD46B0BCD3
S3150802570004B07047DC97002080B586B000AF786099
S315080257100B467B800023FB7500233B610023FB605D
S315080257200023BB6000F03AFD0346002B0BD0444B26
S31508025730D3F844323B61424BD3F8843AFB607B6828
S315080257401B68BB600AE03E4BD3F844323B613C4BD4
S31508025750D3F8843AFB607B681B68BB603A69BB680E
S315080257609A4227D1364B93F86832002B0AD1344B2A
S31508025770D3F850227B881344314AC2F850320123A7
S31508025780FB7558E02E4BB3F86C321A467B881344E5
S31508025790B3F5006F0BDA2A4BB3F86C227B881344F5
S315080257A09AB2274BA3F86C220123FB7543E0002328
S315080257B0FB7540E0FA68BB689A4227D1204B93F8FA
S315080257C0A83A002B0AD11E4BD3F850227B881344E1
S315080257D01B4AC2F850320223FB752CE0184BB3F869
S315080257E0AC3A1A467B881344B3F5006F0BDA144BAE
S315080257F0B3F8AC2A7B8813449AB2114BA3F8AC2AA5
S315080258000223FB7517E00023FB7514E03B69002BA6
S3150802581007D1242279680B481BF037FA0123FB7556
S3150802582009E0FB68002B06D12422796806481BF09A
S315080258302CFA0223FB75FB7D18461837BD4680BD38
S31508025840DC970020209A002060A2002080B584B050
S3150802585000AF03463960FB711346BB800023FB8108
S31508025860FB79012B12D10023FB810AE0FB893A68F6
S31508025870134401221946124815F0D6FAFB89013358
S31508025880FB81FA89BB889A42F0D314E0FB79022B92
S3150802589011D10023FB810AE0FB893A6813440122ED
S315080258A01946084815F0C0FAFB890133FB81FA89C3
S315080258B0BB889A42F0D300BF1037BD4680BD00BFF1
S315080258C0109A002050A2002080B582B000AF03468D
S315080258D0FB71FB1D01221946034815F0A5FA00BF04
S315080258E00837BD4680BD00BF00980020B0B5B6B0E7
S315080258F000AFF860B9607A60002387F8D7300023D2
S3150802590087F8D630F86806F014FCC7F8D0000023EA
S3150802591087F8D73004E097F8D730013387F8D730BD
S315080259200721F86806F01AFD0346002BF3D17A68B8
S31508025930B968F86806F0B9FB0346002B40D097F819
S31508025940D630013387F8D63003F0ECFE0346184604
S3150802595004F0D7F80346002B02D0684804F062FC2C
S31508025960674B1B78012B2BD0654B01221A7007F166
S31508025970C8030622002118461BF0D0F807F1C8030F
S315080259800121184616F0A1FA07F1840207F1C803A5
S315080259901146184616F04AFF15F0F8FD044607F1B7
S315080259A08403184616F071FC054607F18403184667
S315080259B016F077FC03461A462946204619F0E2FDF8
S315080259C097F8D630002B28D14D4B1B78002B24D0C4
S315080259D04B4B00221A7007F1C8030021184616F02D
S315080259E074FA07F1840207F1C8031146184616F03D
S315080259F01DFF15F0CBFD044607F18403184616F081
S31508025A0044FC054607F18403184616F04AFC034689
S31508025A101A462946204619F0B5FDF86800F064FBD7
S31508025A2003461A46374B9A60F86800F027FB034686
S31508025A30344A1360F86800F039FB0346314A53606A
S31508025A40304B9B68002B11D003F06CFE03461846B8
S31508025A5004F057F80346002B08D02A4B1A68294B3C
S31508025A605B6807F1100028491AF0C4FF0C22254981
S31508025A7026481BF043F80346002B36D0214B1B68F9
S31508025A80DAB207F154031146184616F0CDF91D4B42
S31508025A905B68DAB207F154031146184616F0DFF9C5
S31508025AA0184B9B68DAB207F154031146184616F0EA
S31508025AB0F1F907F1100207F154031146184616F0D8
S31508025AC086FE15F063FD044607F11003184616F024
S31508025AD0DCFB054607F11003184616F0E2FB0346FF
S31508025AE01A462946204619F04DFD084B054A07CAAB
S31508025AF083E8070000BFD837BD46B0BD0C4C040882
S31508025B00A8AA002090AA0020304C04089CAA0020CB
S31508025B1080B592B000AF3B464022002118461AF0E3
S31508025B20FDFF0023A7F8423000237B64B44815F032
S31508025B305FF9034683F00103DBB2002B00F0E38032
S31508025B40B04B93F86832002B5FD1AE4BD3F8503284
S31508025B509AB2AC4BA3F86C22AA4B0F22C3F8502276
S31508025B6010233B703B785AB2A64BB3F86C321B0A29
S31508025B709BB25BB203F00F035BB213435BB2DBB2B9
S31508025B803B70A04BB3F86C32DBB27B703B460233F8
S31508025B903E2219469A4815F082F90346002B00F070
S31508025BA02B814FF47A71984814F070FC0346002B47
S31508025BB00AD1FFF7A1FC3B461A469449FFF796FE1F
S31508025BC0914814F0BDFC02E0914804F02BFB8D4B82
S31508025BD0B3F86C323E3B9AB28A4BA3F86C22894BD5
S31508025BE0B3F86A3201339AB2864BA3F86A22854B16
S31508025BF0012283F86822834BFF2283F86E22814BA7
S31508025C004FF4FA62C3F87022F6E07E4B93F86E32CE
S31508025C10002B05D07B4B93F86E32012B40F0EC80BB
S31508025C20784BB3F86C323E2B02D940237B6404E0EE
S31508025C30744BB3F86C3201337B6420233B703B7898
S31508025C405AB2704BB3F86A325BB203F00F035BB217
S31508025C5013435BB2DBB23B707B6C5A1E3B46013385
S31508025C601946674815F01BF90346002B00F0C48055
S31508025C704FF47A71644814F009FC0346002B13D1D9
S31508025C807B6C9BB21846FFF7CFFC03465D4AC2F807
S31508025C905032FFF731FC3B461A465C49FFF726FEAF
S31508025CA0594814F04DFC02E0594804F0BBFA554B2A
S31508025CB0B3F86C227B6C9BB2D31A9BB201339AB2AD
S31508025CC0504BA3F86C224F4BB3F86A3201339AB29F
S31508025CD04C4BA3F86A224B4BB3F86C32002B40F0BC
S31508025CE08B802422002149481AF018FF454B0022CE
S31508025CF083F86822434B0022A3F86A22414BFF220B
S31508025D0083F86E2278E0434815F072F8034683F06A
S31508025D100103DBB2002B6FD03B46012219463D48F0
S31508025D2015F0BDF80346002B63D03B781B09DBB29E
S31508025D30032B1CD13B46013302221946354815F07E
S31508025D40AEF80346002B57D02E4B0322DA604FF4E7
S31508025D507A712D4814F09AFB0346002B4CD1FFF7B3
S31508025D60CBFB3B461A462749FFF7C0FD44E03B7882
S31508025D701B09DBB2002B3FD13B46013301221946F0
S31508025D80244815F08CF80346002B34D03B781B02C6
S31508025D909BB203F47063A7F842307B781A46B7F8C9
S31508025DA042301343A7F84230B7F842203B46023343
S31508025DB01946184815F073F80346002B1CD0B7F895
S31508025DC0423002339BB21846FFF72EFC03460D4AB1
S31508025DD0D3604FF47A710C4814F058FB0346002B33
S31508025DE00AD1FFF789FB3B461A460649FFF77EFDAD
S31508025DF002E000BF00E000BF4837BD4680BD00BFD5
S31508025E00109A0020DC970020F8860020209A0020AD
S31508025E10504C04080098002080B59AB000AF3B4663
S31508025E206822002118461AF079FE0E4814F0E0FF9F
S31508025E30034683F00103DBB2002B0ED004E03B4697
S31508025E406821184600F010F83B46682219460548AC
S31508025E5015F025F80346002BF1D100BF6837BD4679
S31508025E6080BD00BFCC8F002080B582B000AF7860BD
S31508025E700B467B80786800F0FFFB00BF0837BD46FB
S31508025E8080BD000080B500AF174B93F86832002B2F
S31508025E9028D0154B93F86E32FF2B23D1124BD3F829
S31508025EA07032002B07D0104BD3F87032013B0E4AE2
S31508025EB0C2F8703216E0242200210C481AF02EFE8F
S31508025EC04FF400620A490B4814F008FF064B0022F9
S31508025ED083F86822044B0022A3F86A22024BFF22A7
S31508025EE083F86E2200BF80BDDC970020209A00202E
S31508025EF0509A0020109A002080B582B000AF7860D0
S31508025F000B467B80786800F0CFFA00BF0837BD469B
S31508025F1080BD000080B582B000AF78600B467B80FA
S31508025F207B881A467968034814F07EFF00BF083753
S31508025F30BD4680BDBC87002080B59AB000AF3B46FF
S31508025F406822002118461AF0E9FD0E4814F050FF9F
S31508025F50034683F00103DBB2002B0ED004E03B4676
S31508025F6068211846FFF7C8FF3B46682219460548C6
S31508025F7014F095FF0346002BF1D100BF6837BD46E2
S31508025F8080BD00BFBC87002080B582B000AF7860B4
S31508025F900B4A7B681360FFF7BBFA242200210948E3
S31508025FA01AF0BCFD2422002107481AF0B7FD242264
S31508025FB0002106481AF0B2FD00BF0837BD4680BD6B
S31508025FC0B8870020DC970020209A002060A20020D3
S31508025FD080B58AB002AF78600B467B8013463B8059
S31508025FE00023BB600023FB607B683B6101237B6166
S31508025FF07B88BB613B88FB610A4B1B6807F1080279
S315080260001146184605F09EFF064B186801230093B1
S3150802601001230222022105F0EFFF00BF2037BD4609
S3150802602080BD00BFB887002080B58CB002AFF8608B
S31508026030B9607A604FF080433B6100237B61FB685D
S31508026040BB610123FB61BB683B627B687B620A4BCF
S315080260501B6807F110021146184605F073FF064B36
S3150802606018680123009301230222022105F0C4FFC6
S3150802607000BF2837BD4680BDB887002080B485B0EA
S3150802608000AF78607B681B681B6CBB600023FB60F3
S31508026090BB68DBB2002B02D0BB68DBB2FB60FB68D5
S315080260A018461437BD465DF8047B704780B485B040
S315080260B000AF78607B681B681B6CBB600023FB60C3
S315080260C0BB6803F4FE43002B06D0BB6803F4FE4309
S315080260D0FB60FB681B0AFB60FB6818461437BD4663
S315080260E05DF8047B7047000080B485B000AF786025
S315080260F07B681B685B6CBB600023FB60BB6803F0B4
S315080261000703002B2FD0BB6803F00703013B052BBF
S3150802611020D801A252F823F0316102083761020839
S315080261203D61020843610208496102084F6102089B
S315080261300123FB600FE00223FB600CE00323FB60F4
S3150802614009E00423FB6006E00523FB6003E006235F
S31508026150FB6000E000BF7B681B685A6C7B681B68A3
S3150802616022F007025A64FB68DBB218461437BD46AA
S315080261705DF8047B704700BF80B483B000AF034666
S31508026180FB71054AFB791370012318460C37BD4685
S315080261905DF8047B704700BF6C07002080B400AF2F
S315080261A0034B1B781846BD465DF8047B704700BF53
S315080261B06C07002080B500AFFFF7F0FF0346002BFF
S315080261C002D04FF4807301E04FF48073184680BD05
S315080261D080B500AFFFF7E2FF0346002B02D04FF46B
S315080261E0005301E04FF40053184680BD80B500AF56
S315080261F0FFF7D4FF0346002B02D040F2051301E055
S3150802620040F20513184680BDB0B5A4B006AFF860D3
S31508026210B9601346FB800023A7F87630FB683B6516
S31508026220FFF7BCFF0346002B03D04FF080437B6584
S3150802623001E000237B650023BB65FB8802339BB222
S315080262401846FFF7F1F90346FB6500233B664FF450
S3150802625080137B664FF40013BB660023FB6600239C
S315080262603B6700233B743B7C5AB2FB881B0A9BB2F2
S315080262705BB203F00F035BB213435BB2DBB23B7450
S31508026280FB88DBB27B740223A7F8763010E0B7F8F6
S315080262907630023BBA681A44B7F876301278783301
S315080262A03B4403F8682CB7F876300133A7F8763002
S315080262B0B7F87620FB8801339A42E8DD0023A7F86F
S315080262C076300DE0B7F8763078333B4413F8683CFD
S315080262D01846FFF7F9FAB7F876300133A7F8763099
S315080262E0B7F87620FB8801339A42EBDD6D4607F153
S315080262F060040FCC0FC523682B6007F150030FCB40
S31508026300FFF7EAF900BF7837BD46B0BD80B58EB053
S3150802631000AFF860B9601346FB80002387F8373070
S31508026320FB683B61FFF73AFF0346002B03D04FF0A9
S3150802633080437B6101E000237B610023BB61FB880C
S31508026340FB6100233B624FF480137B624FF4001318
S31508026350BB620023FB6200233B63FA8807F1100342
S3150802636011461846FFF7D0F9034687F8373097F8EB
S315080263703730002B06D0FA8897F83730B9681846AE
S31508026380FFF764FA00BF3837BD4680BDB0B5A2B084
S3150802639006AF7860084611461A460346FB700B4656
S315080263A0BB7013467B70002387F86F307B68BB642B
S315080263B0FFF7F4FE0346002B03D04FF08043FB643D
S315080263C001E00023FB6400233B6503237B6500236E
S315080263D0BB654FF48013FB654FF400133B6600233D
S315080263E07B660023BB6630233B723B7A5AB297F927
S315080263F0033003F00F035BB213435BB2DBB23B72AB
S31508026400BB787B727B78BB72002387F86F300DE00E
S3150802641097F86F3070333B4413F8683C1846FFF719
S3150802642053FA97F86F30013387F86F3097F86F3061
S31508026430022BEDD96D4607F158040FCC0FC5236818
S315080264402B6007F148030FCBFFF746F900BF7037F9
S31508026450BD46B0BD80B582B000AF78600023002289
S3150802646000217868FFF792FF00BF0837BD4680BD56
S3150802647080B584B000AFF860B9601346FB80FB882C
S315080264803E2B06D8FB881A46B968F868FFF7BCFEA1
S3150802649005E0FB881A46B968F868FFF737FF00BFB8
S315080264A01037BD4680BD000080B588B000AF786061
S315080264B0FF23FB7600237B610023FB6100237B829B
S315080264C07B68FB60FB6893F828301B09FB76FB6840
S315080264D01B687B61FFF77CFE02467B69934202D109
S315080264E0FFF784FEF861FB7E032B00F2B38001A25C
S315080264F052F823F00565020847650208A3650208F3
S31508026500F7650208FB6893F8283003F00F039AB27E
S31508026510524B1A80514B1B881B029AB24F4B1A8058
S31508026520FB6893F829301A464C4B1B8813439AB2D8
S315080265304A4B1A80FB682A33484A1288114618467B
S3150802654000F088FE86E0FB6893F8283003F00F0314
S315080265509AB2424B1A80414B1B881B029AB23F4B96
S315080265601A80FB6893F829301A463C4B1B8813435A
S315080265709AB23A4B1A803A4B01221A70394B1B7857
S31508026580002B01D000F078FEFB682A333E2118461C
S3150802659000F060FEF869FFF75DFF324B01221A70C0
S315080265A058E0304B00221A702D4B1B781A46FB68AE
S315080265B093F8283003F00F039A4248D1FB68DB6848
S315080265C01846FEF7DBFF0346013B7B82FB6829334D
S315080265D07A8A1146184600F03DFE214B1B78013394
S315080265E0DAB21F4B1A701E4B1B780F2B2FD91C4B76
S315080265F000221A702BE01C4BD3F84432FA699A42ED
S315080266000FD1FB6893F8283003F00F03DAB2164B62
S3150802661083F86E22FB6893F82920134B83F86F22BE
S3150802662017E0114BD3F8843AFA699A4211D1FB68FA
S3150802663093F8283003F00F03DAB20B4B83F8AE2A2D
S31508026640FB6893F82920084B83F8AF2A01E000BFBC
S3150802665000E000BF00BF2037BD4680BDAAAA0020C1
S31508026660ACAA0020ADAA0020DC97002080B500AFB6
S3150802667018F018FF00BF80BD80B485B000AF7860FF
S315080266807B68FB60FB681B68B3F5806F05D1FB6806
S3150802669093F82830002B00D100BF00BF1437BD463F
S315080266A05DF8047B7047000080B500AF40220349BD
S315080266B0034814F013FB0123184680BDC0AA002024
S315080266C0B0AA002080B500AF054814F091FB034636
S315080266D0002B01D0012300E00023184680BD00BF2D
S315080266E0B0AA002080B582B000AF78600B46FB7076
S315080266F04FF47A71094813F0C9FE0346002B08D1F4
S31508026700FB781A467968064814F0FDFC034813F02C
S3150802671017FF012318460837BD4680BDC4860020E8
S31508026720B0AA002080B584B000AF78600023FB735E
S315080267304FF47A71094813F0A9FE0346002B08D1D3
S315080267407968074814F0F0FC0346FB73034813F014
S31508026750F7FEFB7B18461037BD4680BDC48600206F
S31508026760B0AA00202DE9F04796B004AF002387F8B7
S315080267704730002387F84630FFF7A4FF0346002B6D
S3150802678040F0E482C44803F04DFD3B1D402200213F
S3150802679018461AF0C3F93B1D1846FFF7C3FF03460E
S315080267A087F847303B79012B40F0D08297F847307B
S315080267B0002B00F0CB827B79202B49DC002B40F39F
S315080267C0BC82013B1F2B00F2B88201A252F823F0C9
S315080267D057680208A5680208F368020811690208E0
S315080267E02F6902084B6902089D6C0208C96A0208E9
S315080267F0B36B02083B6D0208B76C02083B6D0208D0
S315080268003B6D02083B6D02083B6D02083B6D0208B0
S315080268103B6D02083B6D02083B6D02083B6D0208A0
S315080268203B6D02083B6D02083B6D02083B6D020890
S315080268303B6D02083B6D02083B6D02083B6D020880
S315080268403B6D02083B6D02083B6D0208FD6C0208AF
S31508026850FF2B70D071E23B1D02339049184615F0A2
S31508026860C6FD8E4815F0FDF80346012B10D102F03D
S3150802687059FF0346184602F0BFFF03460021184691
S31508026880FBF736F8FAF7DAFF854803F0CBFC5DE248
S31508026890824815F0CBF803461A4601210020FDF777
S315080268A060FA53E23B1D02337E49184615F0DCFDB9
S315080268B07C4815F00CF90346012B10D102F032FF81
S315080268C00346184602F098FF034600211846FAF7CF
S315080268D0F4FFFAF7B3FF744803F0A4FC36E27148F2
S315080268E015F0DAF803461A4602210020FDF739FAAE
S315080268F02CE23B1D02336D49184615F0F2FD6B4832
S3150802690015F000F9034619460020FDF7FDF91DE2C8
S315080269103B1D02336649184615F015FE644815F004
S315080269200CF9034619460020FDF7D4F90EE2614830
S3150802693003F078FC0AE2604803F074FC02F0F2FE07
S315080269400346184602F06FFF00E23B1D02335B491D
S31508026950184615F075FE594815F016F9034603F060
S315080269607F0387F8463097F84630012B2BD100F083
S3150802697005FD0446514815F022F903461E464F48BE
S3150802698015F038F9034698464C4815F04EF9034671
S3150802699099464A4815F064F903461D46474815F0D4
S315080269A07AF903461A464FF47A7302FB03F31A4638
S315080269B000230293019200954B46424631462046F1
S315080269C001F024FAC2E197F84630022B2BD100F0E7
S315080269D0D5FC0446394815F0F2F803461E463748F0
S315080269E015F008F903469846344815F01EF9034689
S315080269F09946324815F034F903461D462F4815F0D4
S31508026A004AF903461A464FF47A7302FB03F31A4607
S31508026A1000230293019200954B4642463146204690
S31508026A2001F056FA92E197F84630032B2CD1234807
S31508026A3015F0C5F80346002B14D10020FAF7CCFD51
S31508026A401F4B00221A6000F099FC40F6B8330293F5
S31508026A50002301939923009300239922082101F028
S31508026A6037FA73E10120FAF7B7FD00F087FC40F622
S31508026A70B8330293002301939923009300239922A2
S31508026A80072101F025FA61E197F8463019460D48C3
S31508026A9003F0C8FB5AE100BFE44C040800AB00202F
S31508026AA0104D040804AB0020284D04080CAB002046
S31508026AB008AB0020404D04087C4D040810AB0020AA
S31508026AC058830020984D04083B1D0233A2491846F4
S31508026AD015F04EFFA04815F0D9FA0346002B34D11B
S31508026AE09D4815F05AFB0346002B2ED000F046FCB3
S31508026AF00446994815F0E5FA03469846964815F06D
S31508026B00FBFA03469946944815F011FB03461D46BF
S31508026B10914815F027FB03461A464FF47A7302FB8F
S31508026B2003F31E468C4815F038FB03461A464FF403
S31508026B307A7302FB03F30293019600954B4642468B
S31508026B400821204601F062F900E100F017FC04462C
S31508026B50814815F09BFA034698467F4815F0B1FA24
S31508026B60034699467C4815F0C7FA03469A467A4878
S31508026B7015F0DDFA03461D46774815F0F3FA034683
S31508026B801A464FF47A7302FB03F31E46724815F04F
S31508026B9004FB03461A464FF47A7302FB03F3029385
S31508026BA00196009553464A464146204601F02EF97B
S31508026BB0CCE03B1D02336849184615F042FF664889
S31508026BC015F064FA0346002B34D1634815F0E5FA4A
S31508026BD00346002B2ED000F0D1FB04465E4815F082
S31508026BE070FA034698465C4815F086FA03469946B3
S31508026BF0594815F09CFA03461D46574815F0B2FA4D
S31508026C0003461A464FF47A7302FB03F31E465248AA
S31508026C1015F0C3FA03461A464FF47A7302FB03F3D6
S31508026C200293019600954B4642460821204601F0FA
S31508026C304FF98BE000F0A2FB0446474815F026FA06
S31508026C4003469846444815F03CFA03469946424894
S31508026C5015F052FA03469A463F4815F068FA034673
S31508026C601D463D4815F07EFA03461A464FF47A73D6
S31508026C7002FB03F31E46384815F08FFA03461A46F6
S31508026C804FF47A7302FB03F3029301960095534677
S31508026C904A464146204601F01BF957E002F042FDFA
S31508026CA00346184602F03AFF0346002B4BD0002053
S31508026CB0FDF744F847E03B1D02332849184615F00C
S31508026CC03FFF264815F084FA03461946244803F07E
S31508026CD0A9FA224815F07CFA0346002B35D117F09B
S31508026CE0CFFA0346184617F0E1FA0346002118467A
S31508026CF014F07AFD1B4803F095FA26E03A463B1D46
S31508026D0002331146184615F04DFF3B881A46BB78E2
S31508026D101549022002F0CCFFBA78144B1B789A4226
S31508026D2004D11349022002F0C3FF0FE03B88BA7868
S31508026D3019460020FDF730F808E07B7919460D4818
S31508026D4003F070FA02E000BF00E000BF00BF483758
S31508026D50BD46BDE8F08700BF18AB002020AB002077
S31508026D60EC4D0408304E0408504E04086D07002006
S31508026D70684E0408844E040880B582B000AF786075
S31508026D807B681A687B689B881946104606F028FBBA
S31508026D900346002B01D0012300E0002318460837DA
S31508026DA0BD4680BD80B582B000AF78600B46FB70E9
S31508026DB0FB78002B08D07B6898687B689B89012240
S31508026DC0194606F025FB07E07B6898687B689B896D
S31508026DD00022194606F01CFB00BF0837BD4680BDD7
S31508026DE080B584B000AFF860B9603B601346FB809B
S31508026DF0FB68BA681A60FB68FA889A80FB683A6880
S31508026E009A60FB683A8B9A81FB68FA691A613B6A4F
S31508026E1007EE903AB8EEE77ADFED0C6AC7EE267A05
S31508026E20FB68C3ED057AFB6802221A760121F86827
S31508026E30FFF7B8FF642012F0E1FB0021F868FFF7BC
S31508026E40B1FF00BF1037BD4680BD00BF00004843F2
S31508026E5080B582B000AF7860786800F009F802461B
S31508026E607B681B69D31A18460837BD4680BD0000E1
S31508026E7080B588B000AF78600023FB610023FB76FB
S31508026E800023FB7400237B6107E0FB695A1CFA6145
S31508026E90224A934201D900233CE07868FFF76CFF47
S31508026EA00346002BF1D10120F9F72EFAF8600023E8
S31508026EB0FB761BE001217868FFF774FF7B695B00AC
S31508026EC07B6100217868FFF76DFF7868FFF754FF4A
S31508026ED00346FB74FB7C002B02D07B6901337B6182
S31508026EE097F91B30DBB20133DBB2FB7697F91B301D
S31508026EF0172BDFDD01217868FFF754FF7B6983F4DE
S31508026F0000037B6100217868FFF74CFFF868F9F700
S31508026F10FBF97B6918462037BD4680BD40420F0003
S31508026F2080B584B000AF78600B46FB700023FB6027
S31508026F300023FB720023FB7209E07868FFF798FFCB
S31508026F400246FB681344FB60FB7A0133FB72FA7A4A
S31508026F50FB789A42F1D3FB78FA6892FBF3F3184668
S31508026F601037BD4680BD80B483B000AF7860396003
S31508026F707B683A681A6100BF0C37BD465DF8047B28
S31508026F807047000080B582B000AF78600B467B8000
S31508026F900F4813F0CFFE02467B889A4211D34FF46C
S31508026FA07A710C4813F072FA0346002B0BD17B88D0
S31508026FB01A467968064814F0A6F8064813F0C0FA85
S31508026FC001E0002300E0012318460837BD4680BDCC
S31508026FD024AB00202886002080B5C4B000AF024644
S31508026FE007F58873A3F209131A70002387F80F317D
S31508026FF050E007F10C034FF480720021184619F08D
S315080270008DFD4FF47A712C4813F040FA0346002B93
S315080270100BD107F10C031946284814F0EBF803467E
S3150802702087F80F31244813F08BFA4FF47A71224805
S3150802703013F02CFA0346002B0BD107F10C03194661
S315080270401E4814F071F8034687F80F311A4813F0F0
S3150802705077FA4FF47A711A4813F018FA0346002B96
S315080270600DD1FFF7C3F897F80F319AB207F10C035F
S315080270701946FFF7FDF9124813F062FA02E01148C1
S3150802708003F0D0F807F58873A3F209131B7818469C
S3150802709003F032FA094813F0ABFE034683F0010304
S315080270A0DBB2002B03D0084B1B78002BA1D000BF04
S315080270B007F58877BD4680BD2886002024AB0020C8
S315080270C05C860020B04E040834AC002080B483B03D
S315080270D000AF78600B467B8000BF00BF0C37BD4609
S315080270E05DF8047B7047000080B582B000AF0023CC
S315080270F0FB712E4B1B78002B51D02D4B1B7801337D
S31508027100DAB22B4B1A702A4B1B78092B4AD9284B11
S3150802711000221A70254B5B78012B1FD8234B5B780C
S315080271200133DAB2214B5A704FF47A71214813F0BF
S31508027130ADF90346002B0DD1FFF758F803461B4A53
S3150802714092F883201C491846FFF792F9194813F05A
S31508027150F7F927E0194803F065F823E00023FB71E5
S3150802716002E0FB790133FB71104B93F88330FA790D
S315080271709A42F6D34FF47A71114813F087F9034607
S31508027180002B06D10C490F4813F0CEFF0C4813F01A
S31508027190D7F984220021054819F0C0FC02E0044B05
S315080271A000221A7000BF0837BD4680BD34AC0020E5
S315080271B0B8AC00205C86002037AC0020B04E04082C
S315080271C02886002024AB002080B500AF4FF48072D9
S315080271D00249034813F082FD00BF80BD34AB00208C
S315080271E024AB002080B500AFFFF7EEFF00BF80BDDD
S315080271F080B582B000AF786039603B68DBB2194669
S31508027200786800F04BF800BF0837BD4680BD80B5E8
S3150802721082B000AF786039603B689BB219467868DD
S31508027220FFF7B0FE00BF0837BD4680BD80B582B005
S3150802723000AF78603960064B1B683A6892B2796883
S31508027240184613F045FB00BF0837BD4680BD00BF90
S315080272507007002080B582B000AF78603960054BB0
S315080272601B683A687968184613F0CCFB00BF0837E2
S31508027270BD4680BD7007002080B500AF044B186874
S31508027280044B054A002113F0E8FA00BF80BD00BF8F
S31508027290700700200F720208F171020890B585B0D6
S315080272A000AF78600B46FB7002F03CFAF860FB7898
S315080272B09BB219467868FFF709FF7B681B780F2B84
S315080272C023D00F2B4BDC012B02D0052B31D046E005
S315080272D0254B9B781946254816F05DFA224BDB7832
S315080272E01946224816F073FA2149204816F0E1F9A0
S315080272F01F4816F02CFA04461D4816F034FA0346BF
S3150802730019462046FFF792FF2AE01A4B01221A7005
S315080273101749184816F0F0F9154816F018FA0446EF
S31508027320134816F020FA034619462046FFF77EFF51
S3150802733016E0114802F076FFF86802F074FA0C4873
S3150802734016F0F3F90A4816F002FA0446084816F047
S315080273500AFA034619462046FFF768FF00E000BF0F
S3150802736000BF1437BD4690BDE0BF1F08F0BD002020
S31508027370E8BC0020ECBD0020D04E040880B400AF63
S31508027380024B1846BD465DF8047B70470CBE0020CA
S3150802739080B584B000AF7860FFF7F0FFB860174B8E
S315080273A01B78002B26D1154B01221A709422002134
S315080273B0B86819F0B3FB0023FB6009E0BA68FB68FA
S315080273C004339B00134400225A60FB680133FB60B6
S315080273D0FB68042BF2DDBB687A681A6003F02EF9A3
S315080273E005220021064819F099FB0F2200210548BB
S315080273F019F094FB00BF1037BD4680BDF2BD0020D0
S31508027400F4BD0020FCBD002080B586B000AFF86050
S31508027410B9607A60FB700023FB75FA68BB680433AF
S315080274209B0013445A68FB681B6D124912010A44F1
S3150802743013441B78FB75FB7D012B09D1BB68D8B2B7
S3150802744097F8243097F82020F97803F0DDFA06E059
S31508027450BB68D8B200230022002103F0D5FAFB68E4
S315080274601B68184603F018FB002318461837BD4652
S3150802747080BD00BF9C620408B0B588B004AF7860CE
S315080274800023FB600023FB60DEE17B68FA680A32B0
S3150802749053F82230002B00F095807B68FA680A328E
S315080274A053F82230944A934200F28C80934AFB683E
S315080274B0134400221A707A68FB6814339B0013443B
S315080274C05B687C2B57D97A68FB6804339B001344A4
S315080274D05B68072B41D17B68FA681E3253F8222073
S315080274E07968FB6814339B000B445B68D21A7B6885
S315080274F0F9681E3153F821307D3B9A421BD37B68CB
S31508027500FA681E3253F822207968FB6814339B0006
S315080275100B445A607A68FB6813448C331B78002B39
S315080275200CBF01230023DBB219467A68FB681344B1
S315080275308C330A461A707A68FB6813448C331B78B4
S31508027540002B05D0FB681946786800F09BFB04E01F
S31508027550FB681946786800F09FFA7A68FB68143364
S315080275609B0013445B68A3F17D027968FB681433B8
S315080275709B000B445A607A68FB680E339B001344DF
S315080275805B687D2B0ED97A68FB680E339B00134421
S315080275905B68A3F17D027968FB680E339B000B4496
S315080275A05A60CAE0FFF7EAFEF9680023039300234C
S315080275B0029300230193002300930023002200F084
S315080275C05DF9BAE07B68FA680A3253F822304C4A07
S315080275D0934266D1494AFB68134400221A707A68B4
S315080275E0FB6814339B0013445B687C2B40F2A5802E
S315080275F07A68FB6804339B0013445B68072B41D106
S315080276007B68FA681E3253F822207968FB681433BD
S315080276109B000B445B68D21A7B68F9681E3153F8E3
S3150802762021307D3B9A421BD37B68FA681E3253F897
S3150802763022207968FB6814339B000B445A607A68E7
S31508027640FB6813448C331B78002B0CBF01230023E1
S31508027650DBB219467A68FB6813448C330A461A70F9
S315080276607A68FB6813448C331B78002B05D0FB68B9
S315080276701946786800F006FB04E0FB681946786844
S3150802768000F00AFA7A68FB6814339B0013445B68B5
S31508027690A3F17D027968FB6814339B000B445A6098
S315080276A04BE07A68FB6814339B0013445B68002B33
S315080276B043D07B68FA680A3253F82230002B3CD151
S315080276C07A68FB6804339B0013445B68082B19D15C
S315080276D0FB681946786800F0D5FA7A68FB681433AD
S315080276E09B0013445B68A3F17D027968FB68143337
S315080276F09B000B445A6020E017E40300F4BD002007
S3150802770018E403007A68FB6804339B0013445B6839
S31508027710072B12D1FB681946786800F0BDF97A681A
S31508027720FB6814339B0013445B68A3F17D027968F6
S31508027730FB6814339B000B445A607A68FB6804336F
S315080277409B0013445B68002B0DD07A68FB680433F0
S315080277509B0013445B68072B05D0464AFB68134413
S3150802776000221A7018E0FA6813465B001344424A6C
S315080277709818FA6813465B0013447A68134404336C
S315080277800322194619F0BAF90346002B04D0394ADE
S31508027790FB68134400221A70FA6813465B00134406
S315080277A0354A9818FA6813465B0013447A681344F4
S315080277B004330322194619F068FA2E4AFB68134461
S315080277C01B78002B21D17B681C6D7968FA681346F1
S315080277D05B0013440B4404331D787968FA68134630
S315080277E05B0013440B44053319787868FA68134624
S315080277F05B001344034406331B78019300912B461E
S315080278002246F9687868FFF7FFFD7B68FA680A324C
S3150802781053F82230002B14D17A68FB680E339B008A
S3150802782013445B68002B0CD17A68FB6814339B00FF
S3150802783013445B68002B04D10E4AFB6813440122E9
S315080278401A70FB680133FB60FB68042B7FF71DAED9
S315080278507B681B6D5A1C7B681A657B681B6D0F2B30
S3150802786002DD7B6800221A65002318461037BD46DA
S31508027870B0BD00BFF4BD0020FCBD002080B586B0B7
S3150802788002AFF860B96011461A460B46FB711346F9
S31508027890BB71BB68042B01D9002319E0FB791A4690
S315080278A0B968F86800F07DF8397EBA793B7F0093AB
S315080278B00B46B968F86800F02EF83A6AB968F868AB
S315080278C000F00AF87A6AB968F86800F084F803469C
S315080278D018461037BD4680BD80B485B000AFF86043
S315080278E0B9607A60BB68042B01D900230DE0FB68F6
S315080278F0BA680A32796843F82210FA68BB680E3306
S315080279009B0013447A685A60012318461437BD4609
S315080279105DF8047B704780B485B000AFF860B96043
S3150802792011461A460B46FB711346BB71BB68042BFC
S3150802793001D900232FE0F968BA6813465B0013449D
S315080279400B440433FA791A70F968BA6813465B006D
S3150802795013440B440533BA791A70F968BA681346A0
S315080279605B0013440B4406333A7E1A70F968BA6808
S3150802797013465B0013440B4403F16800F968BA68BE
S3150802798013465B0013440B440246043319889B785A
S3150802799011809370012318461437BD465DF8047B9F
S315080279A0704780B485B000AFF860B9601346FB71C2
S315080279B0BB68042B01D9002307E0FA79F968BB688A
S315080279C004339B000B445A60012318461437BD46FC
S315080279D05DF8047B704780B584B000AFF860B96083
S315080279E07A60BB68042B01D9002338E0FA68BB68C1
S315080279F014339B0013447A685A60FB68BA681E32CD
S31508027A00796843F822100022B968F86800F02BF862
S31508027A10FA68BB6804339B0013445B68072B1DD1C5
S31508027A207B68002B1AD0F968BA6813465B001344C0
S31508027A300B44043300221A70F968BA6813465B00CD
S31508027A4013440B44053300221A70F968BA681346C0
S31508027A505B0013440B44063300221A7001231846AE
S31508027A601037BD4680BD80B485B000AFF860B960F6
S31508027A701346FB71BB68042B01D9002306E0FA689A
S31508027A80BB6813448C33FA791A70012318461437E3
S31508027A90BD465DF8047B704780B489B000AFF860D4
S31508027AA0B9604FF00003FB614FF00003BB614FF072
S31508027AB000037B61BB68042B01D90023DCE0FB6869
S31508027AC0BA681E3253F82220F968BB6814339B0041
S31508027AD00B445B68D31A07EE903AF8EE677AC7ED5D
S31508027AE0077AFB69BB61FB697B61FB68BA681E3270
S31508027AF053F822307D3B07EE903AF8EE677A97ED17
S31508027B00077AB4EEE77AF1EE10FA2ADBF968BA6870
S31508027B1013465B0013440B4468331B7807EE903A0E
S31508027B20F8EE677AC7ED077AF968BA6813465B0012
S31508027B3013440B4469331B7807EE903AF8EE677ADA
S31508027B40C7ED067AF968BA6813465B0013440B4414
S31508027B506A331B7807EE903AF8EE677AC7ED057A2C
S31508027B6056E0F968BA6813465B0013440B44683357
S31508027B701B7807EE903AB8EEE77AD7ED077A67EE02
S31508027B80276AFB68BA681E3253F8223007EE903A23
S31508027B90B8EE677AC6EE877AC7ED077AF968BA68E1
S31508027BA013465B0013440B4469331B7807EE903A7D
S31508027BB0B8EEE77AD7ED067A67EE276AFB68BA68FF
S31508027BC01E3253F8223007EE903AB8EE677AC6EEBE
S31508027BD0877AC7ED067AF968BA6813465B001344D2
S31508027BE00B446A331B7807EE903AB8EEE77AD7ED7C
S31508027BF0057A67EE276AFB68BA681E3253F822309E
S31508027C0007EE903AB8EE677AC6EE877AC7ED057A36
S31508027C10D7ED077AFCEEE77AC7ED017A3B79D8B257
S31508027C20F968BA6813465B0013440B4404330246E8
S31508027C301A70D7ED067AFCEEE77AC7ED017A3B7938
S31508027C40D8B2F968BA6813465B0013440B44053385
S31508027C5002461A70D7ED057AFCEEE77AC7ED017A85
S31508027C603B79D8B2F968BA6813465B0013440B44E9
S31508027C70063302461A70012318462437BD465DF8B4
S31508027C80047B704780B489B000AFF860B9604FF0E2
S31508027C900003FB614FF00003BB614FF000037B61F9
S31508027CA0BB68042B01D90023A7E0FA68BB68143322
S31508027CB09B0013445B68544AA2FB0323DB0807EEC6
S31508027CC0903AF8EE677AC7ED077AFB69BB61FB69FA
S31508027CD07B61F968BA6813465B0013440B440433A4
S31508027CE01B7807EE903AB8EEE77AF968BA6813464F
S31508027CF05B0013440B4404331B7807EE903AB8EE44
S31508027D00E76AD7ED076AC6EE267A77EE677AC7ED8F
S31508027D10077AF968BA6813465B0013440B440533BD
S31508027D201B7807EE903AB8EEE77AF968BA6813460E
S31508027D305B0013440B4405331B7807EE903AB8EE02
S31508027D40E76AD7ED066AC6EE267A77EE677AC7ED50
S31508027D50067AF968BA6813465B0013440B4406337D
S31508027D601B7807EE903AB8EEE77AF968BA681346CE
S31508027D705B0013440B4406331B7807EE903AB8EEC1
S31508027D80E76AD7ED056AC6EE267A77EE677AC7ED11
S31508027D90057AD7ED077AFCEEE77AC7ED017A3B79E1
S31508027DA0D8B2F968BA6813465B0013440B44043325
S31508027DB002461A70D7ED067AFCEEE77AC7ED017A23
S31508027DC03B79D8B2F968BA6813465B0013440B4488
S31508027DD0053302461A70D7ED057AFCEEE77AC7ED47
S31508027DE0017A3B79D8B2F968BA6813465B0013443C
S31508027DF00B44063302461A70012318462437BD4639
S31508027E005DF8047B704700BFD34D621080B586B01B
S31508027E1004AF7860084611461A460346FB700B46BD
S31508027E20BB7013467B70FFF7A9FAB978FA78BB6973
S31508027E3003937B6902933B7C01937B7800930B4601
S31508027E400021FFF71BFDFFF799FAB978FA78BB69A3
S31508027E5003937B6902933B7C01937B7800930B46E1
S31508027E600121FFF70BFDFFF789FAB978FA78BB69A2
S31508027E7003937B6902933B7C01937B7800930B46C1
S31508027E800221FFF7FBFCFFF779FAB978FA78BB69A2
S31508027E9003937B6902933B7C01937B7800930B46A1
S31508027EA00321FFF7EBFCFFF769FAB978FA78BB69A1
S31508027EB003937B6902933B7C01937B7800930B4681
S31508027EC00421FFF7DBFC012318460837BD4680BDAF
S31508027ED080B483B000AF7860084611461A46034656
S31508027EE0FB700B46BB7013467B70012318460C3792
S31508027EF0BD465DF8047B704780B500AF03480EF0B7
S31508027F003FF902480DF0FCFF00BF80BD70C2002099
S31508027F1080B500AF00F09AFB02F074F900BF80BD8D
S31508027F2080B500AF204B214A9A6062B600BF02F0C4
S31508027F30F3FD00F041F800F0D5FB00F0F5F800F08B
S31508027F40ABF800F011F900F031F900F08DF900F004
S31508027F50E1F900F061FA00F0E1FA00F02BFB00F01B
S31508027F6075FB00F02BF901F0DDFBFDF7B1F9F9F726
S31508027F708DFAF9F743FA17F02BFAFEF795FB02F09A
S31508027F8041F90B48FEF700F800F088FDFFF774F98F
S31508027F90FFF728F90748FFF7FBF9F9F713FCFDF78E
S31508027FA091F900BFFDE700BF00ED00E000000208FE
S31508027FB0A0BE0020A8BF002080B59CB000AF07F184
S31508027FC0200350220021184618F0A8FD07F10803DD
S31508027FD000221A605A609A60DA601A615A612D4B59
S31508027FE01B692C4A43F0300313612A4B1B6903F0C1
S31508027FF030037B607B6800BF264B5B6903F008038E
S31508028000082BF9D10B233B624FF480337B620123A1
S31508028010FB6200233B6340237B634FF08063BB63B1
S315080280200223BB640323FB6403233B657D237B6531
S315080280300223BB650223FB6502233B6608237B6694
S315080280400023BB660023FB6607F12003184605F0EA
S315080280508FFA0346002B01D000F040FC1F23BB60B9
S315080280600323FB6000233B6100237B610023BB6182
S315080280700023FB6107F108030521184605F0B0FE47
S315080280800346002B01D000F029FC00BF7037BD461D
S3150802809080BD00BF0008024480B500AF204B214ACC
S315080280A01A601F4B00225A601D4B4FF440729A60A9
S315080280B01B4B0022DA601A4B00221A74184B002254
S315080280C05A74174B00229A74154B05225A61144B9F
S315080280D00A229A61124B2722DA61114B0A221A6284
S315080280E00F4B05225A620E4B02229A620C4B07224A
S315080280F0DA620B4B02221A63094B01225A63084BB6
S3150802810001229A63064B0022DA63054803F0C0FD92
S315080281100346002B01D000F0E1FB00BF80BD00BF83
S31508028120A0BE002000A4004080B582B000AF0D4B6F
S31508028130D3F888300B4A43F00103C2F88830094B5A
S31508028140D3F8883003F001037B607B6800220021A4
S315080281501B2002F003FE1B2002F01AFE00BF08379E
S31508028160BD4680BD000C024480B500AF0D4B0E4AD9
S315080281701A600C4B05225A600A4B40F2EE22DA606C
S31508028180084B40F2EE229A60064B00221A61054815
S3150802819005F056F90346002B01D000F09FFB00BFFD
S315080281A080BD00BF04BF00200030004080B400AF8D
S315080281B000BFBD465DF8047B7047000080B500AF7E
S315080281C0274B284A1A60264B4FF480025A60244BE2
S315080281D000229A60224B0722DA60214B00221A619A
S315080281E01F4B00225A611E4B4FF080629A611C4B4C
S315080281F00022DA611A4B00221A62194B00225A62CD
S31508028200174B00229A62164B0722DA62144B4FF07A
S3150802821080425A63124B00229A63114B0022DA6398
S315080282200F4B00229A640E4B0022DA640C4B002292
S315080282301A650B4B00225A65094B00229A65084BB0
S315080282400022DA65064B00221A6605480BF094F9F5
S315080282500346002B01D000F041FB00BF80BD00BFE2
S3150802826018BF00200030014080B500AF274B284ACE
S315080282701A60264B4FF480025A60244B4FF40032A0
S315080282809A60224B0722DA60204B00221A611F4BA2
S3150802829000225A611D4B4FF080629A611B4B4FF0C8
S315080282A00052DA61194B00221A62184B00225A62EE
S315080282B0164B00229A62154B0722DA62134B0022EA
S315080282C05A63124B00229A63104B0022DA630F4B51
S315080282D000229A640D4B0022DA640C4B00221A65BE
S315080282E00A4B00225A65094B00229A65074B00225F
S315080282F0DA65064B00221A6604480BF03DF9034676
S31508028300002B01D000F0EAFA00BF80BDA8BF00200A
S31508028310004C014080B58EB000AF07F12803002259
S315080283201A605A609A60DA6007F11C0300221A6022
S315080283305A609A603B4600221A605A609A60DA606E
S315080283401A615A619A61324B324A1A60304B632279
S315080283505A602F4B00229A602D4B6322DA602C4B0F
S3150802836000221A612A4B00229A6129480BF089FFDA
S315080283700346002B01D000F0B1FA4FF48053BB62DA
S3150802838007F12803194622480CF058FD0346002B2C
S3150802839001D000F0A3FA1E480CF078F80346002B29
S315080283A001D000F09BFA0023FB6100237B6207F1F0
S315080283B01C03194616480DF03DFC0346002B01D056
S315080283C000F08CFA60233B6064237B600023BB6069
S315080283D000233B613B46042219460D480CF01AFC61
S315080283E00346002B01D000F079FA3B4608221946CB
S315080283F007480CF00FFC0346002B01D000F06EFA7A
S31508028400034800F0F3FD00BF3837BD4680BD00BF04
S31508028410B0C000200004004080B58EB000AF07F15E
S31508028420280300221A605A609A60DA6007F11C0370
S3150802843000221A605A609A603B4600221A605A6005
S315080284409A60DA601A615A619A61324B324A1A6044
S31508028450304B63225A602F4B00229A602D4B6322BF
S31508028460DA602C4B00221A612A4B00229A612948AB
S315080284700BF007FF0346002B01D000F02FFA4FF44A
S315080284808053BB6207F12803194622480CF0D6FC32
S315080284900346002B01D000F021FA1E480BF0F6FF26
S315080284A00346002B01D000F019FA0023FB610023D2
S315080284B07B6207F11C03194616480DF0BBFB0346FF
S315080284C0002B01D000F00AFA60233B6064237B602C
S315080284D00023BB6000233B613B46002219460D4838
S315080284E00CF098FB0346002B01D000F0F7F93B4647
S315080284F00422194607480CF08DFB0346002B01D0CF
S3150802850000F0ECF9034800F071FD00BF3837BD46AC
S3150802851080BD00BFFCC000200008004080B500AF47
S31508028520224B234A1A60214B4FF4E1325A601F4B01
S3150802853000229A601D4B0022DA601C4B00221A6147
S315080285401A4B0C225A61194B00229A61174B0022C8
S31508028550DA61164B00221A62144B00225A62134B36
S3150802856000229A6211480DF07BFC0346002B01D0CB
S3150802857000F0B4F900210D480FF0EBFC0346002B7E
S3150802858001D000F0ABF9002108480FF020FD0346A0
S31508028590002B01D000F0A2F904480FF0A1FC034613
S315080285A0002B01D000F09AF900BF80BD48C1002017
S315080285B0004C004080B500AF224B234A1A60214B7B
S315080285C04FF4E1325A601F4B00229A601D4B00227B
S315080285D0DA601C4B00221A611A4B0C225A61194B9B
S315080285E000229A61174B0022DA61164B00221A62A0
S315080285F0144B00225A62134B00229A6211480DF05C
S315080286002FFC0346002B01D000F068F900210D4823
S315080286100FF09FFC0346002B01D000F05FF9002102
S3150802862008480FF0D4FC0346002B01D000F056F997
S3150802863004480FF055FC0346002B01D000F04EF912
S3150802864000BF80BDDCC100200050004080B500AFED
S31508028650224B234A1A60214B4FF4E1325A601F4BD0
S3150802866000229A601D4B0022DA601C4B00221A6116
S315080286701A4B0C225A61194B00229A61174B002297
S31508028680DA61164B00221A62144B00225A62134B05
S3150802869000229A6211480DF0E3FB0346002B01D033
S315080286A000F01CF900210D480FF053FC0346002B7D
S315080286B001D000F013F9002108480FF088FC0346A0
S315080286C0002B01D000F00AF904480FF009FC034612
S315080286D0002B01D000F002F900BF80BD70C2002055
S315080286E00038014080B58CB000AF07F11C030022A8
S315080286F01A605A609A60DA601A616A4BD3F88C304B
S31508028700684A43F01003C2F88C30664BD3F88C30B3
S3150802871003F01003BB61BB69624BD3F88C30614A24
S3150802872043F02003C2F88C305E4BD3F88C3003F04A
S3150802873020037B617B695B4BD3F88C30594A43F043
S315080287408003C2F88C30574BD3F88C3003F0800381
S315080287503B613B69534BD3F88C30524A43F00103D1
S31508028760C2F88C304F4BD3F88C3003F00103FB6010
S31508028770FB684C4BD3F88C304A4A43F00203C2F8E2
S315080287808C30484BD3F88C3003F00203BB60BB68CD
S31508028790444BD3F88C30434A43F00803C2F88C3072
S315080287A0404BD3F88C3003F008037B607B683D4B63
S315080287B0D3F88C303B4A43F00403C2F88C30394B69
S315080287C0D3F88C3003F004033B603B680022012196
S315080287D0354804F01DFE01220E21334804F018FE26
S315080287E001221021314804F013FE01224FF4806160
S315080287F02F4804F00DFE0123FB6101233B6200238F
S315080288007B620323BB6207F11C031946264804F060
S31508028810D9FB0E23FB6101233B6200237B62022301
S31508028820BB6207F11C0319461F4804F0CBFB102351
S31508028830FB6101233B6200237B620323BB6207F1D0
S315080288401C031946194804F0BDFB4FF48063FB610B
S3150802885001233B6200237B620323BB6207F11C03ED
S315080288601946134804F0AEFB44F60F03FB610023D6
S315080288703B6200237B6207F11C0319460C4804F08D
S31508028880A1FB4FF40073FB6100233B6200237B626A
S3150802889007F11C031946074804F094FB00BF30375A
S315080288A0BD4680BD000C024400140242000002428A
S315080288B0000C02420008024280B582B000AF78601E
S315080288C07B681B68044A934201D102F04BF900BF48
S315080288D00837BD4680BD00BF0010004080B400AF17
S315080288E072B600BF00BFFDE7B0B596B000AF7860BC
S315080288F0396000237B653EE05B4B5C4A4021786821
S3150802890003F024FC0346002B03D0594801F08AFCE5
S3150802891031E0564B1B687B65FDF75AFC02467B6DB8
S31508028920934204D168215148FDF7F4FA23E012F084
S3150802893003FE02467B6D934211D012F00BFE0246ED
S315080289407B6D93420BD012F00EFE02467B6D93426C
S3150802895005D012F037FE02467B6D93420BD1434B8C
S31508028960DB681846FCF70AFE0346DBB21A463E499E
S31508028970786D16F083FD4021786803F005FD0346FD
S31508028980002BB9D17868FDF7AFFB03461A46394B77
S315080289909A607868FDF772FB0346364A1360786870
S315080289A0FDF784FB0346334A5360324B9B68002B20
S315080289B011D000F0B7FE0346184601F0A2F80346A6
S315080289C0002B08D02B4B1A682A4B5B6807F10C0060
S315080289D0294918F00FF80C222649284818F08EF86B
S315080289E00346002B36D0234B1B68DAB207F1500335
S315080289F01146184613F018FA1E4B5B68DAB207F1ED
S31508028A0050031146184613F02AFA1A4B9B68DAB233
S31508028A1007F150031146184613F03CFA07F10C0207
S31508028A2007F150031146184613F0D1FE12F0AEFDB7
S31508028A30044607F10C03184613F027FC054607F10E
S31508028A400C03184613F02DFC03461A4629462046FF
S31508028A5016F098FD094B074A07CA83E8070000BFC4
S31508028A605837BD46B0BD00BF2CC3002004C3002042
S31508028A70EC4E040890AA00200C4F04089CAA002079
S31508028A8080B500AF044803F0E8FA00220121024843
S31508028A9003F098FC00BF80BDA0BE002080B500AFE1
S31508028AA0FDF77CFB0346002B09D0FDF791FB034635
S31508028AB01A466FF060410220FDF7B6FA09E0FDF7A3
S31508028AC087FB03469BB21A464FF6FF710220FDF753
S31508028AD07FFAFFF7D5FF00BF80BD000080B58EB0D4
S31508028AE000AFF860B9601346FB71FB79002B02D020
S31508028AF0FB79402B01D900233FE007F11403242216
S31508028B000021184618F00AF8FB687B61FDF746FB58
S31508028B100346002B03D04FF08043BB6101E00023DC
S31508028B20BB610023FB61FB799BB21846FCF77CFD0F
S31508028B3003463B6200237B624FF48013BB624FF409
S31508028B400013FB6200233B6300237B634FF47A71B5
S31508028B500C4811F09BFC0346002B0AD107F11403BB
S31508028B60BA6819460848FCF7C1FE064811F0E8FC3F
S31508028B7002E0064801F056FB012318463837BD467F
S31508028B8080BD00BFF8860020A0BE00202C4F040836
S31508028B9080B400AF00BFBD465DF8047B7047000095
S31508028BA080B5CCB000AF07F59873A3F59673186035
S31508028BB007F58E7300221A605A609A60DA601A61A3
S31508028BC007F59873A3F5907318464FF484731A46FB
S31508028BD0002117F0A3FF07F59873A3F596731B6890
S31508028BE01B68384A934267D107F59873A3F59071C3
S31508028BF04FF000024FF00403C1E9002307F598730A
S31508028C00A3F590734FF48072C3F8BC2007F11003E2
S31508028C10184605F05FFC0346002B01D0FFF75EFEFF
S31508028C20294BD3F8A030284A43F40073C2F8A0307F
S31508028C30254BD3F8A03003F4007207F59873A3F511
S31508028C4092731A6007F59873A3F592731B681E4B05
S31508028C50D3F88C301C4A43F00103C2F88C301A4B05
S31508028C60D3F88C3003F0010207F59873A3F59473D1
S31508028C701A6007F59873A3F594731B684FF4C053EB
S31508028C80C7F81C310223C7F820310023C7F824315C
S31508028C900023C7F828310923C7F82C3107F58E7344
S31508028CA019460A4804F08EF900220021272002F00C
S31508028CB055F8272002F06CF800BF07F59877BD46ED
S31508028CC080BD00BF00A40040000C0244000002421E
S31508028CD080B5CEB000AF07F59C73A3F59A731860FA
S31508028CE007F5927300221A605A609A60DA601A616E
S31508028CF007F59C73A3F5907318464FF484731A46C6
S31508028D00002117F00BFF07F59C73A3F59A731B68EE
S31508028D101B68924A93425ED107F59C73A3F590713C
S31508028D204FF000624FF00003C1E9002307F59C7378
S31508028D30A3F590730022C3F8E02007F1180318463A
S31508028D4005F0C8FB0346002B01D0FFF7C7FD844B8D
S31508028D50D3F8A430824A43F48053C2F8A430804B35
S31508028D60D3F8A43003F4805207F59C73A3F59273E3
S31508028D701A6007F59C73A3F592731B68784BD3F8B0
S31508028D808C30774A43F00103C2F88C30744BD3F81F
S31508028D908C3003F0010207F59C73A3F594731A60ED
S31508028DA007F59C73A3F594731B68E023C7F824316F
S31508028DB00223C7F828310023C7F82C310023C7F845
S31508028DC030310523C7F8343107F5927319466548D9
S31508028DD004F0F8F8BCE007F59C73A3F59A731B68D0
S31508028DE01B68614A934240F0B38007F59C73A3F56A
S31508028DF090714FF080424FF00003C1E9002307F556
S31508028E009C73A3F590734FF4C062C3F8EC2007F184
S31508028E101803184605F05EFB0346002B01D0FFF740
S31508028E205DFD4F4BD3F8A4304D4A43F40023C2F8F4
S31508028E30A4304B4BD3F8A43003F4002207F59C73F5
S31508028E40A3F596731A6007F59C73A3F596731B68C8
S31508028E50434BD3F88C30424A43F01003C2F88C30A5
S31508028E603F4BD3F88C3003F0100207F59C73A3F539
S31508028E7098731A6007F59C73A3F598731B6844F2F6
S31508028E800403C7F824310223C7F828310023C7F898
S31508028E902C310323C7F830310523C7F8343107F5D7
S31508028EA092731946314804F08DF8314B314A1A60EB
S31508028EB02F4B30225A602E4B00229A602C4B4FF4CD
S31508028EC08062DA602A4B08221A61294B00225A610B
S31508028ED0274B00229A61264B0022DA61244B002294
S31508028EE01A62234B01225A62214B01229A62204BB3
S31508028EF00022DA621E4B00221A631D4B00225A63B5
S31508028F001B4801F061FF0346002B01D0FFF7E6FC80
S31508028F1007F59C73A3F59A731B68154AC3F8802054
S31508028F20134A07F59C73A3F59A731B68D365102138
S31508028F300F4802F004FB0346002B01D0FFF7CEFCD4
S31508028F4000220021522001F009FF522001F020FFE1
S31508028F5000BF07F59C77BD4680BD00BF00300140C3
S31508028F60000C024400000242004C0140001002427A
S31508028F7038C000205000024080B485B000AF786047
S31508028F807B681B68164A93420FD1164BD3F89C305E
S31508028F90144A43F00203C2F89C30124BD3F89C30B1
S31508028FA003F00203FB60FB6813E07B681B680E4A4A
S31508028FB093420ED10B4BD3F89C300A4A43F0040372
S31508028FC0C2F89C30074BD3F89C3003F00403BB600D
S31508028FD0BB6800BF1437BD465DF8047B704700BF07
S31508028FE000040040000C02440008004080B58AB024
S31508028FF000AF786007F1140300221A605A609A607B
S31508029000DA601A617B681B68264A934220D1264B8E
S31508029010D3F88C30244A43F00403C2F88C30224B2E
S31508029020D3F88C3003F004033B613B694FF4C073F9
S315080290307B610223BB610023FB6103233B6202239C
S315080290407B6207F114031946184803F0BBFF24E0B4
S315080290507B681B68164A93421FD1134BD3F88C3090
S31508029060114A43F00803C2F88C300F4BD3F88C3000
S3150802907003F00803FB60FB684FF440537B6102234D
S31508029080BB610023FB6103233B6202237B6207F178
S3150802909014031946074803F095FF00BF2837BD4653
S315080290A080BD00BF00040040000C024400080242D2
S315080290B000080040000C024280B5D0B000AF07F5A8
S315080290C0A073A3F59E73186007F5967300221A60BB
S315080290D05A609A60DA601A6107F5A073A3F590736D
S315080290E018464FF484731A46002117F017FD07F540
S315080290F0A073A3F59E731B681B68A64A934265D1A3
S3150802910007F5A073A3F590714FF008024FF000031C
S31508029110C1E9002307F5A073A3F5907300229A66A6
S3150802912007F12003184605F0D5F90346002B01D0AE
S31508029130FFF7D4FB984BD3F89C30974A43F40023A5
S31508029140C2F89C30944BD3F89C3003F4002207F5FE
S31508029150A073A3F592731A6007F5A073A3F5927329
S315080291601B688D4BD3F88C308B4A43F00103C2F847
S315080291708C30894BD3F88C3003F0010207F5A073C3
S31508029180A3F594731A6007F5A073A3F594731B6885
S315080291900323C7F82C310223C7F830310023C7F856
S315080291A034310023C7F838310823C7F83C3107F5AC
S315080291B096731946794803F005FF002200213D20DF
S315080291C001F0CCFD3D2001F0E3FDDEE007F5A073DA
S315080291D0A3F59E731B681B68714A934266D107F50D
S315080291E0A073A3F590714FF010024FF00003C1E986
S315080291F0002307F5A073A3F590730022DA6607F138
S315080292002003184605F066F90346002B01D0FFF73E
S3150802921065FB614BD3F89C305F4A43F48013C2F86E
S315080292209C305D4BD3F89C3003F4801207F5A0738B
S31508029230A3F596731A6007F5A073A3F596731B68D0
S31508029240554BD3F88C30544A43F00203C2F88C309B
S31508029250514BD3F88C3003F0020207F5A073A3F53D
S3150802926098731A6007F5A073A3F598731B684FF4F1
S315080292704053C7F82C310223C7F830310023C7F808
S3150802928034310023C7F838310E23C7F83C3107F5C5
S3150802929096731946434803F095FE002200213E20A4
S315080292A001F05CFD3E2001F073FD6EE007F5A07348
S315080292B0A3F59E731B681B683B4A934265D107F563
S315080292C0A073A3F590714FF001024FF00003C1E9B4
S315080292D0002307F5A073A3F590730022DA6507F158
S315080292E02003184605F0F6F80346002B01D0FFF7CF
S315080292F0F5FA294BD3F8A430274A43F48043C2F837
S31508029300A430254BD3F8A43003F4804207F5A073A2
S31508029310A3F59A731A6007F5A073A3F59A731B68E7
S315080293201D4BD3F88C301C4A43F00103C2F88C302B
S31508029330194BD3F88C3003F0010207F5A073A3F595
S315080293409C731A6007F5A073A3F59C731B684FF408
S31508029350C063C7F82C310223C7F830310023C7F897
S3150802936034310323C7F838310723C7F83C3107F5E8
S3150802937096731946094803F025FE002200213A2071
S3150802938001F0ECFC3A2001F003FD00BF07F5A077D7
S31508029390BD4680BD004C0040000C0244000002425B
S315080293A000500040000402420038014080B582B0F5
S315080293B000AF78607B681B68204A93420FD1204B26
S315080293C0D3F89C301E4A23F40023C2F89C300321AA
S315080293D01C4803F049FF3D2001F0E8FC2AE07B68BF
S315080293E01B68194A934210D1154BD3F89C30144A7C
S315080293F023F48013C2F89C304FF44051134803F00B
S3150802940033FF3E2001F0D2FC14E07B681B68104A49
S3150802941093420FD10A4BD3F8A430094A23F4804366
S31508029420C2F8A4304FF4C061064803F01DFF3A2083
S3150802943001F0BCFC00BF0837BD4680BD004C0040A9
S31508029440000C02440000024200500040000402429E
S315080294500038014080B58EB000AF7860334BD3F840
S315080294609C30324A43F01003C2F89C302F4BD3F893
S315080294709C3003F01003BB60BB6807F10C0207F1CE
S3150802948010031146184604F0EDFFFB69FB62FB6AFE
S31508029490002B03D104F0A4FF786304E004F0A0FFD4
S315080294A003465B007B637B6B5B09214AA2FB0323B2
S315080294B0DB09013BBB621F4B1F4A1A601D4B632225
S315080294C0DA601C4ABB6A53601A4B00221A61194BAE
S315080294D000229A6017480AF0D4FE034687F833300A
S315080294E097F83330002B18D112480AF021FF0346A9
S315080294F087F8333097F83330002B0ED17B680F2B61
S3150802950008D800227968312001F028FC0B4A7B68CA
S31508029510136002E0012387F83330312001F038FC6A
S3150802952097F8333018463837BD4680BD000C0244DA
S31508029530C55A7C0A6CC30020001000407807002038
S3150802954080B400AF00BFFDE780B400AF00BFFDE7FF
S3150802955080B400AF00BFFDE780B400AF00BFFDE7EF
S3150802956080B400AF00BFFDE780B400AF00BFBD46C0
S315080295705DF8047B7047000080B500AF024801F031
S3150802958058FE00BF80BD00BF38C0002080B500AFBE
S31508029590024802F0FDFF00BF80BD00BFA0BE00204A
S315080295A080B500AF02480BF0EBF900BF80BD00BFE3
S315080295B06CC3002080B500AF02480CF095FE00BFD0
S315080295C080BD00BF70C2002080B500AF02480CF013
S315080295D08BFE00BF80BD00BF48C1002080B500AF2A
S315080295E002480CF081FE00BF80BD00BFDCC100202E
S315080295F080B500AF02480AF00BFB00BF80BD00BF72
S31508029600A8BF002080B400AF01231846BD465DF806
S31508029610047B704780B582B000AF7860396017F076
S31508029620F1FA034616221A604FF0FF331846083736
S31508029630BD4680BD80B582B000AF78604FF0FF317D
S315080296407868FFF7E7FF00BFFDE780B586B000AF91
S31508029650F860B9607A6000237B610AE0AFF30080A4
S315080296600146BB685A1CBA60CAB21A707B690133D2
S315080296707B617A697B689A42F0DB7B681846183701
S31508029680BD4680BD80B586B000AFF860B9607A6025
S3150802969000237B6109E0BB685A1CBA601B7818462E
S315080296A0AFF300807B6901337B617A697B689A42F2
S315080296B0F1DB7B6818461837BD4680BD80B483B097
S315080296C000AF78604FF0FF3318460C37BD465DF899
S315080296D0047B704780B483B000AF786039603B681A
S315080296E04FF400525A60002318460C37BD465DF8FF
S315080296F0047B704780B483B000AF786001231846B4
S315080297000C37BD465DF8047B704780B485B000AF60
S31508029710F860B9607A60002318461437BD465DF8CA
S31508029720047B704780B582B000AF0023FB712F4BD4
S315080297301B78DBB2002B53D12C4B01221A70302234
S3150802974000212B4817F0EAF9294800F095F8034654
S315080297500521184612F0C4F8254800F08DF803468C
S315080297600921184612F0D7F80121214800F0B8F964
S315080297701F4800F081F803461021184612F06BF8CC
S315080297801B4800F079F803464021184612F063F8A0
S31508029790174800F071F803460121184612F0F2F84C
S315080297A0134800F069F803460021184612F02FF90B
S315080297B016F02EF902460F4B83FB02131344D911F6
S315080297C0D317C91A0B461B025B1AD11ACBB201333D
S315080297D0FB71074AFB7982F82E300120FCF7CCFC94
S315080297E0034B18460837BD4680BD00BFE8C30020B4
S315080297F0B8C300208180808080B483B000AF7860CF
S315080298007B6818460C37BD465DF8047B704780B402
S3150802981083B000AF78607B681B7C18460C37BD4660
S315080298205DF8047B704780B483B000AF78607B68CC
S3150802983001221A74012318460C37BD465DF8047BCB
S31508029840704780B483B000AF78607B685B7C18464B
S315080298500C37BD465DF8047B704780B483B000AF11
S3150802986078600B46FB707B68FA785A7400BF0C372F
S31508029870BD465DF8047B704780B483B000AF78605C
S315080298807B68123318460C37BD465DF8047B704771
S3150802989080B483B000AF78607B681A3318460C37F9
S315080298A0BD465DF8047B704780B584B000AF78602A
S315080298B00B46FB707B689B7CFB737868FFF7DCFFC3
S315080298C00246FB781946104611F073FFFA7BFB78BD
S315080298D09A4203D001217868FFF7BFFFFB78012B74
S315080298E00CD9FB78052B09D87868FFF7C5FF02461D
S315080298F0FB781946104611F0F3FF0EE0FB78052BAC
S315080299000BD9FB78092B08D87868FFF7B5FF02460A
S31508029910FB781946104611F0FEFF00BF1037BD4608
S3150802992080BD80B584B000AF78600B46FB707B685B
S31508029930DB7CFB737868FFF79FFF0246FB781946C4
S31508029940104611F051FFFA7BFB789A4203D00121A7
S315080299507868FFF782FF00BF1037BD4680BD80B525
S3150802996082B000AF78600B46FB707868FFF784FF19
S315080299700246FB781946104611F051FF034618466F
S315080299800837BD4680BD80B584B000AF78600B4607
S31508029990FB700023FB737B681B7DBB737868FFF73C
S315080299A06BFF0246FB781946104611F054FF034630
S315080299B0FB737B681B7DBA7B9A4203D001217868C8
S315080299C0FFF74BFFFB7B18461037BD4680BD0000EC
S315080299D080B584B000AF78600B46FB700023FB733A
S315080299E07B681B7DBB737868FFF746FF0246FB78E8
S315080299F01946104611F049FF0346FB737B681B7D27
S31508029A00BA7B9A4209D0FB78802B02D1054800F02E
S31508029A1009FC01217868FFF720FFFB7B18461037FF
S31508029A20BD4680BD4C4F040880B582B000AF786051
S31508029A300B46FB707868FFF71FFF0246FB7819464C
S31508029A40104611F083FF034618460837BD4680BD07
S31508029A5080B584B000AF78600B46FB700023FB73B9
S31508029A607B68DB7DBB737868FFF706FF0246FB78E7
S31508029A701946104611F086FF0346FB737B68DB7DA9
S31508029A80BA7B9A4203D001217868FFF7E6FEFB7B90
S31508029A9018461037BD4680BD80B584B000AF7860E1
S31508029AA00B46FB700023FB737B68DB7DBB73786810
S31508029AB0FFF7E2FE0246FB781946104611F07CFFD4
S31508029AC00346FB737B68DB7DBA7B9A4203D001218E
S31508029AD07868FFF7C2FEFB7B18461037BD4680BD85
S31508029AE080B483B000AF78600B46FB707B68FA7867
S31508029AF083F82A20012318460C37BD465DF8047BF5
S31508029B00704780B483B000AF78607B6893F82A30D8
S31508029B1018460C37BD465DF8047B704780B483B09F
S31508029B2000AF78607B6893F82D3018460C37BD462F
S31508029B305DF8047B704780B483B000AF78600B464B
S31508029B40FB707B68FA7883F82B20012318460C37BA
S31508029B50BD465DF8047B704780B483B000AF786079
S31508029B607B6893F82B3018460C37BD465DF8047BA4
S31508029B70704780B483B000AF78600B46FB707B6891
S31508029B80FA7883F82C20012318460C37BD465DF86F
S31508029B90047B704780B483B000AF78607B6893F823
S31508029BA02C3018460C37BD465DF8047B7047B0B5B5
S31508029BB096B000AF7860084611461A460346FB700F
S31508029BC00B46BB7013467B7007F150030622002131
S31508029BD0184616F0A3FFFA7807F1500311461846FD
S31508029BE012F073F9BA7807F150031146184612F0C3
S31508029BF07BF97A7807F150031146184612F083F971
S31508029C0097F8682007F150031146184612F08AF9A8
S31508029C1097F86C2007F150031146184612F091F98D
S31508029C2097F8702007F150031146184612F098F972
S31508029C3007F10C0207F150031146184612F0F6FD19
S31508029C4011F0A4FC044607F10C03184612F01DFB9A
S31508029C50054607F10C03184612F023FB03461A467B
S31508029C602946204615F08EFC00BF5837BD46B0BDC2
S31508029C7080B483B000AF78607B6893F82E30772B78
S31508029C8004D87B6893F82E306E2B03D87B686F2234
S31508029C9083F82E207B6893F82E305A1CD1B27A6844
S31508029CA082F82E1018460C37BD465DF8047B7047BD
S31508029CB00EB490B5ADF5047D00AF024607F5047300
S31508029CC0A3F209231A704FF480720021324816F063
S31508029CD025FF07F5087207F50473A3F502731A60E0
S31508029CE007F50473A3F502731A68D7F81C122A48F3
S31508029CF016F0FAFE284A2949294816F07BFE07F586
S31508029D000473A3F209231B78022B1AD107F10C0359
S31508029D101946234810F073FD07F10C03184610F094
S31508029D203BFD044607F10C03184610F041FD0346B5
S31508029D3019462046FDF77AFA19491A4800F072FAC6
S31508029D4021E007F50473A3F209231B78012B16D128
S31508029D5007F10C031946124810F051FD07F10C03DE
S31508029D60184610F019FD044607F10C03184610F0C0
S31508029D701FFD034619462046FDF758FA03E008492F
S31508029D80084800F04FFA0123184607F50477BD463E
S31508029D90BDE8904003B07047ECC30020644F040846
S31508029DA0ECC400206C4F040880B586B000AF78601A
S31508029DB0144A154BD31A7B617B693B61134B1B68AB
S31508029DC0002B02D1114B124A1A60104B1A687B6893
S31508029DD013443A699A4207D216F014FF03460C2234
S31508029DE01A604FF0FF3309E0084B1B68FB60074B0C
S31508029DF01A687B681344054A1360FB6818461837C5
S31508029E00BD4680BD00000A2000040000FCC50020F3
S31508029E1070E4002080B483B000AF354BD3F88830A5
S31508029E20334A43F47003C2F88830324B01221A606F
S31508029E30304B0022DA612F4B00221A622D4B1A6828
S31508029E402C492D4B13400B602A4B00229A62294B50
S31508029E500022DA62274B00221A63264B274A5A63E4
S31508029E60244B00229A63234B244ADA63214B0022AD
S31508029E701A64204B214A5A641E4B00229A641D4BCF
S31508029E801B681C4A23F4802313601A4B00221A65A6
S31508029E90174B4FF000629A60194B9B6903F06043B7
S31508029EA07B607B68B3F1604F03D07B68B3F1404FA8
S31508029EB017D1134BDB6903F00103002B05D0104BB6
S31508029EC0104ADA600E4B104ADA600D4BDB690C4A0F
S31508029ED043F00203D3610A4BDB69094A43F00103E3
S31508029EE0D36100BF0C37BD465DF8047B704700BFDF
S31508029EF000ED00E0000C0244E3EAE2EA8002010116
S31508029F00002002403B2A19087F6E5D4C80B58EB050
S31508029F1008AF78607B687B6100233B610A220721D0
S31508029F20184800F03FFA03463B6107F10C0100238B
S31508029F304FF48052786910F0F7F80346002B01D0E7
S31508029F4002231AE0FB68B022069201220592002239
S31508029F5004920A2203920A2202924FF48052019232
S31508029F6000933B69084A0749084810F023FB034651
S31508029F70002B01D00E2300E0002318461837BD46F1
S31508029F8080BD00BF704F0408919F020800C60020DA
S31508029F9080B588B004AF78607B68FB60FDF7EEF9A0
S31508029FA00023029300230193FF230093FF23FF223A
S31508029FB00121FDF72BFFFDF7E1F903461846FDF7E8
S31508029FC05BFAFB68DBB2184600F096FA7D200FF0C2
S31508029FD015FB00BFEFE7000080B582B000AF03466D
S31508029FE0FB71FB1D01221946034810F01DFF00BF35
S31508029FF00837BD4680BD00BFB0C6002080B584B014
S3150802A00000AF0346FB710023FB730023BB7326488C
S3150802A01010F0EEFE034683F00103DBB2002B1CD0E0
S3150802A02010E0BB7B1846F7F7C7FF0023BB73FB7B21
S3150802A0300133FB7397F90F30002B30DBFB79184697
S3150802A04000F05AFA07F10E0301221946164810F0D3
S3150802A05026FF0346002BE4D122E014480CF038FC14
S3150802A0600346202B0DD1114B0122A3F85C200F4B7E
S3150802A0700122A3F85E2001220D490C480CF01EF8B5
S3150802A0800EE00A4BB3F85C20084BB3F85E309BB27D
S3150802A0909A4205D0FDF730FFFDF73AFF00E000BF10
S3150802A0A000BF1037BD4680BDB0C6002070C2002072
S3150802A0B050C9002080B582B000AF78600B467B801D
S3150802A0C00F4810F037FE02467B889A4211D34FF4A6
S3150802A0D07A710C4810F0DAF90346002B0BD17B880B
S3150802A0E01A467968064810F09FFE064810F028FAC4
S3150802A0F001E0002300E0012318460837BD4680BD6B
S3150802A100C0C60020F485002080B5ADF5047D00AFF9
S3150802A110024607F50473A3F209231A700023A7F867
S3150802A1200E322EE007F10C034FF400720021184696
S3150802A13016F0F4FC4FF47A71194810F0A7F90346A1
S3150802A140002B0DD107F10C034FF40072194615487E
S3150802A15010F0A5FE0346A7F80E32114810F0F0F9E2
S3150802A160B7F80E2207F10C014FF47A730E480BF07A
S3150802A17006FF07F50473A3F209231B78184600F0B5
S3150802A180BBF9084810F034FE034683F00103DBB23C
S3150802A190002BC7D100BF00BF07F50477BD4680BDB7
S3150802A1A0F4850020C0C6002070C2002080B582B0A7
S3150802A1B000AF78600B467B807A884FF47A737968A9
S3150802A1C003480BF0DCFE012318460837BD4680BD5E
S3150802A1D070C2002080B500AF80220649064810F0FA
S3150802A1E07DFD4FF400720549054810F077FD00BF62
S3150802A1F080BD00BFD0C60020B0C6002050C70020D0
S3150802A200C0C6002080B500AFFFF7E4FF012203496C
S3150802A21003480BF053FF00BF80BD00BF50C90020A2
S3150802A22070C200200FB480B582B000AF4FF48072BE
S3150802A2300021124816F072FC07F114033B603A68D3
S3150802A24039690E4816F050FC78600C4A0C490D48DC
S3150802A25016F0D0FB0B48F6F73FF903469BB21946B0
S3150802A2600848FFF727FF03467B607B6818460837CE
S3150802A270BD46BDE8804004B0704700BF58C90020FB
S3150802A280784F040858CA002080B582B000AF7860BB
S3150802A2907B681B680E4A93420DD10E4B1B781846F3
S3150802A2A0FFF79AFE0B4B00221A70012209490A4847
S3150802A2B00BF004FF07E07B681B68084A934202D149
S3150802A2C0074B00221A7000BF0837BD4680BD00BF83
S3150802A2D00038014050C9002070C2002000480040E2
S3150802A2E051C9002080B582B000AF786078680CF05A
S3150802A2F004FB0346074A13607B681B68064A9342B7
S3150802A30003D1FDF7F9FDFDF703FE00BF0837BD4689
S3150802A31080BD00BF54C900200038014080B58CB00A
S3150802A32008AF78601A4B00221A7088220021194851
S3150802A33016F0F4FB7B68FB6007F1080100234FF473
S3150802A3408062F8680FF0F0FE0346002B01D0022364
S3150802A3501AE0BB68B02206920122059200220492F4
S3150802A3600A2203920A2202924FF480620192009311
S3150802A3700023094A09490A4810F01CF90346002B2A
S3150802A38001D00E2300E0002318461037BD4680BDD3
S3150802A390F0CB002068CB002025A602087C4F0408D3
S3150802A3A0F4CB002080B584B000AF78600B46FB7012
S3150802A3B01346BB70FF23FB73484B1B78032B77D8D6
S3150802A3C0FB78202B0ED8454B1B781A4613461B01E1
S3150802A3D013445B00424A1344FA787968184616F021
S3150802A3E054FC0DE03D4B1B781A4613461B011344D9
S3150802A3F05B003B4A134420227968184616F045FC4E
S3150802A400364B1B781946364A0B461B010B445B0032
S3150802A41013442033BA781A70304B1B7818462F4BE0
S3150802A4201B7819462E4A03461B0103445B00134454
S3150802A430203318782A4A0B461B010B445B00134447
S3150802A440213302461A70254B1B785A1CD1B2234A6D
S3150802A4501170FB731D212348FFF7A8FE07F10C03B1
S3150802A46003220021184616F059FBFA7B07F10C0362
S3150802A4701D49184616F0BEFA07F10C031846F6F7F8
S3150802A4802BF803469AB207F10C0311461846FFF752
S3150802A4908DFE02211548FFF789FEFB789BB2194605
S3150802A4A07868FFF783FE02211148FFF77FFE0FE067
S3150802A4B0FF23FB7334210F48FFF778FEFB789BB224
S3150802A4C019467868FFF772FE02210948FFF76EFE01
S3150802A4D0FB7B18461037BD4680BD00BFF0CB002077
S3150802A4E068CB0020884F0408A84F0408AC4F04081C
S3150802A4F0B04F0408B44F040880B582B000AF0346D3
S3150802A500FB71114B1B78FA799A4213D2F979FA79C7
S3150802A5100E480B461B010B445B0003442033187894
S3150802A5200A4913461B0113445B000B4421330246B6
S3150802A5301A7004E0FB7919460548FFF773FE00BF57
S3150802A5400837BD4680BD00BFF0CB002068CB00208F
S3150802A550EC4F040880B582B000AF0023FB710023DC
S3150802A560BB712A4B1B78002B4BD10023FB7136E0BB
S3150802A570FA79274913461B0113445B000B4421331E
S3150802A5801B78002B17D0FA79214913461B0113446D
S3150802A5905B000B4421331B78BB71BB79013BBB7152
S3150802A5A0FA791B4913461B0113445B000B442133FA
S3150802A5B0BA791A7010E0FA7913461B0113445B0044
S3150802A5C0134A134419461348FFF72CFE1248FFF79D
S3150802A5D029FE0E4B01221A70FB790133FB710F4BD0
S3150802A5E01B78FA799A42C3D3FFF79CF803461846B2
S3150802A5F0FFF70DF90346002B04D1094802F0A8FF1C
S3150802A60000E000BF0837BD4680BD00BFA4CC0020CD
S3150802A61068CB00202450040850500408F0CB0020D0
S3150802A62004BF002080B582B000AF7860FFF792FFC2
S3150802A6304FF47A700EF0E2FF00BFF7E780B500AF7D
S3150802A6400F2200210A4816F069FAD2220021094887
S3150802A65016F064FA23220021074816F05FFA4FF42F
S3150802A6608C720021054816F059FA00BF80BD00BF5A
S3150802A670B8CE0020A8CC00207CCD0020A0CD00209A
S3150802A68080B485B000AF78600B46FB700023FB737D
S3150802A690FB78012202FA03F3DAB27B68DBB21340D3
S3150802A6A0FB73FB7B002B14BF01230023DBB2184686
S3150802A6B01437BD465DF8047B7047000080B485B048
S3150802A6C000AF03463960FB710023FB730023BB739B
S3150802A6D03B68002B02D1774B00221A60FB79012BCB
S3150802A6E056D10023FB7325E0734B1B78072B10D931
S3150802A6F0704B1B68714A1178714AD1546D4B1B68AD
S3150802A70001336C4A13606C4B00221A706B4B0022A1
S3150802A7101A706A4B1B785B00DBB20133DAB2674BFD
S3150802A7201A70654B1B780133DAB2634B1A70FB7BDE
S3150802A7300133FB73FB7B052BD6D90623BB7323E0B8
S3150802A7405D4B1B78072B10D95A4B1B685B4A11784D
S3150802A7505B4AD154574B1B680133564A1360564B12
S3150802A76000221A70554B00221A70544B1B785B0054
S3150802A770DAB2524B1A70504B1B780133DAB24E4B8F
S3150802A7801A70BB7B0133BB73BB7B0D2BD8D955E043
S3150802A7900023FB7325E0484B1B78072B10D9454B42
S3150802A7A01B68464A1178464AD154424B1B68013304
S3150802A7B0404A1360404B00221A70404B00221A701E
S3150802A7C03E4B1B785B00DBB20133DAB23B4B1A70A5
S3150802A7D0394B1B780133DAB2374B1A70FB7B0133DC
S3150802A7E0FB73FB7B022BD6D90323BB7323E0324BC5
S3150802A7F01B78072B10D92F4B1B68304A1178304A21
S3150802A800D1542C4B1B6801332A4A13602A4B002267
S3150802A8101A702A4B00221A70284B1B785B00DAB290
S3150802A820264B1A70244B1B780133DAB2224B1A7064
S3150802A830BB7B0133BB73BB7B0D2BD8D93B68762B0D
S3150802A84032D91D4B1B78072B1DD81C4B1B781A4671
S3150802A850194B1B78C3F1080302FA03F3DAB2174B52
S3150802A8601A70144B1B68154A1178154AD154114BA4
S3150802A8701B6801330F4A13600F4B00221A700F4BE5
S3150802A88000221A7010E00B4B1B680C4A11780C4A0E
S3150802A890D154084B1B680133064A1360064B002243
S3150802A8A01A70064B00221A7000BF1437BD465DF8AF
S3150802A8B0047B7047C8CE0020CCCE0020CDCE002027
S3150802A8C0A8CC002080B584B000AF0023FB73D22247
S3150802A8D000213D4816F022F900237B6000233B60E5
S3150802A8E00023BB6068E0BB68384A82FB03129210F9
S3150802A8F0DB17D31A7B60BA68344B83FB02139910B1
S3150802A900D317C91A0B465B000B44DB00D31A3B600C
S3150802A9102F4B1B78002B03D12D4B07221A7005E00B
S3150802A9202B4B1B78013BDAB2294B1A703B68072B73
S3150802A93011DC28497A6813465B0013440B44013339
S3150802A9401B781A46224B1B7819461046FFF798FEC3
S3150802A9500346FB7327E03B680F2B10DC1D497A6818
S3150802A96013465B0013440B441B781A46184B1B7894
S3150802A97019461046FFF784FE0346FB7313E03B684D
S3150802A980172B10DC13497A6813465B0013440B44F1
S3150802A99002331B781A460E4B1B7819461046FFF7E8
S3150802A9A06FFE0346FB73BA68FB7B11461846FFF730
S3150802A9B085FEBB680133BB60BB68772B93DD00BF9E
S3150802A9C000BF1037BD4680BDA8CC0020ABAAAA2A74
S3150802A9D0CECE0020B8CE002080B500AF4FF48C72E0
S3150802A9E00021064816F09AF8054A064B10461946FB
S3150802A9F0D2231A4616F049F900BF80BDA0CD002021
S3150802AA00C3CD0020A8CC002090B482B000AF044683
S3150802AA10084611461A462346FB710346BB710B4686
S3150802AA207B7113463B71FA790E4913465B00134450
S3150802AA300B44BA791A70FA790A4913465B00134429
S3150802AA400B4401337A791A70FA79064913465B0080
S3150802AA5013440B4402333A791A7000BF0837BD46CD
S3150802AA6090BC7047B8CE002080B584B000AFF860BD
S3150802AA70B9601346FB80FB881A46B968F86808F07D
S3150802AA80EBFE0346002B01D0002300E00123184603
S3150802AA901037BD4680BD000080B582B000AF786031
S3150802AAA0FFF710FFFFF798FF4FF48C720449786896
S3150802AAB0FFF7DAFF034618460837BD4680BD00BFD2
S3150802AAC0A0CD00200D488546FFF7A4F90C480D498C
S3150802AAD00D4A002302E0D458C4500433C4188C42E9
S3150802AAE0F9D30A4A0A4C002301E013600432A2424F
S3150802AAF0FBD316F08DF8FDF713FAFEE700000A20DD
S3150802AB00000000206809002040680408680900203F
S3150802AB106CE40020FEE7000080B500AF032000F0D9
S3150802AB2012F903F015FB02460B4B1B6A03F00F03DF
S3150802AB300A49CB5C22FA03F3094A13600F20FEF78F
S3150802AB4089FC0346002B01D0012302E0FEF720F818
S3150802AB500023184680BD00BF000C02442C6304087B
S3150802AB607407002080B400AF064B1B781A46064BC2
S3150802AB701B681344044A136000BFBD465DF8047B94
S3150802AB80704700BF7C070020D0CE002080B400AFFB
S3150802AB90034B1B681846BD465DF8047B704700BF29
S3150802ABA0D0CE002080B485B000AF78607B6803F011
S3150802ABB00703FB600C4BDB68BB60BA684FF6FF0302
S3150802ABC01340BB60FB681A02BB68134343F0BF63BA
S3150802ABD043F40033BB60044ABB68D36000BF143732
S3150802ABE0BD465DF8047B704700ED00E080B400AF17
S3150802ABF0044BDB681B0A03F007031846BD465DF8DB
S3150802AC00047B704700ED00E080B483B000AF0346D2
S3150802AC10FB80B7F90630002B0BDBFB8803F01F021B
S3150802AC200749B7F906305B09012000FA02F241F832
S3150802AC30232000BF0C37BD465DF8047B704700BF72
S3150802AC4000E100E080B483B000AF0346FB80B7F9A9
S3150802AC500630002B12DBFB8803F01F020A49B7F9FC
S3150802AC6006305B09012000FA02F2203341F823205C
S3150802AC70BFF34F8F00BFBFF36F8F00BF00BF0C3704
S3150802AC80BD465DF8047B704700E100E080B483B0FE
S3150802AC9000AF03463960FB80B7F90630002B0ADBA2
S3150802ACA03B68DAB20C49B7F906301201D2B20B4444
S3150802ACB083F800230AE03B68DAB20849FB8803F006
S3150802ACC00F03043B1201D2B20B441A7600BF0C37AB
S3150802ACD0BD465DF8047B704700E100E000ED00E048
S3150802ACE080B489B000AFF860B9607A60FB6803F097
S3150802ACF00703FB61FB69C3F10703042B28BF04237F
S3150802AD00BB61FB690433062B02D9FB69033B00E0EE
S3150802AD1000237B614FF0FF32BB6902FA03F3DA4381
S3150802AD20BB681A407B699A404FF0FF317B6901FA8A
S3150802AD3003F3D9437B680B40134318462437BD46B1
S3150802AD405DF8047B704780B582B000AF786078689A
S3150802AD50FFF728FF00BF0837BD4680BD80B586B01D
S3150802AD6000AF0346B9607A60FB81FFF73FFF78615F
S3150802AD707A68B9687869FFF7B3FF0246B7F90E3001
S3150802AD8011461846FFF782FF00BF1837BD4680BD39
S3150802AD9080B582B000AF0346FB80B7F90630184685
S3150802ADA0FFF732FF00BF0837BD4680BD80B582B0C7
S3150802ADB000AF0346FB80B7F906301846FFF742FF95
S3150802ADC000BF0837BD4680BD80B584B000AF786045
S3150802ADD0FFF7DCFEF8607B68002B01D10123DFE078
S3150802ADE07B68DB68B3F5806F7B681B686E4A9342A3
S3150802ADF000F09F807B681B686C4A934200F099803A
S3150802AE007B681B686A4A934200F093807B681B68DA
S3150802AE10684A934200F08D807B681B68664A9342B3
S3150802AE2000F087807B681B68644A934200F0818041
S3150802AE307B681B68624A93427BD07B681B68614ABF
S3150802AE40934276D07B681B685F4A934271D07B68CF
S3150802AE501B685E4A93426CD07B681B685C4A9342C5
S3150802AE6067D07B681B685B4A934262D07B681B6823
S3150802AE70594A93425DD07B681B68584A934258D018
S3150802AE807B681B68564A934253D07B681B68554AAF
S3150802AE9093424ED07B681B68534A934249D07B68DB
S3150802AEA01B68524A934244D07B681B68504A9342B5
S3150802AEB03FD07B681B684F4A93423AD07B681B682F
S3150802AEC04D4A934235D07B681B684C4A934230D030
S3150802AED07B681B684A4A93422BD07B681B68494A9F
S3150802AEE0934226D07B681B68474A934221D07B68E7
S3150802AEF01B68464A93421CD07B681B68444A9342A5
S3150802AF0017D07B681B68434A934212D07B681B683A
S3150802AF10414A93420DD07B681B68404A934208D047
S3150802AF207B681B683E4A934203D07B681B683D4A8E
S3150802AF3093427B68002283F84C207B68022283F8BE
S3150802AF4054207B681B685A697B681B6842F00602B4
S3150802AF505A610FE0FFF71AFE0246FB68D31A052B61
S3150802AF6008D97B6810229A657B68032283F85420E5
S3150802AF70012315E07B681B685B6903F00103002B5C
S3150802AF80E8D1786800F03CFB7B685A6B7B681A65E7
S3150802AF907B6800229A657B68012283F85420002385
S3150802AFA018461037BD4680BD500002405000025078
S3150802AFB0D0000240D0000250500102405001025017
S3150802AFC0D0010240D0010250500202405002025003
S3150802AFD0D0020240D00202505003024050030250EF
S3150802AFE0D0030240D00302505010024050100250C3
S3150802AFF0D0100240D0100250501102405011025097
S3150802B000D0110240D0110250501202405012025082
S3150802B010D0120240D012025050130240501302506E
S3150802B020D0130240D013025080B584B000AFF86046
S3150802B030B9607A603B60FB68002B01D101234FE0BF
S3150802B040FB6893F84C30012B01D1022348E0FB68D8
S3150802B050012283F84C20FB6893F85430DBB2012BAB
S3150802B06036D1FB68022283F85420FB6800229A65CF
S3150802B0703B687A68B968F86800F09DFAFB681B684D
S3150802B0805A69FB681B6842F4BA425A61FB685B6EEE
S3150802B090002B07D0FB681B685A69FB681B6842F4D9
S3150802B0A000725A61FB681B6F002B07D0FB681B688E
S3150802B0B05A69FB681B6842F400525A61FB681B68AE
S3150802B0C05A69FB681B6842F001025A61002307E0CD
S3150802B0D0FB6840229A65FB68002283F84C2001230C
S3150802B0E018461037BD4680BD80B584B000AF78607B
S3150802B0F0FFF74CFDF8607B68002B01D101236BE05A
S3150802B1007B6893F85430DBB2022B08D07B68202286
S3150802B1109A657B68002283F84C2001235CE07B68F1
S3150802B1201B685A697B681B6842F004025A617B688D
S3150802B130052283F8542020E0FFF728FD0246FB6823
S3150802B140D31A052B19D97B689B6D43F010027B68CD
S3150802B1509A657B68032283F854207B681B6D03F08B
S3150802B1608003002B03D07B685B6F01221A737B680E
S3150802B170002283F84C2001232EE07B681B681B699A
S3150802B18003F40053002BD7D07B681B685A697B6887
S3150802B1901B6842F002025A617B68042283F8542033
S3150802B1A07B681B684FF4FE42DA607B68012283F8EB
S3150802B1B054207B681B6D03F08003002B07D07B6845
S3150802B1C05B6F01221A737B681B6800229A647B688C
S3150802B1D0002283F84C20002318461037BD4680BD4E
S3150802B1E080B483B000AF78607B68002B01D101235D
S3150802B1F019E07B6893F85430DBB2022B04D07B68E3
S3150802B20020229A6501230EE07B68042283F85420E3
S3150802B2107B681B685B697A68126843F4005343F0DB
S3150802B22004035361002318460C37BD465DF8047BB8
S3150802B230704780B586B000AF78607B681B6823F4D8
S3150802B2407F6323F00F037B617B681B68C3F30B03E1
S3150802B250503BDB0903F01F03012202FA03F33B61A9
S3150802B2607B69DB683A691340FB60FB68002B00F0D8
S3150802B27054817B681B681B6903F48063002B11D019
S3150802B2807B681B685B6903F48063002B0AD07B68C2
S3150802B2901B684FF48062DA607B689B6D43F001029B
S3150802B2A07B689A657B681B681B6903F40063002B3D
S3150802B2B011D07B681B685B6903F40063002B0AD014
S3150802B2C07B681B684FF40062DA607B689B6D43F00B
S3150802B2D002027B689A657B681B681B6903F48053C4
S3150802B2E0002B11D07B681B685B6903F48053002B23
S3150802B2F00AD07B681B684FF48052DA607B689B6DC4
S3150802B30043F004027B689A657B681B681B6903F431
S3150802B3108043002B11D07B681B685B6903F480436A
S3150802B320002B0AD07B681B684FF48042DA607B6880
S3150802B3309B6D43F008027B689A657B681B681B69EC
S3150802B34003F40073002B13D07B681B685B6903F454
S3150802B3500073002B0CD07B681B684FF40072DA600E
S3150802B3607B685B6E002B03D07B685B6E78689847B8
S3150802B3707B681B681B6903F40053002B59D07B6852
S3150802B3801B685B6903F40053002B52D07B681B6869
S3150802B3904FF40052DA607B6893F85430DBB2042B20
S3150802B3A03BD17B681B685A697B681B6822F400528A
S3150802B3B05A617B681B685A697B681B6842F00202FD
S3150802B3C05A617B681B685B6903F00103002B04D092
S3150802B3D07B68032283F8542003E07B68012283F802
S3150802B3E054207B681B6D03F08003002B07D07B6813
S3150802B3F05B6F01221A737B681B6800229A647B685A
S3150802B400002283F84C207B68DB6E002B00F08780D5
S3150802B4107B68DB6E7868984781E07B68052283F84B
S3150802B42054207B681B6F002B03D07B681B6F7868E0
S3150802B43098477B681B681B6903F48073002B39D015
S3150802B4407B681B685B6903F48073002B32D07B68C8
S3150802B4501B6D03F08003002B12D07B681B68DB6F21
S3150802B460002B16D17B681B689B6C002B11D17B685D
S3150802B470012283F854207B685B6F01221A7308E065
S3150802B4807B681B689B6C002B03D17B68012283F8BF
S3150802B49054207B681B684FF44072DA607B6800228E
S3150802B4A083F84C207B681B6E002B03D07B681B6ECF
S3150802B4B0786898477B689B6D002B31D07B681B6840
S3150802B4C05A697B681B6842F002025A617B681B68EC
S3150802B4D05B6903F00103002B04D07B68032283F81F
S3150802B4E0542003E07B68012283F854207B681B6D95
S3150802B4F003F08003002B03D07B685B6F01221A736B
S3150802B5007B68002283F84C207B689B6E002B07D051
S3150802B5107B689B6E7868984702E000BF00E000BF30
S3150802B5201837BD4680BD80B483B000AF78607B68AB
S3150802B5309B6D18460C37BD465DF8047B704780B490
S3150802B54085B000AF786039607B68002B01D1012392
S3150802B5502BE07B681B6823F47F6323F00F03FB60F1
S3150802B5607B681B68C3F30B03503BDB0903F01F031D
S3150802B570012202FA03F3BB603B6803F01003002BB7
S3150802B58012D03B6803F01103112B06D1FB685A68E7
S3150802B590BB681A43FB685A6006E0FB685A68BB68D0
S3150802B5A0DB431A40FB685A60002318461437BD4627
S3150802B5B05DF8047B704780B485B000AFF860B96067
S3150802B5C07A603B60FB681B689B6C1B0C1B043A6821
S3150802B5D091B2FA6812680B439364FB681B684FF4CE
S3150802B5E0FE42DA60FB681B68BA68DA64FB681B68A5
S3150802B5F07A681A6500BF1437BD465DF8047B704742
S3150802B60080B485B000AF78607B681B6AFB607B6894
S3150802B6101B685B6923F443017B681B68FA680A4363
S3150802B6205A617B685A697B68DB691A437B681B69BE
S3150802B6301A437B689B691343FB607B681B68534A02
S3150802B640934200F0A0807B681B68514A934200F03F
S3150802B6509A807B681B684F4A934200F094807B6805
S3150802B6601B684D4A934200F08E807B681B684B4AE2
S3150802B670934200F088807B681B68494A934200F02F
S3150802B68082807B681B68474A93427CD07B681B682A
S3150802B690454A934277D07B681B68444A934272D0E4
S3150802B6A07B681B68424A93426DD07B681B68414A95
S3150802B6B0934268D07B681B683F4A934263D07B6893
S3150802B6C01B683E4A93425ED07B681B683C4A93429B
S3150802B6D059D07B681B683B4A934254D07B681B68E7
S3150802B6E0394A93424FD07B681B68384A93424AD0FC
S3150802B6F07B681B68364A934245D07B681B68354A85
S3150802B700934240D07B681B68334A93423BD07B689E
S3150802B7101B68324A934236D07B681B68304A93428A
S3150802B72031D07B681B682F4A93422CD07B681B68F2
S3150802B7302D4A934227D07B681B682C4A934222D013
S3150802B7407B681B682A4A93421DD07B681B68294A74
S3150802B750934218D07B681B68274A934213D07B68AA
S3150802B7601B68264A93420ED07B681B68244A93427A
S3150802B77009D07B681B68234A934204D07B681B68FE
S3150802B780214A934242D1012341E000BF50000240C0
S3150802B79050000250D0000240D00002505001024030
S3150802B7A050010250D0010240D0010250500202401C
S3150802B7B050020250D0020240D00202505003024008
S3150802B7C050030250D0030240D003025050100240E8
S3150802B7D050100250D0100240D010025050110240B0
S3150802B7E050110250D0110240D0110250501202409C
S3150802B7F050120250D0120240D01202505013024088
S3150802B80050130250D0130240D01302500023002BCB
S3150802B81012D07B68DA6A7B689B6A013B1B0503F0D8
S3150802B8207C731A437B685B6A013B1B0103F47C73D6
S3150802B8301343FA681343FB607B681B681B6C03F0AF
S3150802B84080217B681B68FA680A431A647B689A68CF
S3150802B8507B685B68DBB21A437B681B6B1343FB602E
S3150802B8607B68DB68B3F5806F40F0B0807B681B6845
S3150802B870844A934200F0A0807B681B68824A9342FE
S3150802B88000F09A807B681B68804A934200F0948095
S3150802B8907B681B687E4A934200F08E807B681B6831
S3150802B8A07C4A934200F088807B681B687A4A9342F6
S3150802B8B000F082807B681B68784A93427CD07B685A
S3150802B8C01B68774A934277D07B681B68754A93420E
S3150802B8D072D07B681B68744A93426DD07B681B687A
S3150802B8E0724A934268D07B681B68714A934263D056
S3150802B8F07B681B686F4A93425ED07B681B686E4AF8
S3150802B900934259D07B681B686C4A934254D07B6831
S3150802B9101B686B4A93424FD07B681B68694A9342FD
S3150802B9204AD07B681B68684A934245D07B681B6885
S3150802B930664A934240D07B681B68654A93423BD06D
S3150802B9407B681B68634A934236D07B681B68624AE7
S3150802B950934231D07B681B68604A93422CD07B683D
S3150802B9601B685F4A934227D07B681B685D4A9342ED
S3150802B97022D07B681B685C4A93421DD07B681B6891
S3150802B9805A4A934218D07B681B68594A934213D085
S3150802B9907B681B68574A93420ED07B681B68564AD7
S3150802B9A0934209D07B681B68544A934204D07B6849
S3150802B9B01B68534A934201D1012300E00023002B5E
S3150802B9C00DD0FB6843F48063FB6008E07B68DB68A4
S3150802B9D0B3F5007F03D1FB6843F40073FB607B6811
S3150802B9E05B6BFA681343FB607B681B685A6C454BB2
S3150802B9F013407A681268F9680B4353647B681B68BC
S3150802BA0000229A647B681B682A4A934222D07B6882
S3150802BA101B68294A93421DD07B681B68274A9342B2
S3150802BA2018D07B681B68264A934213D07B681B682A
S3150802BA30304A93420ED07B681B682F4A934209D03C
S3150802BA407B681B682D4A934204D07B681B682C4A84
S3150802BA50934201D1012300E00023002B07D07B6823
S3150802BA601B6800225A657B681B6800229A657B68F8
S3150802BA701B680022DA6700BF1437BD465DF8047BEF
S3150802BA80704700BF5000024050000250D0000240EA
S3150802BA90D00002505001024050010250D00102402B
S3150802BAA0D00102505002024050020250D002024017
S3150802BAB0D00202505003024050030250D003024003
S3150802BAC0D00302505010024050100250D0100240CB
S3150802BAD0D01002505011024050110250D0110240AB
S3150802BAE0D01102505012024050120250D012024097
S3150802BAF0D01202505013024050130250D013024083
S3150802BB00D01302500021C03C80B586B000AF7860E1
S3150802BB107B68002B03D07B685B6F002B01D1012366
S3150802BB2082E07B6893F85430FB757B681B685B6917
S3150802BB3003F480333B61FB7D012B05D0FB7D022B91
S3150802BB406AD13B69002B67D07B6893F85430DBB225
S3150802BB50012B57D17B6893F84C30012B01D1022374
S3150802BB6062E07B68012283F84C207B68022283F814
S3150802BB7054207B685B6F02221A737B6800229A65DF
S3150802BB807B685B6F00221A617B681B685A697B684F
S3150802BB901B6842F4BA425A617B685B6E002B07D077
S3150802BBA07B681B685A697B681B6842F400725A6193
S3150802BBB07B681B6F002B07D07B681B685A697B68FA
S3150802BBC01B6842F400525A617B685B6F1B6807F177
S3150802BBD00C010022184600F02BF87B685B6F1B6885
S3150802BBE019467B681A680B0C1B0413607B685B6F2B
S3150802BBF01B681A464FF6FC731340F9687A6812688E
S3150802BC000B43D3677B681B685A697B681B6842F0DB
S3150802BC1001025A61002307E07B6840229A657B6825
S3150802BC20002283F84C20012318461837BD4680BDEA
S3150802BC3080B485B000AFF860B9607A60FB681B6AA9
S3150802BC4003F00203002B0CD0BB68002B02D0BB68A2
S3150802BC500D4A1A607B68002B0FD07B6807221A6090
S3150802BC600BE0BB68002B02D0BB68084A1A607B68E7
S3150802BC70002B02D07B6805221A6000BF1437BD4626
S3150802BC805DF8047B704700BF000001FE000001F862
S3150802BC9080B584B000AF78607B68002B01D10123A0
S3150802BCA047E17B6893F85C30DBB2002B06D17B68F0
S3150802BCB0002283F85D207868FCF772FF7B681B68B0
S3150802BCC09A697B681B6822F010029A61FEF75EFF8A
S3150802BCD0F86012E0FEF75AFF0246FB68D31A0A2BEF
S3150802BCE00BD97B681B6E43F001027B681A667B6878
S3150802BCF0032283F85C2001231BE17B681B689B698E
S3150802BD0003F00803082BE5D07B681B689A697B68F1
S3150802BD101B6842F001029A61FEF738FFF86012E0EA
S3150802BD20FEF734FF0246FB68D31A0A2B0BD97B6847
S3150802BD301B6E43F001027B681A667B68032283F84E
S3150802BD405C200123F5E07B681B689B6903F001030D
S3150802BD50002BE5D07B681B689A697B681B6842F0F2
S3150802BD6002029A617B681B68744A934203D1744A39
S3150802BD707B685B6813607B681B7C012B08D17B6838
S3150802BD801B689A697B681B6822F040029A6107E081
S3150802BD907B681B689A697B681B6842F040029A6155
S3150802BDA07B685B7C012B08D17B681B689A697B6878
S3150802BDB01B6842F480429A6107E07B681B689A69AD
S3150802BDC07B681B6822F480429A617B689B7C012B04
S3150802BDD008D17B681B689A697B681B6822F48052C3
S3150802BDE09A6107E07B681B689A697B681B6842F45C
S3150802BDF080529A617B681B689B6923F440717B6851
S3150802BE009A687B681B680A439A617B681B689A6909
S3150802BE107B681B6822F0A4029A617B681B681A6910
S3150802BE207B681B6822F010021A617B68DB68012BAB
S3150802BE3008D17B681B689A697B681B6842F0040212
S3150802BE409A612CE07B68DB68002B28D07B68DB686C
S3150802BE50022B1CD07B681B689A697B681B6842F0B8
S3150802BE6080029A617B681B681A697B681B6842F0C4
S3150802BE7010021A617B68DB68032B10D17B681B688A
S3150802BE809A697B681B6842F020029A6107E07B6820
S3150802BE901B689A697B681B6842F020029A617B6874
S3150802BEA09B69013B5A067B68DB69013B1B021A4305
S3150802BEB07B681B6A013B42EA03017B685B69013BBB
S3150802BEC01A047B681B680A43DA617B689B68B3F5C8
S3150802BED0407F15D17B689B6A5A1E7B68DB6A013BE9
S3150802BEE01B021A437B681B6B013B1B0142EA0301D7
S3150802BEF07B685B6A013B1A047B681B680A43DA6043
S3150802BF007B681B68D3F8C0107B68DA6B7B681B6892
S3150802BF100A43C3F8C020786800F0C8FC7B68002290
S3150802BF209A657B6800221A667B68012283F85C2080
S3150802BF30002318461037BD4680BD00BF00A4004046
S3150802BF4000A5004080B487B000AF786039607B688E
S3150802BF5093F85C30FB75FB7D012B02D0FB7D022B2F
S3150802BF603DD13B681B68002B19D13B689B689A0731
S3150802BF703B68DB68DB061A433B681B691B041A43EA
S3150802BF803B685B6913433B617B681A6C3B685B6879
S3150802BF909B001344BB60BB683A691A601DE03B68A4
S3150802BFA0DB685A073B681B6913433B613B689B681E
S3150802BFB09A073B685B691343FB607B685A6C3B686C
S3150802BFC05B68DB001344BB60BB683A691A60BB68EE
S3150802BFD00433BB60BB68FA681A60002306E07B6814
S3150802BFE01B6E43F002027B681A66012318461C3749
S3150802BFF0BD465DF8047B704780B485B000AFF86033
S3150802C000B9607A603B60FB6893F85C30DBB2012B5F
S3150802C01016D1FB681B68D3F8803023F03F01BB6852
S3150802C0201A017B689B001A433B685B001A43BB698B
S3150802C0301A43FB681B680A43C3F88020002306E0FC
S3150802C040FB681B6E43F00402FB681A660123184656
S3150802C0501437BD465DF8047B704780B483B000AFE1
S3150802C06078607B6893F85C30DBB2012B10D17B6871
S3150802C070022283F85C207B681B689A697B681B68C6
S3150802C08022F001029A617B6800221A66002306E002
S3150802C0907B681B6E43F004027B681A660123184606
S3150802C0A00C37BD465DF8047B704780B586B000AF95
S3150802C0B0F860B9607A60FB6893F85C30DBB2022BF1
S3150802C0C02CD1FB681B68D3F8C43003F40013002B89
S3150802C0D007D0FB681B6E43F40072FB681A660123DD
S3150802C0E023E0FB681B68D3F8C4301B0C03F0030378
S3150802C0F07B617B697A68B968F86800F039FCFB6885
S3150802C1001B6801217A6901FA02F2C3F8CC200122DE
S3150802C1107B699A40FB689A65002306E0FB681B6EFA
S3150802C12043F00802FB681A66012318461837BD460B
S3150802C13080BD80B483B000AF78607B689B6D18467B
S3150802C1400C37BD465DF8047B7047000080B48BB09F
S3150802C15000AFF860B9607A603B600023FB61FB6858
S3150802C16093F85C30FB76FB7E022B40F0E880BB68D6
S3150802C170402B37D1FB681B68D3F8903003F00F03C6
S3150802C180002B07D1FB681B6E43F48072FB681A66A4
S3150802C1900123DBE0FB681B68D3F890301B0E03F023
S3150802C1A00103012B0AD1FB681B68D3F880305B0AAE
S3150802C1B003F00103012B01D10123FB61FB681B6814
S3150802C1C0D3F890301B0A03F00303FA691344FB61A0
S3150802C1D0FB68996CFA691346DB001344DB000B44CF
S3150802C1E07B6236E0FB681B68D3F8983003F00F03CE
S3150802C1F0002B07D1FB681B6E43F48072FB681A6634
S3150802C2000123A3E0FB681B68D3F898301B0E03F0E2
S3150802C2100103012B0AD1FB681B68D3F880301B0A7D
S3150802C22003F00103012B01D10123FB61FB681B68A3
S3150802C230D3F898301B0A03F00303FA691344FB6127
S3150802C240FB68D96CFA691346DB001344DB000B441E
S3150802C2507B627B6A1B6803F080427B685A607B6854
S3150802C2605B68002B07D17B6A1B689B0CC3F30A0227
S3150802C2707B681A6005E07B6A1B6823F060427B686C
S3150802C2801A607B6A1B6803F000527B689A607B6AB5
S3150802C2901B6803F000427B681A617B6A04337B627F
S3150802C2A07B6A1B689AB27B68DA617B6A1B681B0C1D
S3150802C2B003F00F027B68DA607B6A1B6803F480125C
S3150802C2C07B685A617B6A1B6803F400127B689A6171
S3150802C2D07B6A1B681B0E03F07F027B681A627B6A05
S3150802C2E01B68DA0F7B685A627B6A04337B627B6A55
S3150802C2F07B6100233B620AE07A693B6A1A44396821
S3150802C3003B6A0B4412781A703B6A01333B627B68BC
S3150802C310DB68114AD35C1A463B6A9342ECD3BB6884
S3150802C320402B05D1FB681B68FA69C3F8942004E020
S3150802C330FB681B68FA69C3F89C20002306E0FB68C1
S3150802C3401B6E43F00802FB681A66012318462C374F
S3150802C350BD465DF8047B70474463040880B483B025
S3150802C36000AF786039607B681B68D3F8C8203B68E1
S3150802C3701340002B01D1002300E0012318460C3795
S3150802C380BD465DF8047B704780B485B000AF78601F
S3150802C39039603B68402B07D17B681B68D3F890301D
S3150802C3A003F00F03FB6006E07B681B68D3F898303E
S3150802C3B003F00F03FB60FB6818461437BD465DF8A9
S3150802C3C0047B704780B487B000AFF860B9607A60C2
S3150802C3D0FB6893F85C30FB75FB7D012B03D0FB7D74
S3150802C3E0022B40F0C880FB681B689B6D3B61BB68EB
S3150802C3F003F00703002B04D03B6903F00103002B6B
S3150802C4003BD0BB6803F03803002B04D03B6903F02A
S3150802C4100203002B31D0BB6803F4E073002B04D06F
S3150802C4203B6903F00403002B27D0BB6803F4F053DF
S3150802C430002B04D03B6903F00803002B1DD0BB6810
S3150802C44003F46043002B04D03B6903F01003002B6E
S3150802C45013D0BB6803F44033002B04D03B6903F0C6
S3150802C4602003002B09D0BB6803F47C03002B0CD0F5
S3150802C4703B6903F04003002B07D1FB681B68DA6DA2
S3150802C480FB681B6842F00102DA65BB6803F0070322
S3150802C490002B04D03B6903F00103002B3BD1BB6898
S3150802C4A003F03803002B04D03B6903F00203002B88
S3150802C4B031D1BB6803F4E073002B04D03B6903F067
S3150802C4C00403002B27D1BB6803F4F053002B04D0D6
S3150802C4D03B6903F00803002B1DD1BB6803F46043D4
S3150802C4E0002B04D03B6903F01003002B13D1BB6861
S3150802C4F003F44033002B04D03B6903F02003002BDE
S3150802C50009D1BB6803F47C03002B0CD03B6903F00A
S3150802C5104003002B07D0FB681B68DA6DFB681B68B3
S3150802C52042F00202DA65BB6803F08003002B09D0E9
S3150802C530FB681B68D3F8DC10FB681B687A680A4339
S3150802C540C3F8DC20BB6803F48073002B09D0FB68B0
S3150802C5501B68D3F8E010FB681B687A680A43C3F8BD
S3150802C560E020FB681B68596DFB681B68BA680A43BA
S3150802C5705A65002306E0FB681B6E43F00202FB685D
S3150802C5801A66012318461C37BD465DF8047B7047B8
S3150802C59080B58CB000AF78607B681B681B6D03F4AE
S3150802C5A0E053FB627B681B685B6DFA6A1340FB62A9
S3150802C5B07B681B681B6D03F00703BB627B681B68FD
S3150802C5C05B6DBA6A1340BB627B681B681B6D03F01E
S3150802C5D038037B627B681B685B6D7A6A13407B62F1
S3150802C5E07B681B681B6D03F471033B627B681B68DF
S3150802C5F05B6D3A6A13403B627B681B681B6D03F4EA
S3150802C6006023FB617B681B685B6DFA691340FB61FB
S3150802C6107B681B685B6DBB617B681B681B6D7B61F6
S3150802C6207B6903F04003002B0BD0BB6903F0400380
S3150802C630002B06D07B681B6840221A65786800F0D2
S3150802C64016F97B6903F48073002B19D0BB6903F4CE
S3150802C6508073002B14D07B681B68D3F8D8303B61F3
S3150802C6607B681B68D3F8E0303A6913403B617B6804
S3150802C6701B684FF480721A653969786800F0D8F831
S3150802C680FB6A002B07D07B681B68FA6A1A65F96A87
S3150802C690786800F0A2F8BB6A002B07D07B681B6893
S3150802C6A0BA6A1A65B96A7868FCF71EF97B6A002BBA
S3150802C6B007D07B681B687A6A1A65796A786800F017
S3150802C6C097F87B6903F40073002B0CD0BB6903F45B
S3150802C6D00073002B07D07B681B684FF400721A653B
S3150802C6E0786800F090F87B6903F08003002B18D075
S3150802C6F0BB6903F08003002B13D07B681B68D3F851
S3150802C700D430FB607B681B68D3F8DC30FA681340C8
S3150802C710FB607B681B6880221A65F968786800F0F6
S3150802C7207CF87B6903F40053002B0CD0BB6903F435
S3150802C7300053002B07D07B681B684FF400521A651A
S3150802C740786800F080F87B6903F40043002B0CD06C
S3150802C750BB6903F40043002B07D07B681B684FF4C0
S3150802C76000421A65786800F078F87B6903F480431A
S3150802C770002B0FD0BB6903F48043002B0AD07B68D9
S3150802C7801B684FF480421A657B681B6E43F0800271
S3150802C7907B681A66FB69002B07D07B681B68FA69F7
S3150802C7A01A65F969786800F076F83B6A002B09D0B1
S3150802C7B07B681B683A6A1A657B681A6E3B6A1A4373
S3150802C7C07B681A667B681B6E002B02D0786800F0BD
S3150802C7D058F800BF3037BD4680BD80B483B000AF7D
S3150802C7E07860396000BF0C37BD465DF8047B704738
S3150802C7F080B483B000AF7860396000BF0C37BD469D
S3150802C8005DF8047B704780B483B000AF786000BFE0
S3150802C8100C37BD465DF8047B704780B483B000AF21
S3150802C8207860396000BF0C37BD465DF8047B7047F7
S3150802C83080B483B000AF7860396000BF0C37BD465C
S3150802C8405DF8047B704780B483B000AF786000BFA0
S3150802C8500C37BD465DF8047B704780B483B000AFE1
S3150802C860786000BF0C37BD465DF8047B704780B41C
S3150802C87083B000AF786000BF0C37BD465DF8047B15
S3150802C880704780B483B000AF786000BF0C37BD46EE
S3150802C8905DF8047B704780B483B000AF7860396076
S3150802C8A000BF0C37BD465DF8047B704780B485B07F
S3150802C8B000AF78602C4BBB607B681B682B4A93429F
S3150802C8C003D1BB6803F55473BB607B68BA681A6404
S3150802C8D07B681B68D3F8803023F4F8117B685B6B9E
S3150802C8E01A047B681B680A43C3F88020BB6803F1F5
S3150802C8F070027B685A647B681B68D3F8803023F021
S3150802C90070617B689B6B1A067B681B680A43C3F8CF
S3150802C9108020BB6803F1B0027B689A64BB6803F5A2
S3150802C920C4727B68DA64BB6803F518727B681A6599
S3150802C930BB6803F51E727B685A65BB68FB6005E037
S3150802C940FB6800221A60FB680433FB60BB6803F5C8
S3150802C9505473FA689A42F3D300BF00BF1437BD4630
S3150802C9605DF8047B704700BF00AC004000A8004099
S3150802C97080B489B000AFF860B9607A603B60BB6882
S3150802C9805B68002B0AD1BB681A69BB689B681A43A5
S3150802C990BB681B689B041343FB610AE0BB681A6900
S3150802C9A0BB689B681A43BB681B68134343F0804302
S3150802C9B0FB61BB681B6A1A06BB68DB691A43BB685C
S3150802C9C09B691A43BB685B691A43BB68DB681B042D
S3150802C9D013433B61FB68596D3A681346DB001344FF
S3150802C9E0DB000B44BB61BB69FA691A60BB69043395
S3150802C9F0BB61BB693A691A60BB690433BB61002330
S3150802CA007B6120E07B6903337A6813441B781A0634
S3150802CA107B69023379680B441B781B041A437B69CA
S3150802CA20013379680B441B781B02134379687A69C8
S3150802CA300A4412781A43BB691A60BB690433BB619C
S3150802CA407B6904337B61BB68DB68064AD35C1A469A
S3150802CA507B699342D6D300BF00BF2437BD465DF833
S3150802CA60047B70474463040880B588B000AFF86059
S3150802CA70B9607A60324B1B78012B01D102235AE046
S3150802CA802F4B01221A702E4B00225A604FF47A70ED
S3150802CA9000F0A4F80346FB77FB7F002B47D1284A10
S3150802CAA0FB689360274BBB61FB6823F00043022BAC
S3150802CAB004D17968B86800F0DFF81BE0FB68224AFF
S3150802CAC0934203D0FB68214A934204D17968B86835
S3150802CAD000F00EF90EE0FB6823F000431C4A93426D
S3150802CAE004D17968B86800F04FF903E07968B86844
S3150802CAF000F04AF94FF47A7000F070F80346FB77B3
S3150802CB00BB691A68FB6823F0304323F00403DB434E
S3150802CB101A40BB691A60FB680C4A934207D10D4B4F
S3150802CB207B617B691B6823F004027B691A60044BEC
S3150802CB3000221A70FB7F18462037BD4680BD00BF0B
S3150802CB40800700202820024002000010060000107C
S3150802CB50020000404020024080B483B000AF0023A8
S3150802CB60FB710D4B9B6A03F00103002B0DD00A4B98
S3150802CB700A4A5A60084B0A4A5A60074B9B6A03F0EC
S3150802CB800103002B01D00123FB71FB7918460C37F0
S3150802CB90BD465DF8047B70470020024023016745C5
S3150802CBA0AB89EFCD80B483B000AF0023FB710A4B8B
S3150802CBB09B6A094A43F001039362074B9B6A03F097
S3150802CBC00103002B01D10123FB71FB7918460C37AF
S3150802CBD0BD465DF8047B70470020024080B586B0EA
S3150802CBE000AF7860FDF7D2FF7861204B3B6110E019
S3150802CBF07B68B3F1FF3F0CD0FDF7C8FF02467B699D
S3150802CC00D31A7A689A4202D37B68002B01D103238E
S3150802CC1027E03B691B6803F00B03002BE8D1144B92
S3150802CC20FB603B691B6803F47E03BB60BB68002B91
S3150802CC300CD0104B5A68BB6813430E4A5360BB6844
S3150802CC4003F47E02FB681A6001230AE03B691B684B
S3150802CC5003F48033002B03D0FB684FF480321A604A
S3150802CC60002318461837BD4680BD00BF2020024063
S3150802CC70302002408007002080B48BB000AF786075
S3150802CC803960042387F827307B683B623B68FB617F
S3150802CC90164BBB61BB691B6843F00202BB691A608B
S3150802CCA0EFF310833B613B697B6172B600BFFB6998
S3150802CCB01A683B6A1A603B6A04333B62FB690433AF
S3150802CCC0FB6197F82730013B87F8273097F827301A
S3150802CCD0002BECD17B69FB60FB6883F3108800BFED
S3150802CCE000BF2C37BD465DF8047B704728200240FA
S3150802CCF080B48BB000AF78603960042387F8273098
S3150802CD007B683B623B68FB611C4BBB611C4B7B61CE
S3150802CD10BB691B6843F00202BB691A607B691A6821
S3150802CD20184B9B6803F004031A437B691A60EFF3F6
S3150802CD301083FB60FB683B6172B600BFFB691A6829
S3150802CD403B6A1A603B6A04333B62FB690433FB6144
S3150802CD5097F82730013B87F8273097F82730002BBA
S3150802CD60ECD13B69BB60BB6883F3108800BF00BF88
S3150802CD702C37BD465DF8047B704700BF2820024069
S3150802CD80402002408007002080B485B000AF78605A
S3150802CD903960094BFB60FB681B6843F00202FB68BB
S3150802CDA01A603A687B68128892B21A8000BF1437F2
S3150802CDB0BD465DF8047B70472820024080B586B0E0
S3150802CDC000AF786039603A4B1B78012B01D10223F8
S3150802CDD06AE0374B01221A70354B00225A604FF42B
S3150802CDE07A70FFF7FBFE0346FB75FB7D002B57D1D6
S3150802CDF07B681B682E4A93602E4BFB607B681B6818
S3150802CE0023F0004348F2080293420BD17B685B6821
S3150802CE10184600F053F84FF47A70FFF7DFFE034620
S3150802CE20FB7533E07B681B68234A934208D100F0FE
S3150802CE30B5F84FF47A70FFF7D1FE0346FB7525E085
S3150802CE403B684FF0FF321A607B689B683B6115E0CE
S3150802CE507B685B681946386900F068F84FF47A709F
S3150802CE60FFF7BCFE0346FB75FB7D002B03D03B6830
S3150802CE703A691A600AE03B6901333B617B68DA6802
S3150802CE807B689B6813443A699A42E1D3FB681A683D
S3150802CE907B681B6823F00043DB431A40FB681A6071
S3150802CEA0034B00221A70FB7D18461837BD4680BD13
S3150802CEB080070020282002400800008080B485B040
S3150802CEC000AF7860184BFB607B6803F00303032B03
S3150802CED008D1FB681B6843F4004343F02003FA6851
S3150802CEE013601BE07B6803F00103002B09D0FB6883
S3150802CEF01B6823F0004323F0280343F02802FB684B
S3150802CF001A607B6803F00203002B07D0FB681B68D4
S3150802CF1043F0004343F02803FA68136000BF14374E
S3150802CF20BD465DF8047B70472820024080B485B070
S3150802CF3000AF78603960184BFB603B6803F0010369
S3150802CF40002B11D0FB681B6823F0004323F4FE5321
S3150802CF50FA681360FB681A687B689B01134343F0FF
S3150802CF602402FB681A6010E0FB681B6823F4FE5271
S3150802CF70FB681A60FB681A687B689B01134343F0D7
S3150802CF80004343F02403FA68136000BF1437BD4612
S3150802CF905DF8047B704700BF2820024080B483B046
S3150802CFA000AF074B7B607B681B6843F008027B680F
S3150802CFB01A6000BF0C37BD465DF8047B704700BF98
S3150802CFC04020024080B487B000AF78603960002301
S3150802CFD03B6136E13B681A6801213B6901FA03F3B2
S3150802CFE01340FB60FB68002B00F028813B685B68F6
S3150802CFF0022B03D03B685B68122B25D13B69DA0802
S3150802D0007B68083253F822307B613B6903F00703D9
S3150802D0109B000F2202FA03F3DB437A6913407B6112
S3150802D0203B681B6903F00F023B6903F007039B0089
S3150802D03002FA03F37A6913437B613B69DA087B6870
S3150802D0400832796943F822107B681B687B613B6961
S3150802D0505B00032202FA03F3DB437A6913407B611E
S3150802D0603B685B6803F003023B695B0002FA03F361
S3150802D0707A6913437B617B687A691A603B685B68E5
S3150802D080012B0BD03B685B68022B07D03B685B68B9
S3150802D090112B03D03B685B68122B30D17B689B68E7
S3150802D0A07B613B695B00032202FA03F3DB437A697D
S3150802D0B013407B613B68DA683B695B0002FA03F35B
S3150802D0C07A6913437B617B687A699A607B685B68D5
S3150802D0D07B6101223B6902FA03F3DB437A69134057
S3150802D0E07B613B685B681B0903F001023B6902FA34
S3150802D0F003F37A6913437B617B687A695A603B68F2
S3150802D1005B68032B17D07B68DB687B613B695B0036
S3150802D110032202FA03F3DB437A6913407B613B6815
S3150802D1209A683B695B0002FA03F37A6913437B61E7
S3150802D1307B687A69DA603B685B6803F08053002B88
S3150802D1407CD0474A3B699B08183352F823307B61E7
S3150802D1503B6903F00303DB000F2202FA03F3DB4306
S3150802D1607A6913407B617B689A0A3E4B13403A6997
S3150802D17002F00302D20093407A6913437B6138496D
S3150802D1803B699B0818337A6941F82320344B1B689C
S3150802D1907B61FB68DB437A6913407B613B685B68AA
S3150802D1A003F48013002B03D07A69FB6813437B616F
S3150802D1B02B4A7B6913602A4B5B687B61FB68DB43FE
S3150802D1C07A6913407B613B685B6803F40013002BA2
S3150802D1D003D07A69FB6813437B61214A7B695360F2
S3150802D1E01F4BD3F884307B61FB68DB437A691340B3
S3150802D1F07B613B685B6803F40033002B03D07A69D2
S3150802D200FB6813437B61164A7B69C2F88430144B68
S3150802D210D3F880307B61FB68DB437A6913407B6114
S3150802D2203B685B6803F48033002B03D07A69FB689A
S3150802D23013437B610A4A7B69C2F880303B69013332
S3150802D2403B613B681A683B6922FA03F3002B7FF4B9
S3150802D250C1AE00BF00BF1C37BD465DF8047B7047F0
S3150802D260002002447F7F2F0080B487B000AF786029
S3150802D270396000237B61A0E001227B6902FA03F38D
S3150802D2803A6813403B613B69002B00F09380524A8F
S3150802D2907B699B08183352F82330FB607B6903F0DD
S3150802D2A00303DB000F2202FA03F3FA681340FB605A
S3150802D2B07B689A0A494B13407A6902F00302D20044
S3150802D2C09340FA689A4236D1434BD3F880203B6999
S3150802D2D0DB4341491340C1F880303F4BD3F88420E1
S3150802D2E03B69DB433C491340C1F884303A4B1A6820
S3150802D2F03B69DB43384913400B60374B5A683B6935
S3150802D300DB43354913404B607B6903F00303DB00BB
S3150802D3100F2202FA03F3FB602F4A7B699B08183334
S3150802D32052F82310FB68DA432B487B699B080A40AC
S3150802D330183340F823207B681A687B695B0003214F
S3150802D34001FA03F31A437B681A607B69DA087B6879
S3150802D350083253F822107B6903F007039B000F2259
S3150802D36002FA03F3DB437A69D20819407B6808326A
S3150802D37043F822107B689A687B695B00032101FAED
S3150802D38003F3DB431A407B689A607B685A6801217B
S3150802D3907B6901FA03F3DB431A407B685A607B68B0
S3150802D3A0DA687B695B00032101FA03F3DB431A405F
S3150802D3B07B68DA607B6901337B613A687B6922FAAA
S3150802D3C003F3002B7FF458AF00BF00BF1C37BD46DE
S3150802D3D05DF8047B704700BF002002447F7F2F0060
S3150802D3E080B485B000AF78600B467B807B681A698B
S3150802D3F07B881340002B02D00123FB7301E0002334
S3150802D400FB73FB7B18461437BD465DF8047B7047F1
S3150802D41080B483B000AF78600B467B8013467B707E
S3150802D4207B78002B03D07A887B689A6102E07A8837
S3150802D4307B689A6200BF0C37BD465DF8047B70476D
S3150802D44080B584B000AF78607B68002B01D10123D8
S3150802D45070E0786800F072F87B681B684CF6CC427C
S3150802D4601A607B681B6845F255521A607B681B680E
S3150802D4707A6852685A607B681B687A6892689A600A
S3150802D480FDF784FBF8600FE0FDF780FB0246FB68B8
S3150802D490D31A212B08D97B681B68DB6803F00203C1
S3150802D4A0002B01D0032345E07B681B68DB6803F089
S3150802D4B00203002BE8D17B681B69002B05D17B6828
S3150802D4C01B684FF480425A6106E07B681A697B68DA
S3150802D4D01B6842F440425A61FDF758FBF8600FE0B8
S3150802D4E0FDF754FB0246FB68D31A212B08D97B6841
S3150802D4F01B68DB6803F00F03002B01D0032319E036
S3150802D5007B681B68DB6803F00F03002BE8D17B6896
S3150802D5101B681A697B68DB689A4205D07B681B68B8
S3150802D5207A68D2681A6104E07B681B684AF6AA22FE
S3150802D5301A60002318461037BD4680BD80B483B0F2
S3150802D54000AF786000BF0C37BD465DF8047B7047B4
S3150802D55080B483B000AF78607B681B684AF6AA225B
S3150802D5601A60002318460C37BD465DF8047B7047DF
S3150802D57080B588B000AF78607B68002B02D10123A2
S3150802D58000F028BC944BDB6903F01803FB61924B4D
S3150802D5909B6A03F00303BB617B681B6803F01003F5
S3150802D5A0002B5BD0FB69082B05D0FB69182B14D11D
S3150802D5B0BB69022B11D17B68DB69002B02D10123DF
S3150802D5C000F008BC844B9B6923F47C127B681B6AB7
S3150802D5D01B04814913438B6140E07B68DB69002B9E
S3150802D5E023D07D4B1B687C4A43F480731360FDF796
S3150802D5F0CDFA786108E0FDF7C9FA02467B69D31AC3
S3150802D600022B01D90323E5E3734B1B6803F400736A
S3150802D610002BF0D0704B9B6923F47C127B681B6A43
S3150802D6201B046D4913438B6118E06B4B1B686A4AEE
S3150802D63023F480731360FDF7A9FA786108E0FDF711
S3150802D640A5FA02467B69D31A022B01D90323C1E341
S3150802D650614B1B6803F40073002BF0D17B681B68CF
S3150802D66003F00103002B00F0A080FB69102B05D004
S3150802D670FB69182B09D1BB69032B06D17B685B684A
S3150802D680002B40F092800123A4E37B685B68B3F524
S3150802D690803F06D1504B1B684F4A43F480331360D0
S3150802D6A058E07B685B68002B12D14B4B1B684A4AD1
S3150802D6B023F480331360484B1B68474A23F48013CC
S3150802D6C01360454B1B68444A23F48023136041E0E8
S3150802D6D07B685B68B3F5A02F12D13F4B1B683E4AA5
S3150802D6E043F4802313603C4B1B683B4A23F48013A4
S3150802D6F01360394B1B68384A43F48033136029E0B8
S3150802D7007B685B68B3F5A81F12D1334B1B68324A94
S3150802D71043F480231360304B1B682F4A43F480136B
S3150802D72013602D4B1B682C4A43F48033136011E0B7
S3150802D730294B1B68284A23F480331360264B1B683F
S3150802D740254A23F480231360234B1B68224A23F4B9
S3150802D750801313607B685B68002B13D0FDF716FAFB
S3150802D760786108E0FDF712FA02467B69D31A642B40
S3150802D77001D903232EE3184B1B6803F40033002B4D
S3150802D780F0D012E0FDF702FA786108E0FDF7FEF93B
S3150802D79002467B69D31A642B01D903231AE30E4B7B
S3150802D7A01B6803F40033002BF0D17B681B6803F077
S3150802D7B00203002B00F09A80FB69002B05D0FB6957
S3150802D7C0182B49D1BB69012B46D17B68DB68002B34
S3150802D7D004D10123FEE200BF000C0244FB69002BC0
S3150802D7E01CD19A4B1B6803F018027B681B699A4284
S3150802D7F014D0964B1B6823F018027B681B69934961
S3150802D80013430B6000F0D0FD914B1B681846FBF7DB
S3150802D81021FE0346002B01D00123DBE2FDF7B6F910
S3150802D820786108E0FDF7B2F902467B69D31A022B42
S3150802D83001D90323CEE2854B1B6803F00203002BB2
S3150802D840F0D0824B1B6923F4FE027B685B691B04DA
S3150802D8507E4913430B6149E07B68DB68002B2CD0B9
S3150802D8607A4B1B6823F018027B681B6977491343B6
S3150802D8700B60764B1B68754A43F001031360FDF78C
S3150802D88085F9786108E0FDF781F902467B69D31AC2
S3150802D890022B01D903239DE26C4B1B6803F002039A
S3150802D8A0002BF0D0694B1B6923F4FE027B685B6987
S3150802D8B01B04664913430B6118E0644B1B68634AF1
S3150802D8C023F001031360FDF761F9786108E0FDF7BB
S3150802D8D05DF902467B69D31A022B01D9032379E241
S3150802D8E05A4B1B6803F00203002BF0D17B681B68B6
S3150802D8F003F00803002B3CD07B689B69002B1CD0E5
S3150802D900524BD3F8F030514A43F08063C2F8F030F4
S3150802D910FDF73CF9786108E0FDF738F902467B69BC
S3150802D920D31A022B01D9032354E2484BD3F8F03019
S3150802D93003F00063002BEFD01BE0444BD3F8F03022
S3150802D940424A23F08063C2F8F030FDF71FF9786186
S3150802D95008E0FDF71BF902467B69D31A022B01D9A7
S3150802D960032337E2394BD3F8F03003F00063002B78
S3150802D970EFD17B681B6803F00403002B00F0D2800A
S3150802D980344B5B6A03F00103002B18D1314B5B6AF7
S3150802D990304A43F001035362FDF7F8F8786108E06C
S3150802D9A0FDF7F4F802467B69D31A022B01D9032341
S3150802D9B010E2284B5B6A03F00103002BF0D07B6868
S3150802D9C09B68012B08D1214BD3F8F0301F4A43F04C
S3150802D9D00103C2F8F03074E07B689B68002B18D10B
S3150802D9E01A4BD3F8F030194A23F00103C2F8F03083
S3150802D9F0164BD3F8F030154A23F08003C2F8F030FC
S3150802DA00124BD3F8F030114A23F00403C2F8F0306F
S3150802DA1057E07B689B68052B1ED10C4BD3F8F03078
S3150802DA200A4A43F00403C2F8F030084BD3F8F03040
S3150802DA30064A23F08003C2F8F030044BD3F8F030DC
S3150802DA40024A43F00103C2F8F0303AE0000C0244FD
S3150802DA5078070020000802447B689B68852B18D14A
S3150802DA60A24BD3F8F030A14A43F00403C2F8F030CF
S3150802DA709E4BD3F8F0309D4A43F08003C2F8F0304B
S3150802DA809A4BD3F8F030994A43F00103C2F8F030C2
S3150802DA9017E0964BD3F8F030944A23F00103C2F804
S3150802DAA0F030924BD3F8F030904A23F00403C2F8D0
S3150802DAB0F0308E4BD3F8F0308C4A23F08003C2F84C
S3150802DAC0F0307B689B68002B16D0FDF75FF878610B
S3150802DAD00AE0FDF75BF802467B69D31A41F28832FF
S3150802DAE0934201D9032375E1804BD3F8F03003F052
S3150802DAF00203002BEDD015E0FDF748F878610AE03D
S3150802DB00FDF744F802467B69D31A41F288329342FA
S3150802DB1001D903235EE1754BD3F8F03003F0020313
S3150802DB20002BEDD17B681B6803F02003002B36D04F
S3150802DB307B685B6A002B19D06C4B1B686B4A43F4F3
S3150802DB4080531360FDF722F8786108E0FDF71EF8A6
S3150802DB5002467B69D31A022B01D903233AE1634BA6
S3150802DB601B6803F40053002BF0D018E05F4B1B68C8
S3150802DB705E4A23F480531360FDF708F8786108E0DB
S3150802DB80FDF704F802467B69D31A022B01D903234F
S3150802DB9020E1564B1B6803F40053002BF0D17B6837
S3150802DBA09B6A002B00F01581FB69182B00F0AF80E9
S3150802DBB07B689B6A022B40F086804C4B1B684B4A5B
S3150802DBC023F080731360FCF7E1FF786108E0FCF745
S3150802DBD0DDFF02467B69D31A022B01D90323F9E03A
S3150802DBE0424B1B6803F00073002BF0D13F4B9B6A34
S3150802DBF023F47C5323F003037A68D16A7A68126B9A
S3150802DC0012020A43394913438B627B685B6B013BF9
S3150802DC10C3F308027B689B6B013B5B029BB21A4308
S3150802DC207B68DB6B013B1B0403F4FE031A437B6828
S3150802DC301B6C013B1B0603F0FE432C4913434B6343
S3150802DC402A4B9B6A294A23F0100393627B68DB6C92
S3150802DC50264ADB009363254B9B6A244A43F010034A
S3150802DC609362224B9B6A23F00C027B685B6C1F490A
S3150802DC7013438B621D4B9B6A23F020027B689B6CC5
S3150802DC801A4913438B62194B9B6A184A43F4803329
S3150802DC909362164B1B68154A43F080731360FCF7B0
S3150802DCA075FF786108E0FCF771FF02467B69D31AB3
S3150802DCB0022B01D903238DE00C4B1B6803F000737A
S3150802DCC0002BF0D085E0094B1B68084A23F08073C5
S3150802DCD01360FCF75BFF78610AE0FCF757FF024620
S3150802DCE07B69D31A022B03D9032373E0000C02447F
S3150802DCF03A4B1B6803F00073002BEED1374B9B6A35
S3150802DD00364A23F4E02323F00303936261E0334B9C
S3150802DD109B6A3B61314B5B6BFB607B689B6A012BA1
S3150802DD2031D03B6903F003027B68DB6A9A422AD147
S3150802DD303B691B0A03F03F027B681B6B9A4222D19E
S3150802DD40FB68C3F308027B685B6B013B9A421AD1F4
S3150802DD50FB685B0A03F07F027B689B6B013B9A4276
S3150802DD6011D1FB681B0C03F07F027B68DB6B013B5E
S3150802DD709A4208D1FB681B0E03F07F027B681B6C74
S3150802DD80013B9A4201D0012324E0144B9B6BDB082A
S3150802DD90C3F30C027B68DB6C9A421AD00F4B9B6A60
S3150802DDA00E4A23F010039362FCF7F0FE786100BF77
S3150802DDB0FCF7ECFE02467B699342F9D07B68DB6C82
S3150802DDC0064ADB009363054B9B6A044A43F0100339
S3150802DDD09362002318462037BD4680BD000C0244D4
S3150802DDE080B584B000AF786039607B68002B01D1BA
S3150802DDF001239EE1834B1B6803F00F033A689A429C
S3150802DE0010D9804B1B6823F00F027E493B681343E7
S3150802DE100B607C4B1B6803F00F033A689A4201D0E9
S3150802DE20012386E17B681B6803F01003002B12D0DE
S3150802DE307B685A69744B1B6A1B0A03F070039A4281
S3150802DE4009D9714B1B6A23F4E0427B685B691B02A2
S3150802DE506D4913430B627B681B6803F00803002BAA
S3150802DE6012D07B681A69684B1B6A1B0903F0700398
S3150802DE709A4209D9644B1B6A23F4E0627B681B69E0
S3150802DE801B01614913430B627B681B6803F0040399
S3150802DE90002B10D07B68DA685B4B1B6A03F07003B1
S3150802DEA09A4208D9584B1B6A23F070027B68DB68D2
S3150802DEB0554913430B627B681B6803F00203002B68
S3150802DEC010D07B689A68504B1B6A03F00F039A427C
S3150802DED008D94D4B1B6A23F00F027B689B684A4997
S3150802DEE013430B627B681B6803F00103002B00F0E7
S3150802DEF093807B685B68032B07D1434B1B6803F04F
S3150802DF000073002B21D1012313E17B685B68022B86
S3150802DF1007D13D4B1B6803F40033002B15D10123AF
S3150802DF2007E17B685B68012B07D1374B1B6803F453
S3150802DF300073002B09D10123FBE0334B1B6803F066
S3150802DF400203002B01D10123F3E02F4BDB6923F0F7
S3150802DF5003027B685B682C491343CB61FCF716FE08
S3150802DF60F8607B685B68032B12D10AE0FCF70EFEA9
S3150802DF700246FB68D31A41F28832934201D9032337
S3150802DF80D7E0214BDB6903F01803182BEED143E0E7
S3150802DF907B685B68022B12D10AE0FCF7F7FD0246A2
S3150802DFA0FB68D31A41F28832934201D90323C0E0AF
S3150802DFB0154BDB6903F01803102BEED12CE07B68B6
S3150802DFC05B68012B22D10AE0FCF7E0FD0246FB68FA
S3150802DFD0D31A41F28832934201D90323A9E00A4BA4
S3150802DFE0DB6903F01803082BEED115E0FCF7CEFD2A
S3150802DFF00246FB68D31A41F28832934206D90323B2
S3150802E00097E000BF00200240000C02444B4BDB693C
S3150802E01003F01803002BE9D17B681B6803F002039F
S3150802E020002B10D07B689A68444B1B6A03F00F03D7
S3150802E0309A4208D2414B1B6A23F00F027B689B68FF
S3150802E0403E4913430B623E4B1B6803F00F033A68C3
S3150802E0509A4210D23A4B1B6823F00F0238493B68A2
S3150802E06013430B60364B1B6803F00F033A689A4258
S3150802E07001D001235DE07B681B6803F00403002BD3
S3150802E08010D07B68DA682D4B1B6A03F070039A423C
S3150802E09008D22A4B1B6A23F070027B68DB68274981
S3150802E0A013430B627B681B6803F00803002B12D02C
S3150802E0B07B681A69214B1B6A1B0903F070039A4293
S3150802E0C009D21E4B1B6A23F4E0627B681B691B019B
S3150802E0D01A4913430B627B681B6803F01003002B73
S3150802E0E012D07B685A69154B1B6A1B0A03F0700328
S3150802E0F09A4209D2114B1B6A23F4E0427B685B6998
S3150802E1001B020E4913430B6200F022F802460B4B20
S3150802E1101B6A03F00F030B49CB5C22FA03F30A4A84
S3150802E12013600A4B1B681846FBF794F90346FB7201
S3150802E130FB7A18461037BD4680BD00BF000C024464
S3150802E140002002402C630408740700207807002088
S3150802E15080B489B000AF8C4BDB6903F01803082B37
S3150802E16002D18A4BFB6107E1874BDB6903F018038F
S3150802E170002B12D1844B1B6803F02003002B09D015
S3150802E180814B1B68DB0803F00303814A22FA03F377
S3150802E190FB61F1E07E4BFB61EEE07B4BDB6903F052
S3150802E1A01803102B02D17B4BFB61E5E0764BDB694A
S3150802E1B003F01803182B40F0DD80734B9B6A03F0BB
S3150802E1C003037B61704B9B6A1B0A03F03F033B61A7
S3150802E1D06D4B9B6A1B0903F00103FB606A4B9B6B41
S3150802E1E0DB08C3F30C03FA6802FB03F307EE903A63
S3150802E1F0F8EE677AC7ED027A3B69002B00F0B78022
S3150802E2007B69012B03D07B69032B56D077E05E4BE3
S3150802E2101B6803F02003002B2DD05B4B1B68DB0821
S3150802E22003F003035A4A22FA03F37B607B6807EE7C
S3150802E230903AF8EE676A3B6907EE903AF8EE677A23
S3150802E24086EEA77A504B5B6BC3F3080307EE903A48
S3150802E250F8EE676A97ED026ADFED4F5AC6EE257A3F
S3150802E26076EEA77AF7EE006A77EEA67A67EE277A4F
S3150802E270C7ED067A65E03B6907EE903AF8EE677AEB
S3150802E280DFED466A86EEA77A3F4B5B6BC3F308035C
S3150802E29007EE903AF8EE676A97ED026ADFED3E5AA4
S3150802E2A0C6EE257A76EEA77AF7EE006A77EEA67AB2
S3150802E2B067EE277AC7ED067A43E03B6907EE903A9E
S3150802E2C0F8EE677ADFED366A86EEA77A2E4B5B6B37
S3150802E2D0C3F3080307EE903AF8EE676A97ED026A07
S3150802E2E0DFED2D5AC6EE257A76EEA77AF7EE006AA4
S3150802E2F077EEA67A67EE277AC7ED067A21E03B69BA
S3150802E30007EE903AF8EE677ADFED266A86EEA77A86
S3150802E3101D4B5B6BC3F3080307EE903AF8EE676A88
S3150802E32097ED026ADFED1C5AC6EE257A76EEA77AD3
S3150802E330F7EE006A77EEA67A67EE277AC7ED067ACF
S3150802E34000BF114B5B6B5B0A03F07F0301333B6033
S3150802E3503B6807EE903AB8EE677AD7ED066AC6EEDC
S3150802E360877AFCEEE77A17EE903AFB6104E000231F
S3150802E370FB6101E0064BFB61FB6918462437BD4683
S3150802E3805DF8047B704700BF000C024400093D009B
S3150802E3900090D003001BB700000000460024744C0E
S3150802E3A0001B374B0024744A80B500AFFFF7D0FE36
S3150802E3B00246084B1B6A03F00F030749CB5C03F0BE
S3150802E3C01F0322FA03F3054A1360044B1B68184617
S3150802E3D080BD00BF000C02442C63040874070020A9
S3150802E3E080B500AFFFF7E0FF0246064B1B6A1B0922
S3150802E3F003F007030449CB5C03F01F0322FA03F375
S3150802E400184680BD000C02443C63040880B500AF80
S3150802E410FFF7CAFF0246064B1B6A1B0A03F00703ED
S3150802E4200449CB5C03F01F0322FA03F3184680BDA6
S3150802E430000C02443C63040880B500AFFFF7B4FF42
S3150802E4400246064B1B6A1B0B03F007030449CB5C07
S3150802E45003F01F0322FA03F3184680BD000C024498
S3150802E4603C63040880B485B000AF786039607B6885
S3150802E4701F221A60154BDB6903F003027B685A6098
S3150802E480124B1B6AFB60FB6803F00F027B689A60FB
S3150802E490FB6803F070027B68DA60FB681B0903F00D
S3150802E4A070027B681A61FB681B0A03F070027B68BC
S3150802E4B05A61074B1B6803F00F023B681A6000BFDC
S3150802E4C01437BD465DF8047B704700BF000C024452
S3150802E4D0002002402DE9B04FD8B000AFC7F84C0172
S3150802E4E0002387F85B31002387F85A31D7F84C3175
S3150802E4F0D3E9002302F08074002554EA05030BD001
S3150802E500CD4BD3F8E83023F04041D7F84C319B6D18
S3150802E510C94A0B43C2F8E830D7F84C31D3E900238D
S3150802E52002F001084FF0000958EA090342D0D7F869
S3150802E5304C31DB6D052B23D801A252F823F000BF1C
S3150802E54089E5020859E502086DE5020889E5020827
S3150802E55089E5020889E50208D7F84C3108331846D6
S3150802E56004F0DAFE034687F85B310EE0D7F84C3141
S3150802E5703033184604F068FF034687F85B3104E037
S3150802E580012387F85B3100E000BF97F85B31002B67
S3150802E5900CD1A94BD3F8D83023F00701D7F84C3160
S3150802E5A0DB6DA54A0B43C2F8D83003E097F85B3116
S3150802E5B087F85A31D7F84C31D3E9002302F0020A18
S3150802E5C04FF0000B5AEA0B0300F08880D7F84C315B
S3150802E5D01B6E282B68D801A252F823F0B1E602086E
S3150802E5E0A9E60208A9E60208A9E60208A9E60208B7
S3150802E5F0A9E60208A9E60208A9E6020881E60208CF
S3150802E600A9E60208A9E60208A9E60208A9E6020896
S3150802E610A9E60208A9E60208A9E6020895E602089A
S3150802E620A9E60208A9E60208A9E60208A9E6020876
S3150802E630A9E60208A9E60208A9E60208B1E602085E
S3150802E640A9E60208A9E60208A9E60208A9E6020856
S3150802E650A9E60208A9E60208A9E60208B1E602083E
S3150802E660A9E60208A9E60208A9E60208A9E6020836
S3150802E670A9E60208A9E60208A9E60208B1E602081E
S3150802E680D7F84C310833184604F046FE034687F895
S3150802E6905B310EE0D7F84C313033184604F0D4FE1D
S3150802E6A0034687F85B3104E0012387F85B3100E013
S3150802E6B000BF97F85B31002B0CD15F4BD3F8D830EB
S3150802E6C023F03801D7F84C311B6E5B4A0B43C2F86C
S3150802E6D0D83003E097F85B3187F85A31D7F84C31CE
S3150802E6E0D3E9002302F00403C7F840310023C7F830
S3150802E6F04431D7E950120B4613434ED0D7F84C3162
S3150802E7005B6EB3F5A07F2CD0B3F5A07F25D8B3F501
S3150802E710807F28D0B3F5807F1FD8C02B25D0C02B89
S3150802E7201BD8802B0FD0802B17D8002B1FD0402B3D
S3150802E73013D1D7F84C310833184604F0EDFD0346D9
S3150802E74087F85B3114E0D7F84C313033184604F0B9
S3150802E7507BFE034687F85B310AE0012387F85B31C3
S3150802E76006E000BF04E000BF02E000BF00E000BF11
S3150802E77097F85B31002B0CD12F4BD3F8D83023F402
S3150802E780E071D7F84C315B6E2B4A0B43C2F8D8308E
S3150802E79003E097F85B3187F85A31D7F84C31D3E959
S3150802E7A0002302F00803C7F838310023C7F83C31C2
S3150802E7B0D7E94E120B46134356D0D7F84C319B6E07
S3150802E7C0B3F5206F31D0B3F5206F2AD8B3F5006FB1
S3150802E7D02DD0B3F5006F24D8B3F5C06F29D0B3F5A1
S3150802E7E0C06F1ED8B3F5806F11D0B3F5806F18D8F5
S3150802E7F0002B23D0B3F5007F13D1D7F84C31083359
S3150802E800184604F089FD034687F85B3117E0D7F806
S3150802E8104C313033184604F017FE034687F85B314D
S3150802E8200DE0012387F85B3109E000BF07E000BF6E
S3150802E83005E000BF03E000BF000C024400BF97F8E2
S3150802E8405B31002B0CD1BB4BD3F8D83023F4606173
S3150802E850D7F84C319B6EB74A0B43C2F8D83003E05F
S3150802E86097F85B3187F85A31D7F84C31D3E9002348
S3150802E87002F01003C7F830310023C7F83431D7E95C
S3150802E8804C120B46134353D0D7F84C31DB6EB3F513
S3150802E890A04F31D0B3F5A04F2AD8B3F5804F2DD06B
S3150802E8A0B3F5804F24D8B3F5405F29D0B3F5405F5E
S3150802E8B01ED8B3F5005F11D0B3F5005F18D8002B48
S3150802E8C020D0B3F5805F13D1D7F84C3108331846F8
S3150802E8D004F022FD034687F85B3114E0D7F84C3181
S3150802E8E03033184604F0B0FD034687F85B310AE078
S3150802E8F0012387F85B3106E000BF04E000BF02E0AF
S3150802E90000BF00E000BF97F85B31002B0CD1894BA2
S3150802E910D3F8D83023F4E041D7F84C31DB6E854A78
S3150802E9200B43C2F8D83003E097F85B3187F85A31BF
S3150802E930D7F84C31D3E9002302F02003C7F828316F
S3150802E9400023C7F82C31D7E94A120B46134353D092
S3150802E950D7F84C311B6FB3F5203F31D0B3F5203FC2
S3150802E9602AD8B3F5003F2DD0B3F5003F24D8B3F526
S3150802E970C03F29D0B3F5C03F1ED8B3F5803F11D0AA
S3150802E980B3F5803F18D8002B20D0B3F5004F13D12A
S3150802E990D7F84C310833184604F0BEFC034687F80C
S3150802E9A05B3114E0D7F84C313033184604F04CFD8D
S3150802E9B0034687F85B310AE0012387F85B3106E0F4
S3150802E9C000BF04E000BF02E000BF00E000BF97F806
S3150802E9D05B31002B0CD1574BD3F8D83023F4603176
S3150802E9E0D7F84C311B6F534A0B43C2F8D83003E0B1
S3150802E9F097F85B3187F85A31D7F84C31D3E90023B7
S3150802EA0002F04003C7F820310023C7F82431D7E9BA
S3150802EA1048120B46134353D0D7F84C315B6FB3F504
S3150802EA20A01F31D0B3F5A01F2AD8B3F5801F2DD069
S3150802EA30B3F5801F24D8B3F5402F29D0B3F5402F5C
S3150802EA401ED8B3F5002F11D0B3F5002F18D8002B16
S3150802EA5020D0B3F5802F13D1D7F84C310833184696
S3150802EA6004F05AFC034687F85B3114E0D7F84C31B8
S3150802EA703033184604F0E8FC034687F85B310AE0AF
S3150802EA80012387F85B3106E000BF04E000BF02E01D
S3150802EA9000BF00E000BF97F85B31002B0CD1254B75
S3150802EAA0D3F8D83023F4E011D7F84C315B6F214AFA
S3150802EAB00B43C2F8D83003E097F85B3187F85A312E
S3150802EAC0D7F84C31D3E9002302F08003C7F818318E
S3150802EAD00023C7F81C31D7E946120B46134355D013
S3150802EAE0D7F84C319B6FB3F5200F33D0B3F5200F0F
S3150802EAF02CD8B3F5000F2FD0B3F5000F26D8B3F5EF
S3150802EB00C00F2BD0B3F5C00F20D8B3F5800F13D0A2
S3150802EB10B3F5800F1AD8002B22D0B3F5001F15D1F2
S3150802EB20D7F84C310833184604F0F6FB034687F843
S3150802EB305B3116E0000C0244D7F84C3130331846E4
S3150802EB4004F082FC034687F85B310AE0012387F862
S3150802EB505B3106E000BF04E000BF02E000BF00E050
S3150802EB6000BF97F85B31002B0CD1BB4BD3F8D830DA
S3150802EB7023F46001D7F84C319B6FB74A0B43C2F8AE
S3150802EB80D83003E097F85B3187F85A31D7F84C3119
S3150802EB90D3E9002302F48073C7F810310023C7F8BB
S3150802EBA01431D7E944120B46134353D0D7F84C31E4
S3150802EBB0DB6FB3F1A06F31D0B3F1A06F2AD8B3F1EE
S3150802EBC0806F2DD0B3F1806F24D8B3F1407F29D05E
S3150802EBD0B3F1407F1ED8B3F1007F11D0B3F1007FA5
S3150802EBE018D8002B20D0B3F1807F13D1D7F84C3137
S3150802EBF00833184604F090FB034687F85B3114E0A5
S3150802EC00D7F84C313033184604F01EFC034687F811
S3150802EC105B310AE0012387F85B3106E000BF04E0B6
S3150802EC2000BF02E000BF00E000BF97F85B31002B8F
S3150802EC300CD1894BD3F8D83023F0E061D7F84C31A0
S3150802EC40DB6F854A0B43C2F8D83003E097F85B318D
S3150802EC5087F85A31D7F84C31D3E9002302F4007306
S3150802EC60C7F808310023C7F80C31D7E942120B4618
S3150802EC70134355D0D7F84C31D3F88030B3F1205F1F
S3150802EC8031D0B3F1205F2AD8B3F1005F2DD0B3F1AA
S3150802EC90005F24D8B3F1C05F29D0B3F1C05F1ED894
S3150802ECA0B3F1805F11D0B3F1805F18D8002B20D062
S3150802ECB0B3F1006F13D1D7F84C310833184604F074
S3150802ECC02BFB034687F85B3114E0D7F84C31303317
S3150802ECD0184604F0B9FB034687F85B310AE00123BC
S3150802ECE087F85B3106E000BF04E000BF02E000BF20
S3150802ECF000E000BF97F85B31002B0DD1564BD3F8D5
S3150802ED00D83023F06051D7F84C31D3F88030524AC4
S3150802ED100B43C2F8D83003E097F85B3187F85A31CB
S3150802ED20D7F84C31D3E9002302F48063C7F80031DF
S3150802ED300023C7F80431D7E940120B46134344D0DF
S3150802ED40D7F84C31D3F88430052B23D801A252F8D0
S3150802ED5023F000BF9DED02086DED020881ED020861
S3150802ED609DED02089DED02089DED0208D7F84C318B
S3150802ED700833184604F0D0FA034687F85B310EE0EA
S3150802ED80D7F84C313033184604F05EFB034687F851
S3150802ED905B3104E0012387F85B3100E000BF97F896
S3150802EDA05B31002B0DD12C4BD3F8DC3023F0070155
S3150802EDB0D7F84C31D3F88430274A0B43C2F8DC30F3
S3150802EDC003E097F85B3187F85A31D7F84C31D3E923
S3150802EDD0002302F40063C7F8F8300023C7F8FC30B2
S3150802EDE0D7E93E120B4613434FD0D7F84C31D3F826
S3150802EDF08830502B29D0502B23D8402B27D0402B94
S3150802EE001FD8302B25D0302B1BD8202B0FD0202BE8
S3150802EE1017D8002B22D0102B13D1D7F84C31083330
S3150802EE20184604F079FA034687F85B3117E0D7F8F3
S3150802EE304C313033184604F007FB034687F85B313A
S3150802EE400DE0012387F85B3109E000BF07E000BF48
S3150802EE5005E000BF03E000BF000C024400BF97F8BC
S3150802EE605B31002B0DD1AF4BD3F8DC3023F07001A8
S3150802EE70D7F84C31D3F88830AA4A0B43C2F8DC30AB
S3150802EE8003E097F85B3187F85A31D7F84C31D3E962
S3150802EE90002302F48053C7F8F0300023C7F8F43091
S3150802EEA0D7E93C120B46134355D0D7F84C31D3F861
S3150802EEB08C30B3F1A06F31D0B3F1A06F2AD8B3F179
S3150802EEC0806F2DD0B3F1806F24D8B3F1407F29D05B
S3150802EED0B3F1407F1ED8B3F1007F11D0B3F1007FA2
S3150802EEE018D8002B20D0B3F1807F13D1D7F84C3134
S3150802EEF00833184604F010FA034687F85B3114E023
S3150802EF00D7F84C313033184604F09EFA034687F890
S3150802EF105B310AE0012387F85B3106E000BF04E0B3
S3150802EF2000BF02E000BF00E000BF97F85B31002B8C
S3150802EF300DD17C4BD3F8E03023F0E061D7F84C31A1
S3150802EF40D3F88C30774A0B43C2F8E03003E097F8DF
S3150802EF505B3187F85A31D7F84C31D3E9002302F4EA
S3150802EF600053C7F8E8300023C7F8EC30D7E93A125D
S3150802EF700B4613433DD0D7F84C31D3F89030B3F54E
S3150802EF80403F1BD0B3F5403F14D8B3F5003F17D026
S3150802EF90B3F5003F0ED8002B14D0B3F5803F09D144
S3150802EFA0D7F84C313033184604F04EFA034687F840
S3150802EFB05B3108E0012387F85B3104E000BF02E019
S3150802EFC000BF00E000BF97F85B31002B0DD1554B0F
S3150802EFD0D3F8E43023F44031D7F84C31D3F89030E3
S3150802EFE0504A0B43C2F8E43003E097F85B3187F8DE
S3150802EFF05A31D7F84C31D3E9002302F48043C7F8D3
S3150802F000E0300023C7F8E430D7E938120B46134339
S3150802F0103DD0D7F84C31D3F89430B3F5402F1BD0F6
S3150802F020B3F5402F14D8B3F5002F17D0B3F5002F38
S3150802F0300ED8002B14D0B3F5802F09D1D7F84C314E
S3150802F0403033184604F000FA034687F85B3108E0C5
S3150802F050012387F85B3104E000BF02E000BF00E04D
S3150802F06000BF97F85B31002B0DD12E4BD3F8E43055
S3150802F07023F44021D7F84C31D3F89430294A0B436C
S3150802F080C2F8E43003E097F85B3187F85A31D7F8CB
S3150802F0904C31D3E9002302F40043C7F8D8300023E1
S3150802F0A0C7F8DC30D7E936120B46134340D0D7F8F7
S3150802F0B04C31D3F89830B3F5401F1BD0B3F5401F37
S3150802F0C014D8B3F5001F17D0B3F5001F0ED8002BBE
S3150802F0D014D0B3F5801F09D1D7F84C31303318460E
S3150802F0E004F0B2F9034687F85B3108E0012387F892
S3150802F0F05B3104E000BF02E000BF00E000BF97F802
S3150802F1005B31002B10D1074BD3F8E43023F44011BE
S3150802F110D7F84C31D3F89830024A0B43C2F8E43098
S3150802F12006E000BF000C024497F85B3187F85A31B3
S3150802F130D7F84C31D3E900230021C7F8D01003F4DD
S3150802F1408063C7F8D430D7E934120B4613433DD04F
S3150802F150D7F84C31D3F89C30B3F5400F1BD0B3F532
S3150802F160400F14D8B3F5000F17D0B3F5000F0ED819
S3150802F170002B14D0B3F5800F09D1D7F84C313033B0
S3150802F180184604F061F9034687F85B3108E0012363
S3150802F19087F85B3104E000BF02E000BF00E000BF71
S3150802F1A097F85B31002B0DD1BE4BD3F8E43023F42C
S3150802F1B04001D7F84C31D3F89C30BA4A0B43C2F80F
S3150802F1C0E43003E097F85B3187F85A31D7F84C31C7
S3150802F1D0D3E9002302F48033C7F8C8300023C7F8FE
S3150802F1E0CC30D7E932120B46134335D0D7F84C3117
S3150802F1F0D3F8A030B3F1007F15D0B3F1007F0ED853
S3150802F200002B12D0B3F1807F09D1D7F84C313033B5
S3150802F210184604F019F9034687F85B3106E001231C
S3150802F22087F85B3102E000BF00E000BF97F85B3168
S3150802F230002B0DD19B4BD3F8E43023F04071D7F85D
S3150802F2404C31D3F8A030974A0B43C2F8E43003E0B6
S3150802F25097F85B3187F85A31D7F84C31D3E900234E
S3150802F2600021C7F8C01003F40063C7F8C430D7E911
S3150802F27030120B4613430ED08A4BDB69894A23F4B4
S3150802F2800043D361874BD969D7F84C31D3F8043197
S3150802F290844A0B43D361D7F84C31D3E9002302F4ED
S3150802F2A00033C7F8B8300023C7F8BC30D7E92E12A6
S3150802F2B00B46134355D0D7F84C31D3F8A430B3F5DF
S3150802F2C0A06F31D0B3F5A06F2AD8B3F5806F2DD0D1
S3150802F2D0B3F5806F24D8B3F5407F29D0B3F5407FC4
S3150802F2E01ED8B3F5007F11D0B3F5007F18D8002BCE
S3150802F2F020D0B3F5807F13D1D7F84C31083318469E
S3150802F30004F00AF8034687F85B3114E0D7F84C3163
S3150802F3103033184604F098F8034687F85B310AE05A
S3150802F320012387F85B3106E000BF04E000BF02E074
S3150802F33000BF00E000BF97F85B31002B0DD1594B97
S3150802F340D3F8DC3023F4E061D7F84C31D3F8A43093
S3150802F350544A0B43C2F8DC3003E097F85B3187F86E
S3150802F3605A31D7F84C31D3E9002302F48023C7F87F
S3150802F370B0300023C7F8B430D7E92C120B46134332
S3150802F38055D0D7F84C31D3F8A830B3F5A04F31D0C1
S3150802F390B3F5A04F2AD8B3F5804F2DD0B3F5804FD9
S3150802F3A024D8B3F5405F29D0B3F5405F1ED8B3F52C
S3150802F3B0005F11D0B3F5005F18D8002B20D0B3F543
S3150802F3C0805F13D1D7F84C310833184603F0A4FFEF
S3150802F3D0034687F85B3114E0D7F84C3130331846C8
S3150802F3E004F032F8034687F85B310AE0012387F80E
S3150802F3F05B3106E000BF04E000BF02E000BF00E0A8
S3150802F40000BF97F85B31002B0DD1264BD3F8DC30C1
S3150802F41023F4E041D7F84C31D3F8A830214A0B43FC
S3150802F420C2F8DC3003E097F85B3187F85A31D7F82F
S3150802F4304C31D3E900230021C7F8A81003F02003B2
S3150802F440C7F8AC30D7E92A120B46134357D0D7F878
S3150802F4504C31D3F8AC30B3F5A02F33D0B3F5A02F87
S3150802F4602CD8B3F5802F2FD0B3F5802F26D8B3F535
S3150802F470403F2BD0B3F5403F20D8B3F5003F13D019
S3150802F480B3F5003F1AD8002B22D0B3F5803F15D129
S3150802F490D7F84C310833184603F03EFF034687F87F
S3150802F4A05B3116E0000C0244D7F84C31303318466B
S3150802F4B003F0CAFF034687F85B310AE0012387F89F
S3150802F4C05B3106E000BF04E000BF02E000BF00E0D7
S3150802F4D000BF97F85B31002B0DD1BB4BD3F8DC305C
S3150802F4E023F4E021D7F84C31D3F8AC30B64A0B43B3
S3150802F4F0C2F8DC3003E097F85B3187F85A31D7F85F
S3150802F5004C31D3E900230021C7F8A01003F04003C9
S3150802F510C7F8A430D7E928120B46134355D0D7F8B3
S3150802F5204C31D3F8B030B3F5A00F31D0B3F5A00FF4
S3150802F5302AD8B3F5800F2DD0B3F5800F24D8B3F5AA
S3150802F540401F29D0B3F5401F1ED8B3F5001F11D0AE
S3150802F550B3F5001F18D8002B20D0B3F5801F13D19E
S3150802F560D7F84C310833184603F0D6FE034687F817
S3150802F5705B3114E0D7F84C313033184603F064FF98
S3150802F580034687F85B310AE0012387F85B3106E018
S3150802F59000BF04E000BF02E000BF00E000BF97F82A
S3150802F5A05B31002B0DD1884BD3F8DC3023F4E00114
S3150802F5B0D7F84C31D3F8B030834A0B43C2F8DC3063
S3150802F5C003E097F85B3187F85A31D7F84C31D3E91B
S3150802F5D000230021C7F8981003F08003C7F89C306F
S3150802F5E0D7E926120B46134355D0D7F84C31D3F830
S3150802F5F0B430B3F1A06F31D0B3F1A06F2AD8B3F10A
S3150802F600806F2DD0B3F1806F24D8B3F1407F29D013
S3150802F610B3F1407F1ED8B3F1007F11D0B3F1007F5A
S3150802F62018D8002B20D0B3F1807F13D1D7F84C31EC
S3150802F6300833184603F070FE034687F85B3114E078
S3150802F640D7F84C313033184603F0FEFE034687F8E6
S3150802F6505B310AE0012387F85B3106E000BF04E06C
S3150802F66000BF02E000BF00E000BF97F85B31002B45
S3150802F6700DD1554BD3F8DC3023F0E061D7F84C3185
S3150802F680D3F8B430504A0B43C2F8DC3003E097F89B
S3150802F6905B3187F85A31D7F84C31D3E90023002178
S3150802F6A0C7F8901003F48073C7F89430D7E9241288
S3150802F6B00B46134355D0D7F84C31D3F8B830B3F1CB
S3150802F6C0A04F31D0B3F1A04F2AD8B3F1804F2DD035
S3150802F6D0B3F1804F24D8B3F1405F29D0B3F1405F2C
S3150802F6E01ED8B3F1005F11D0B3F1005F18D8002B12
S3150802F6F020D0B3F1805F13D1D7F84C3108331846BE
S3150802F70003F00AFE034687F85B3114E0D7F84C315A
S3150802F7103033184603F098FE034687F85B310AE051
S3150802F720012387F85B3106E000BF04E000BF02E070
S3150802F73000BF00E000BF97F85B31002B0DD1224BCA
S3150802F740D3F8DC3023F0E041D7F84C31D3F8B8309F
S3150802F7501D4A0B43C2F8DC3003E097F85B3187F8A1
S3150802F7605A31D7F84C31D3E9002302F40023C7F8FB
S3150802F77088300023C7F88C30D7E922120B46134388
S3150802F78055D0D7F84C31D3F8C030B3F5802F35D0E1
S3150802F790B3F5802F2ED8B3F5403F31D0B3F5403FAD
S3150802F7A028D8B3F5003F1BD0B3F5003F22D8002B6B
S3150802F7B003D0B3F5803F09D01CE0034B9B6A024A8B
S3150802F7C043F4003393621CE0000C0244D7F84C3130
S3150802F7D00833184603F0A0FD034687F85B3110E0AC
S3150802F7E0D7F84C313033184603F02EFE034687F815
S3150802F7F05B3106E0012387F85B3102E000BF00E0D7
S3150802F80000BF97F85B31002B0DD1C34BD3F8E83014
S3150802F81023F4E021D7F84C31D3F8C030BE4A0B4363
S3150802F820C2F8E83003E097F85B3187F85A31D7F81F
S3150802F8304C31D3E9002302F48013C7F88030002341
S3150802F840C7F88430D7E920120B46134351D0D7F8AC
S3150802F8504C31D3F8C430B3F5001F33D0B3F5001FCB
S3150802F8602CD8B3F5C01F2DD0B3F5C01F26D8B3F5D3
S3150802F870801F19D0B3F5801F20D8002B03D0B3F50B
S3150802F880002F07D01AE0A44B9B6AA34A43F400331D
S3150802F890936218E0D7F84C310833184603F03CFD5A
S3150802F8A0034687F85B310EE0D7F84C3130331846F9
S3150802F8B003F0CAFD034687F85B3104E0012387F8A3
S3150802F8C05B3100E000BF97F85B31002B0DD1924BFC
S3150802F8D0D3F8E83023F46011D7F84C31D3F8C430A2
S3150802F8E08D4A0B43C2F8E83003E097F85B3187F894
S3150802F8F05A31D7F84C31D3E9002302F40013BB6717
S3150802F9000023FB67D7E91E120B46134332D0D7F8FA
S3150802F9104C31D3F8D430052B0FD8032B11D2012B37
S3150802F92011D9022B09D1D7F84C310833184603F0FE
S3150802F930F3FC034687F85B3106E0012387F85B315F
S3150802F94002E000BF00E000BF97F85B31002B0DD143
S3150802F950714BD3F8E83023F00701D7F84C31D3F8C6
S3150802F960D4306D4A0B43C2F8E83003E097F85B31AE
S3150802F97087F85A31D7F84C31D3E900230021396781
S3150802F98003F400737B67D7E91C120B46134324D092
S3150802F990D7F84C31D3F8D830002B05D0082B05D030
S3150802F9A0012387F85B3102E000BF00E000BF97F849
S3150802F9B05B31002B0DD1584BD3F8E83023F0080100
S3150802F9C0D7F84C31D3F8D830534A0B43C2F8E8304B
S3150802F9D003E097F85B3187F85A31D7F84C31D3E907
S3150802F9E0002302F00073BB660023FB66D7E91A12EE
S3150802F9F00B46134300F0B980484B5B6A474A43F00B
S3150802FA0001035362FBF7C2F8C7F854010BE0FBF790
S3150802FA10BDF80246D7F85431D31A022B03D9032369
S3150802FA2087F85B3105E03D4B5B6A03F00103002B67
S3150802FA30EDD097F85B31002B40F09380364BD3F824
S3150802FA40F03003F44073C7F85C31D7F85C31002B09
S3150802FA5023D0D7F84C31D3F8F820D7F85C31934243
S3150802FA601BD02D4BD3F8F03023F44073C7F85C3122
S3150802FA70294BD3F8F030284A43F48033C2F8F030E1
S3150802FA80254BD3F8F030244A23F48033C2F8F030F9
S3150802FA90214AD7F85C31C2F8F030D7F85C3103F066
S3150802FAA00103002B19D0FBF771F8C7F854010DE0D2
S3150802FAB0FBF76CF80246D7F85431D21A41F288336A
S3150802FAC09A4203D9032387F85B3106E0124BD3F82F
S3150802FAD0F03003F00203002BEAD097F85B31002BD3
S3150802FAE03AD1D7F84C31D3F8F83003F44073B3F56A
S3150802FAF0407F15D1084BDB6923F47C51D7F84C318A
S3150802FB00D3F8F8301B0923F07F4323F03003024A67
S3150802FB100B43D3610AE000BF000C0244000802440A
S3150802FB209F4BDB699E4A23F47C53D3619C4BD3F8E3
S3150802FB30F0309B4A23F44073C2F8F030984BD3F85E
S3150802FB40F010D7F84C31D3F8F830C3F30B03944AC4
S3150802FB500B43C2F8F03008E097F85B3187F85A3160
S3150802FB6003E097F85B3187F85A31D7F84C31D3E975
S3150802FB70002302F080633B6600237B66D7E91812EE
S3150802FB800B46134335D0D7F84C31D3F8C830302B4F
S3150802FB9014D0302B0ED8202B12D0202B0AD8002BAB
S3150802FBA010D0102B06D17E4B9B6A7D4A43F4003354
S3150802FBB0936208E0012387F85B3104E000BF02E0A4
S3150802FBC000BF00E000BF97F85B31002B0DD1744BE4
S3150802FBD0D3F8E83023F03001D7F84C31D3F8C830DF
S3150802FBE06F4A0B43C2F8E83003E097F85B3187F8AF
S3150802FBF05A31D7F84C31D3E9002302F48003BB65A6
S3150802FC000023FB65D7E916120B46134333D0D7F800
S3150802FC104C31D3F8CC30002B02D0402B07D010E061
S3150802FC205F4B9B6A5E4A43F4003393620DE0D7F852
S3150802FC304C310833184603F06FFB034687F85B31ED
S3150802FC4003E0012387F85B3100BF97F85B31002B8D
S3150802FC500DD1534BD3F8E43023F04001D7F84C3199
S3150802FC60D3F8CC304E4A0B43C2F8E43003E097F897
S3150802FC705B3187F85A31D7F84C31D3E9002302F4BD
S3150802FC8000033B6500237B65D7E914120B46134331
S3150802FC9033D0D7F84C31D3F8D030002B02D0802B92
S3150802FCA007D010E03E4B9B6A3D4A43F40033936209
S3150802FCB00DE0D7F84C310833184603F02DFB0346FE
S3150802FCC087F85B3103E0012387F85B3100BF97F8B9
S3150802FCD05B31002B0DD1324BD3F8E43023F080018F
S3150802FCE0D7F84C31D3F8D0302D4A0B43C2F8E4305A
S3150802FCF003E097F85B3187F85A31D7F84C31D3E9E4
S3150802FD00002302F00063BB640023FB64D7E91212E6
S3150802FD100B4613434AD0D7F84C31D3F8E030042BBC
S3150802FD2027D801A252F823F03DFD02084BFD02082E
S3150802FD305FFD02087BFD02087BFD0208184B9B6AE1
S3150802FD40174A43F40033936218E0D7F84C31083364
S3150802FD50184603F0E1FA034687F85B310EE0D7F856
S3150802FD604C313033184603F06FFB034687F85B3194
S3150802FD7004E0012387F85B3100E000BF97F85B31A6
S3150802FD80002B0FD1064BD3F8E03023F00701D7F842
S3150802FD904C31D3F8E030024A0B43C2F8E03005E0B2
S3150802FDA0000C024497F85B3187F85A31D7F84C3180
S3150802FDB0D3E9002302F080533B6400237B64D7E92E
S3150802FDC010120B46134300F08180D7F84C31D3F852
S3150802FDD0E430202B5FD801A252F823F061FE020814
S3150802FDE097FE020897FE020897FE020897FE020887
S3150802FDF097FE020897FE020897FE02086FFE02089F
S3150802FE0097FE020897FE020897FE020897FE020866
S3150802FE1097FE020897FE020897FE020883FE02086A
S3150802FE2097FE020897FE020897FE020897FE020846
S3150802FE3097FE020897FE020897FE02089FFE02082E
S3150802FE4097FE020897FE020897FE020897FE020826
S3150802FE5097FE020897FE020897FE02089FFE02080E
S3150802FE60AB4B9B6AAA4A43F40033936218E0D7F86D
S3150802FE704C310833184603F04FFA034687F85B31CC
S3150802FE800EE0D7F84C313033184603F0DDFA034654
S3150802FE9087F85B3104E0012387F85B3100E000BF95
S3150802FEA097F85B31002B0DD1994BD3F8E03023F04C
S3150802FEB03801D7F84C31D3F8E430954A0B43C2F8E7
S3150802FEC0E03003E097F85B3187F85A31D7F84C31BE
S3150802FED0D3E9002302F00053BB630023FB63D7E98F
S3150802FEE00E120B4613434ED0D7F84C31D3F8E830EE
S3150802FEF0B3F5807F2ED0B3F5807F27D8C02B2BD0C1
S3150802FF00C02B23D8802B17D0802B1FD8002B02D0CA
S3150802FF10402B07D01AE07E4B9B6A7D4A43F4003396
S3150802FF2093621AE0D7F84C310833184603F0F4F90D
S3150802FF30034687F85B3110E0D7F84C313033184660
S3150802FF4003F082FA034687F85B3106E0012387F855
S3150802FF505B3102E000BF00E000BF97F85B31002B7F
S3150802FF600DD16B4BD3F8E03023F4E071D7F84C315E
S3150802FF70D3F8E830664A0B43C2F8E03003E097F854
S3150802FF805B3187F85A31D7F84C31D3E9002302F0AE
S3150802FF9080433B6300237B63D7E90C120B4613436A
S3150802FFA055D0D7F84C31D3F8EC30B3F5206F31D0B1
S3150802FFB0B3F5206F2AD8B3F5006F2DD0B3F5006FCD
S3150802FFC024D8B3F5C06F29D0B3F5C06F1ED8B3F5E0
S3150802FFD0806F11D0B3F5806F18D8002B20D0B3F5F7
S3150802FFE0007F13D1D7F84C310833184603F094F939
S3150802FFF0034687F85B3114E0D7F84C31303318469C
S3150803000003F022FA034687F85B310AE0012387F8EF
S315080300105B3106E000BF04E000BF02E000BF00E07A
S3150803002000BF97F85B31002B0DD1394BD3F8E0307D
S3150803003023F46061D7F84C31D3F8EC30344A0B43D8
S31508030040C2F8E03003E097F85B3187F85A31D7F8FE
S315080300504C31D3E9002302F00043BB620023FB6261
S31508030060D7E90A120B46134358D0D7F84C31D3F8BD
S31508030070F030B3F5A04F31D0B3F5A04F2AD8B3F576
S31508030080804F2DD0B3F5804F24D8B3F5405F29D0E0
S31508030090B3F5405F1ED8B3F5005F11D0B3F5005F23
S315080300A018D8002B20D0B3F5805F13D1D7F84C317D
S315080300B00833184603F030F9034687F85B3114E032
S315080300C0D7F84C313033184603F0BEF9034687F8A0
S315080300D05B310AE0012387F85B3106E000BF04E0E1
S315080300E000BF02E000BF00E000BF97F85B31002BBA
S315080300F010D1074BD3F8E03023F4E042D7F84C315C
S31508030100D3F8F03002491343C1F8E03006E000BFE4
S31508030110000C024497F85B3187F85A31D7F84C310B
S31508030120D3E900230021396203F001037B62D7E98F
S3150803013008120B46134355D0D7F84C31D3F8F4308D
S31508030140B3F5203F31D0B3F5203F2AD8B3F5003FA6
S315080301502DD0B3F5003F24D8B3F5C03F29D0B3F566
S31508030160C03F1ED8B3F5803F11D0B3F5803F18D8EA
S31508030170002B20D0B3F5004F13D1D7F84C310833F1
S31508030180184603F0C9F8034687F85B3114E0D7F835
S315080301904C313033184603F057F9034687F85B3179
S315080301A00AE0012387F85B3106E000BF04E000BFDD
S315080301B002E000BF00E000BF97F85B31002B0DD1CA
S315080301C0884BD3F8E03023F46032D7F84C31D3F8B0
S315080301D0F43084491343C1F8E03003E097F85B3100
S315080301E087F85A31D7F84C31D3E900230021B9618E
S315080301F003F00203FB61D7E906120B4613433DD00E
S31508030200D7F84C31D3F8DC30032B1CD801A252F8AB
S3150803021023F000BF4F02030825020308330203082D
S315080302204F0203086F4B9B6A6E4A43F4003393628B
S315080302300EE0D7F84C310833184603F06DF8034639
S3150803024087F85B3104E0012387F85B3100E000BFE0
S3150803025097F85B31002B0DD1624BD3F8E43023F0CA
S315080302600302D7F84C31D3F8DC305E491343C1F89F
S31508030270E43003E097F85B3187F85A31D7F84C3105
S31508030280D3E900230021396103F004037B61D7E92D
S3150803029004120B4613433AD0D7F84C31D3F8BC3083
S315080302A0B3F5007F0ED0B3F5007F15D8002B17D012
S315080302B0B3F5807F10D14B4B9B6A4A4A43F400330C
S315080302C093620EE0D7F84C310833184603F024F846
S315080302D0034687F85B3104E0012387F85B3100E0C6
S315080302E000BF97F85B31002B0DD13E4BD3F8E830AE
S315080302F023F44072D7F84C31D3F8BC303949134349
S31508030300C1F8E83003E097F85B3187F85A31D7F834
S315080303104C31D3E900230021B96003F01003FB60D5
S31508030320D7E902120B46134338D0D7F84C31D3F822
S315080303300031302B1BD0302B15D8102B02D0202B95
S3150803034007D010E0274B9B6A264A43F4003393628F
S315080303500EE0D7F84C313033184603F075F80346E8
S3150803036087F85B3104E0012387F85B3100E000BFBF
S3150803037097F85B31002B0DD11A4BD3F8E43023F0F1
S315080303803002D7F84C31D3F8003116491343C1F874
S31508030390E43003E097F85B3187F85A31D7F84C31E4
S315080303A0D3E900230021396003F008037B60D7E90A
S315080303B000120B4613430CD00A4BD3F8E83023F04C
S315080303C0C002D7F84C31D3F8FC3006491343C1F8B9
S315080303D0E83097F85A31184607F5B077BD46BDE8B1
S315080303E0B08F00BF000C024480B48BB000AF7860B6
S315080303F0AD4B5B6BC3F308033B62AB4B9B6A03F0E2
S315080304000303FB61A84B9B6A1B0A03F03F03BB610B
S31508030410A54B9B6A03F010037B61A34B9B6BDB081D
S31508030420C3F30C037A6902FB03F307EE903AF8EE7B
S31508030430677AC7ED047ABB69002B00F02681FB694E
S31508030440032B53D0FB69032B6FD8FB69012B03D00E
S31508030450FB69022B2BD068E0934B1B68DB0803F080
S315080304600303924A22FA03F3FB60FB6807EE903A0A
S31508030470F8EE676ABB6907EE903AF8EE677A86EE96
S31508030480A77A3B6A07EE903AF8EE676A97ED046A2D
S31508030490DFED875AC6EE257A76EEA77AF7EE006A77
S315080304A077EEA67A67EE277AC7ED097A68E0BB691D
S315080304B007EE903AF8EE677ADFED7E6A86EEA77A5C
S315080304C03B6A07EE903AF8EE676A97ED046ADFED42
S315080304D0785AC6EE257A76EEA77AF7EE006A77EEAD
S315080304E0A67A67EE277AC7ED097A49E0BB6907EE6C
S315080304F0903AF8EE677ADFED706A86EEA77A3B6A7A
S3150803050007EE903AF8EE676A97ED046ADFED685AE4
S31508030510C6EE257A76EEA77AF7EE006A77EEA67A1E
S3150803052067EE277AC7ED097A2AE05F4B1B68DB0873
S3150803053003F003035D4A22FA03F3FB60FB6807EE45
S31508030540903AF8EE676ABB6907EE903AF8EE677A6F
S3150803055086EEA77A3B6A07EE903AF8EE676A97ED56
S31508030560046ADFED535AC6EE257A76EEA77AF7EED6
S31508030570006A77EEA67A67EE277AC7ED097A00BF8F
S31508030580494B1B6803F00073B3F1007F21D1464B37
S315080305909B6A03F48033002B17D0434B5B6B5B0AD0
S315080305A003F07F0307EE903AF8EE677AB7EE007A20
S315080305B037EE877AD7ED096AC6EE877AFCEEE77ACD
S315080305C017EE902A7B681A6006E07B6800221A6099
S315080305D002E07B6800221A60334B1B6803F0007342
S315080305E0B3F1007F21D1304B9B6A03F40033002B10
S315080305F017D02D4B5B6B1B0C03F07F0307EE903A6A
S31508030600F8EE677AB7EE007A37EE877AD7ED096A96
S31508030610C6EE877AFCEEE77A17EE902A7B685A606D
S3150803062006E07B6800225A6002E07B6800225A6073
S315080306301D4B1B6803F00073B3F1007F21D11A4BDE
S315080306409B6A03F48023002B17D0174B5B6B1B0E97
S3150803065003F07F0307EE903AF8EE677AB7EE007A6F
S3150803066037EE877AD7ED096AC6EE877AFCEEE77A1C
S3150803067017EE902A7B689A6010E07B6800229A60DE
S315080306800CE07B6800229A6008E07B6800221A6007
S315080306907B6800225A607B6800229A6000BF2C3769
S315080306A0BD465DF8047B7047000C02440090D003F6
S315080306B0000000460024744A001B374B80B48BB0F5
S315080306C000AF7860AD4BDB6BC3F308033B62AB4B00
S315080306D0DB6A03F00303FB61A84BDB6A1B0A03F01F
S315080306E03F03BB61A54BDB6A03F010037B61A34B96
S315080306F01B6CDB08C3F30C037A6902FB03F307EEEF
S31508030700903AF8EE677AC7ED047ABB69002B00F0D6
S315080307102681FB69032B53D0FB69032B6FD8FB692F
S31508030720012B03D0FB69022B2BD068E0934B1B6884
S31508030730DB0803F00303924A22FA03F3FB60FB6820
S3150803074007EE903AF8EE676ABB6907EE903AF8EE59
S31508030750677A86EEA77A3B6A07EE903AF8EE676AF7
S3150803076097ED046ADFED875AC6EE257A76EEA77A01
S31508030770F7EE006A77EEA67A67EE277AC7ED097A67
S3150803078068E0BB6907EE903AF8EE677ADFED7E6AB2
S3150803079086EEA77A3B6A07EE903AF8EE676A97ED14
S315080307A0046ADFED785AC6EE257A76EEA77AF7EE6F
S315080307B0006A77EEA67A67EE277AC7ED097A49E0E3
S315080307C0BB6907EE903AF8EE677ADFED706A86EE54
S315080307D0A77A3B6A07EE903AF8EE676A97ED046ADA
S315080307E0DFED685AC6EE257A76EEA77AF7EE006A43
S315080307F077EEA67A67EE277AC7ED097A2AE05F4B82
S315080308001B68DB0803F003035D4A22FA03F3FB6064
S31508030810FB6807EE903AF8EE676ABB6907EE903A0B
S31508030820F8EE677A86EEA77A3B6A07EE903AF8EE11
S31508030830676A97ED046ADFED535AC6EE257A76EEB4
S31508030840A77AF7EE006A77EEA67A67EE277AC7EDF8
S31508030850097A00BF494B1B6803F00063B3F1006FC5
S3150803086021D1464BDB6A03F48033002B17D0434B65
S31508030870DB6B5B0A03F07F0307EE903AF8EE677AC1
S31508030880B7EE007A37EE877AD7ED096AC6EE877A26
S31508030890FCEEE77A17EE902A7B681A6006E07B6817
S315080308A000221A6002E07B6800221A60334B1B6839
S315080308B003F00063B3F1006F21D1304BDB6A03F415
S315080308C00033002B17D02D4BDB6B1B0C03F07F0378
S315080308D007EE903AF8EE677AB7EE007A37EE877A3C
S315080308E0D7ED096AC6EE877AFCEEE77A17EE902A01
S315080308F07B685A6006E07B6800225A6002E07B68E0
S3150803090000225A601D4B1B6803F00063B3F1006FA6
S3150803091021D11A4BDB6A03F48023002B17D0174B1C
S31508030920DB6B1B0E03F07F0307EE903AF8EE677A4C
S31508030930B7EE007A37EE877AD7ED096AC6EE877A75
S31508030940FCEEE77A17EE902A7B689A6010E07B68DC
S3150803095000229A600CE07B6800229A6008E07B68B4
S3150803096000221A607B6800225A607B6800229A601C
S3150803097000BF2C37BD465DF8047B7047000C024464
S315080309800090D003000000460024744A001B374B2E
S3150803099080B48BB000AF7860AD4B5B6CC3F30803D0
S315080309A03B62AB4B1B6B03F00303FB61A84B1B6B4F
S315080309B01B0A03F03F03BB61A54B1B6B03F0100334
S315080309C07B61A34B9B6CDB08C3F30C037A6902FBBD
S315080309D003F307EE903AF8EE677AC7ED047ABB6934
